:020000040800F2
:100000000000022049A30508399A00080556020895
:10001000F9A30508F9A30508F9A3050800000000E5
:100020000000000000000000000000001DB10008FA
:100030001FB100080000000021B10008A91001084C
:10004000F9A30508F9A30508F9A30508F9A305080C
:10005000F9A30508F9A3050893FD000897FD00081A
:10006000F9A305089BFD00089FFD0008F1A000080A
:1000700005A1000819A100082DA1000841A1000850
:1000800055A1000869A10008F9A3050800000000B7
:10009000000000000000000000000000A3FD0008B8
:1000A00029A0000851A0000879A0000813A00008AA
:1000B000A1A00008B5A00008C9A00008F9A3050880
:1000C000F9A30508F9A30508F9A30508F9A305088C
:1000D000F9A30508559B0008619B0008000000007B
:1000E000A7FD0008F9A3050823B1000800000000DF
:1000F0000000000000000000000000007DA10008DA
:1001000000000000F9A30508DDA00008F9A3050818
:1001100000000000000000000000000000000000DF
:1001200091A10008A5A10008B9A10008CDA100086F
:10013000E1A1000800000000000000000000000035
:100140000000000000000000000000006DB1000889
:10015000F5A1000809A200081DA20008F9A30508DE
:10016000F9A30508F9A3050800000000000000003D
:10017000000000000000000000000000000000007F
:1001800000000000F9A305080000000000000000C6
:08019000F9A30508F9A3050815
:0801980038940500010000008D
:1001A000A45001200201000002001400C4500120EC
:1001B0000202000002001400E4500120020A0000C4
:1001C0000200140004510120020600000200140085
:1001D00024510120020700000200140044510120B4
:1001E0000203000004001400645101200208000012
:1001F0000400140084510120010B0000000077006E
:10020000A4510120010C000000007600C45101201F
:100210000110000000007600E4510120010D0100F2
:100220000000770004520120011200000000760057
:10023000245201200114000000001E00445201203D
:10024000011A000000000D0064520120011C000092
:1002500000000E0084520120011D000000001E005D
:10026000A45201200117000000000C00C45201201C
:100270000118000000000E00E452012001290100D5
:100280000000180004530120012100000000480074
:1002900024530120012200000000490044530120A2
:1002A0000123000000004A006453012001240000E3
:1002B00000004B00845301200125000000004C0089
:1002C000A45301200126000000004D00C45301206A
:1002D0000127000000004E00E45301200128000027
:1002E00000004F0004540120012C000000002900F0
:1002F00024540120012D0100000029004454012054
:10030000012E01000000700064540120012F010043
:100310000000520084540120013001000000280038
:10032000A45401200131010000002800C454012020
:100330000235040000012C00E454012001340000C7
:1003400000003C000455012001370000000020009F
:10800000D0E907239A423CBFC1685218D01A704782
:10801000D0E9092300699A4238BF1218D31A0138EF
:10802000C01A7047D0E90902131A584258417047E4
:10803000036A41690246C85CD16801338B4228BF9C
:10804000002313627047436A8269D154436A02690C
:108050000133934228BF0023426B4362D36843F04D
:108060008003D3607047436B188810F010001EBF68
:108070001A889B8801207047436B99891A88890662
:1080800010B592B2044607D5900605D5E26A2AB328
:108090009888216B80B29047636B99891A8809068A
:1080A00092B210D510060ED5D4E909128A4223D017
:1080B000A169895CC9B2998021690132B2FBF1F0F2
:1080C00001FB1022A262998A1A88C90592B204D5CE
:1080D000D20744BF4FF6F7721A8010BD9B88E26941
:1080E0006169DBB28B54E369E2680133B3FBF2F1FF
:1080F00002FB1133E361CFE7DA6822F08002DA6035
:10810000E1E7036941681F2B30B54FF0200285BFBE
:10811000A3F120054C680C68AA4098BF9A402242FF
:108120001DD0826900201074D0688468206820F017
:1081300001002060546820686579094C828934F810
:10814000154092B21F2B22EA0402828188BF203B95
:108150004FF020028BBF9A409A40CA608A6030BDBF
:10816000B00F06080E4BDA68D20310D4DA68D106D5
:108170000FD4DA68D2050ED4DA6812F0E00F0CD111
:10818000DB6813F0020F0CBF0920082070470120A4
:10819000704706207047022070470720704700BFD5
:1081A000003C024007B509238DF80730FFF7DAFFDE
:1081B0008DF807009DF80730012BF7D09DF80700D8
:1081C00003B05DF804FB838A028B9BB243EA02434F
:1081D00099430CBF01200020704782B00023019317
:1081E0000093012300900193019B63B1009A21F059
:1081F0007F4314320092009A12681A4214BF012081
:10820000002002B07047009A1832F3E770477047B9
:1082100001207047034BD3E90003C01AC0F30A00E2
:10822000704700BFC8180020054AD2E900138B42EE
:10823000FDD0D1180133C3F30A03087A53607047A5
:10824000C8180020044BD3F8080820B1D3F8080858
:10825000431F584258417047C8180020012380F836
:1082600049307047044BD3E90003C01AC0F30A0039
:10827000C0F50060704700BFC818002010B5D0F8E6
:10828000E83504461B699847032384F8123100201F
:1082900010BD08B590F8123180F81331042380F82E
:1082A0001231D0F8E835DB689847002008BD08B5E2
:1082B000D0F8E435DB6903B19847002008BD08B564
:1082C000D0F8E4351B6A9847002008BD08B5D0F8FF
:1082D000E4355B6A9847002008BD70B504460D463A
:1082E000164651F0D5F9C3B201335B0033802B70D1
:1082F00003236B70601E0223002410F8011F01B9D4
:1083000070BD5A1CD2B2E9540233AC54DBB2F4E76C
:1083100010B5074C2068FF2808D00649D1F80C2872
:1083200001F5016100F07AF8FF232360002010BD01
:1083300000000020C8180020432301480B8070472C
:1083400004000020122301480B80704747000020E2
:10835000042301480B8070475900002010B5044CDD
:1083600004480A462146FFF7B8FF204610BD00BF6B
:10837000E0200020A0B4060810B5044C04480A46CA
:108380002146FFF7AAFF204610BD00BFE0200020D5
:10839000AFB4060810B5044C04480A462146FFF75E
:1083A0009CFF204610BD00BFE0200020B4B40608AA
:1083B00010B5044C04480A462146FFF78EFF2046BC
:1083C00010BD00BFE0200020BEB4060810B5044C6C
:1083D00004480A462146FFF780FF204610BD00BF33
:1083E000E0200020C9B40608704770477047704706
:1083F00070477047044B00200522C3F80828C3F8D3
:108400001809C3F81C097047C8180020024B002047
:10841000C3F80808704700BFC8180020212838B5E5
:108420000C461BD022282BD0202815D1A1B1072A19
:1084300012D11A4DD5F81C3913B10968002098479C
:108440002368C5F82039237985F82439637985F8BC
:108450002539A37985F82639002038BD0029FBD0BD
:10846000072AF9D10D4BD3F820290A6093F8242963
:108470000A7193F825294A7193F826398B71EBE735
:108480000029E9D0022AE7D1044BD3F81839002B90
:10849000E2D0098800209847DEE700BFC818002016
:1084A00030B50E4CD4E900329A1AC2F30A020A44DB
:1084B000B2F5006F10D801440022814203D102B10D
:1084C0002360002030BDE21810F8015B1572013303
:1084D000C3F30A030122F0E70220F3E7C8180020E3
:1084E000034BD3F8280908B103691847704700BF48
:1084F000C8180020034B93F85009003818BF01201A
:10850000704700BFC8180020034B93F85009032898
:1085100094BF002001207047C81800200048704711
:108520001C220020837B042B0DD0074BD3F898200E
:108530000132C3F89820426004228273D3F89C2051
:108540000132C3F89C2070479C6000202023014822
:108550000B8070475D000020122301480B8070479C
:108560007D000020042301480B8070478F0000200D
:108570000A4608B5044920B90448FFF7AEFE024890
:1085800008BD0348F9E700BF4C220020D7B4060815
:10859000EFB4060810B5044C04480A462146FFF71C
:1085A0009CFE204610BD00BF4C22002007B50608E7
:1085B00010B5044C04480A462146FFF78EFE2046BB
:1085C00010BD00BF4C2200201AB5060810B5044C9F
:1085D00004480A462146FFF780FE204610BD00BF32
:1085E0004C22002025B50608002370B54D1C1E4600
:1085F000040FB0F1204F34BF3034373401F813404A
:1086000005F813600133DCB2A2424FEA0010EFD844
:1086100070BD1A2310B50B80094BD3F8E807D3F8C7
:10862000EC2780180AD0D3F8EA4706490822FFF75A
:10863000DBFF042210312046FFF7D6FF024810BDB1
:1086400000F0FF1F950000209300002008B5FFF701
:1086500047FF013840B208BD002070470020704736
:1086600070477047D0ED007AD0ED036A30EE677A3C
:10867000E6EE877AB0EE670AC0ED007A704790EDBB
:10868000017AB5EE407AF1EE10FAF0EE407A09D1B7
:108690009FED0E7A60EE870AF7EE006A86EEA07A0A
:1086A00080ED017A90ED017A90ED000A80ED021ADA
:1086B00031EE077A77EEC07AC1EE076AA6EEA70A16
:1086C000C0ED036A80ED000A704700BFDB0FC940B0
:1086D000D0ED017AD0ED036A30EE670AE6EE807ADB
:1086E00090ED000AC0ED017AB0EE677AD0ED027A23
:1086F00037EE677AE6EE877AC0ED027A77EEC07AD7
:10870000A6EEA70A80ED000A7047D0ED056AD0ED0D
:10871000017A90ED026AD0ED045AB0EE407A26EE6E
:10872000A70AD0ED007A80ED057AA7EE870AD0ED92
:10873000067AC0ED066AA6EE270AD0ED077A90ED1C
:10874000036AA6EE670A90ED086AC0ED087AA5EE06
:10875000C60A80ED070A7047B0EE407AD0ED007A85
:1087600090ED050AD0ED016AA7EE870AD0ED037AF5
:1087700067EEC07AE6EE877AD0ED066A76EEA77AE3
:10878000D0ED026AC0ED057AD0ED047A67EEC07ACA
:10879000E6EE877AC0ED067A704703685A1C0260DD
:1087A0001970704703690133012B036108D1DFEDB4
:1087B000117A80ED010A80ED000AC0ED027A70475F
:1087C00090ED006A07EE903A70EE466AF8EEE77AAE
:1087D00086EEA77AD0ED027A37EE067A30EE470AB7
:1087E00080ED017AE6EE807AB0EE470AC0ED037ABA
:1087F000E1E700BF0000000003685A1C0260197026
:108800007047007970470079C0F3401070470079D5
:10881000400970472DE9F843D0F81480074689468F
:10882000B8F1000F57D10568C5F30D0606B3D9F8A6
:108830000060FFF7B7FC092840F08680444C2369AC
:1088400023F440732361236943F400732361236994
:1088500043F0010323612E60FFF7A4FC236909287C
:1088600023F0010323616FD13B6804333B6032E0A6
:10887000384B9D4229D303F580439D4224D303F511
:1088800080439D422AD3344B9D4229D903F580333E
:108890009D4227D903F500339D4225D903F50033C6
:1088A0009D4223D903F500339D4221D903F50033BE
:1088B0009D421FD903F580239D421DD9B5F1016F5B
:1088C0001CD305200AF020FE0826FFF76BFC0928C0
:1088D00016D04FF0FF384046BDE8F8831026F4E785
:1088E0001826F2E72026F0E72826EEE73026ECE708
:1088F0003826EAE74026E8E74826E6E75826E4E790
:10890000134C236923F440732361236943F40073F8
:108910002361236923F0F80323612369334343F080
:1089200002032361236943F480332361FFF73AFC98
:10893000236923F0020323612369092823F0F80344
:1089400023613FF474AFC4E76FF00108C3E700BFD1
:10895000003C024000400008FFFF000803682DE9CA
:10896000F0410D46416813448B42044619D8AE18B5
:1089700000F10C074FF00008B54202D16069BDE874
:10898000F08123695A1C2261234415F8011B1973D5
:10899000042AF1D139462046FFF73CFFC4E90480A0
:1089A000EAE74FF0FF30EAE72DE9F0479846444BFD
:1089B000914603EB800205469468002C51D0283381
:1089C000636004F13E03A36104F59F73E3614FF418
:1089D0008073C4E90433236894F83D00E160A36325
:1089E00007F068FA064694F8440294F83CA0271D64
:1089F00008B14DF051FC94F8450208B14DF04CFC23
:108A0000D4F840321BB12F4A116B0B43136318F09B
:108A1000080F2FD00135EDB21EB140F20673F3807E
:108A2000357218F0100F94F846221DD002213046FE
:108A300007F000FAD4F8482294F9471294F8473224
:108A400012010029D2B236DB1F49C81880F8002372
:108A50005809012203F01F0302FA03F341F8203002
:108A60003C462046BDE8F08718F0200F0CBF3221AD
:108A70001221DCE719F0020F0CD06B1CDBB21EB127
:108A800040F20652F280337294F8462202213046B8
:108A900007F0D0F919F0010FCCD0504607F00AFAD0
:108AA0000135EDB218B140F20663C380057294F847
:108AB00046220221BCE7054903F00F03CA54CFE761
:108AC000B00F06080038024000E100E014ED00E0BD
:108AD0002DE9F341038A8689B6B205460C461E404D
:108AE0004FF0004816B902B0BDE8F081B6FA86F33F
:108AF00028FA03F2D24391B2298216401B3B002C84
:108B00003ED0042BEED8DFE803F037312B250300ED
:108B1000E368EF6A23B19B6813B1B9B2201D98478F
:108B2000636A2BB19B681BB1B9B204F11C00984772
:108B3000E36B2BB19B681BB1B9B204F134009847C9
:108B4000636D002BCED09B68002BCBD0B9B204F163
:108B50004C0003E0E368696B5B68201D9847C1E740
:108B6000636AA96B5B6804F11C00F7E7E36BE96BD0
:108B70005B6804F13400F1E7636D296C5B68E6E73C
:108B8000042B06D8DFE803F00D0B09070300EB6A9E
:108B90000193019BA6E76B6BFAE7AB6BF8E7EB6B16
:108BA000F6E72B6CF4E790F84820531C0244DBB244
:108BB00080F8483082F8341090F849200AB1132B1D
:108BC00001D950F017BC7047002280F8492050F0BE
:108BD00011BC70B5124D044695F8833A002BFBD1B9
:108BE0006618B44204D1002070BD01200AF032F9A9
:108BF000D5F8843AD5F8882A0133C3F30A0393429F
:108C0000F3D0D5F8843A14F8012B2B4483F88C2A3E
:108C1000D5F8843A0133C3F30A03C5F8843AE0E790
:108C2000C818002038B50C461146FFF70BFB48B1B9
:108C3000054D002AD5F8943104DD2046FFF7C9FF21
:108C4000D5F8943138BD00BFC0290020F0B585B0FB
:108C5000D0F8CC1590F8CC650291D0F8D0150391DE
:108C6000012180F8111106F01F01B0F8D22590F80B
:108C7000CD75B0F8CE35B0F8D055C0F840210129F7
:108C8000044600F00981022900F01A81002940F011
:108C90009381092F5ED8DFE817F0B600F4005D007D
:108CA000C8005D0057000A005D00A90076001D0A9B
:108CB000022DADF806200BD0032D25D0012D49D172
:108CC000D0F8EC351B68A0780DF10601984709E053
:108CD000D0F8E43580789B6A0DF10601984745701D
:108CE000C4F8F005BDF80620002A47D0BDF80E30C4
:108CF000002B43D09A4228BF1A46ADF80620014601
:108D0000204650F065FA39E0DBB2052B22D8DFE8C7
:108D100003F003070B0F1317D0F8EC355B68D2E7AD
:108D2000D0F8EC359B68CEE7D0F8EC35DB68CAE7C5
:108D3000D0F8EC351B69C6E7D0F8EC355B69C2E7C3
:108D4000D0F8EC359B69BEE72A4303D190F81211A5
:108D5000032903D1204650F065F90FE003F07F05A9
:108D6000016980F8145163F30A120B681A430A6010
:108D700050F042FA2DB1022384F81231002005B0E0
:108D8000F0BD0123F8E7D9B28D4D012985F898117E
:108D9000E0D890F81231022B0FD0032BDAD1C1B9F1
:108DA000022380F81231D0F8E43580F810115B68A6
:108DB0009847204650F020FAE0E70029F9D0012139
:108DC000032380F8101180F81231204650F0ECF89F
:108DD000EFE790F810110129EBD0D0F8E4355B688B
:108DE000984795F8981184F81011EEE7012AB1D14F
:108DF00090F81231022B04D0032BABD100F588710F
:108E00007EE770497CE790F81231023B012BA1D834
:108E10006B4B0022C3F8A021D0F8182112B1022216
:108E2000C3F8A021684902226AE7012B08D1C4F8DF
:108E30001831D4F8E43502A99B6820469847B8E772
:108E4000022B9BD1EBB2002B98D103692D0A023D76
:108E50005A68032D13D8DFE805F0020C0E10022328
:108E600063F30612564BC3F8A421012384F816318C
:108E70009FE70323F4E70423F2E70523F0E7012348
:108E8000EEE790F81221023A012A3FF663AF012B78
:108E90007FF474AF0023CAE790F81231032B7FF4FC
:108EA00059AFEDB2012D3FF655AFD0F8E43502A928
:108EB0009B689847BDF80E30002B7FF45FAF78E7D2
:108EC00006F06006202EE9B205D1D0F8E43502A9FB
:108ED0009B68984752E7012F35D0032F23D0002FEE
:108EE0007FF44CAF90F81231022B5FD0032B7FF44C
:108EF00031AF15F0800F4FF028031BBF01F07F0149
:108F000003FB010103FB010191F81E3108BF91F839
:108F100076332B49003B18BF0123C1F8A831022248
:108F200001F5D471ECE690F81221022A3ED0032A12
:108F30007FF410AF002B7FF47CAF4A063FF479AF8B
:108F400050F03EF875E790F81221022A2ED0032A3D
:108F50007FF400AF002B7FF411AF11F07F023FF4DC
:108F600028AF6DB22823002DB5BF03FB020303FB1E
:108F7000010303F58E7303F55D73002199701A7078
:108F8000E90F00EB82025970002DB4BF9269526D57
:108F9000D9781368023923F4001301298CBFC3F375
:108FA0000071012161F31C73136042E74B063FF42B
:108FB000E5AE50F005F8E1E606F08001F9E700BF04
:108FC000C02900205C2B0020602B002010B5044637
:108FD00071BB90F81131032B1BD1D0F89023D0F83E
:108FE0007C339A4217D9C178012908BFD0F8801381
:108FF000A2EB030204BFC918C0F88013934228BF34
:109000001346C0F890239BB2D0F88023002150F083
:10901000A3F9002010BDD0F8E4351B6923B190F806
:109020001221032A00D19847204650F0E5F8F0E7D6
:10903000D0F8E4359B69002BEBD090F81221032A7D
:10904000E7D19847E5E770B50A7812F06003054666
:109050000C4628D0202B2DD1CB884E78EBB11206B0
:109060000AD51D491A463046FFF7D8F9E2881A4951
:10907000284650F0ADF80EE0184A1660184A032151
:10908000C2F80C3880F81111C0E9E43302F501622E
:10909000002150F061F9002070BD022211443046D9
:1090A000FFF7BCF9F7E74B780A2B08D00B2B09D058
:1090B000062BF0D128464FF0B5FF0220ECE7094916
:1090C0000122D6E78B781BB9074AC2F8AC31E2E738
:1090D0004FF0A8FFDFE700BFD820002000000020ED
:1090E000C81800206C2B0020C029002038B5282388
:1090F00003FB0101074DB1F88C1304462846FFF726
:10910000CFF9204640232A46012150F025F90020BE
:1091100038BD00BF702B002070B50E4BD3F8FC217A
:1091200093F8F051044632B193F800322B4302D148
:1091300001214FF045FF812120464FF041FF022DD4
:1091400007D12046044ABDE870401F23012150F09A
:1091500003B970BDC0290020B42B0020002310B536
:109160001946044640224FF095FF402280212046B8
:1091700000234FF08FFF012384F81231D4F8E83533
:10918000A0785B689847002010BD38B5402204469F
:10919000022381214FF07EFF20460223402201213D
:1091A0004FF078FF20460323082282214FF072FF00
:1091B000084B0222002583F84B2083F84C500121F4
:1091C000FFF718F92046044A402350F0C5F8284616
:1091D00038BD00BF00000020702B002010B5812199
:1091E00004464FF02DFF204601214FF029FF204675
:1091F00082214FF025FFFFF709F9002010BD10B5BF
:10920000812104464FF01CFF204601214FF018FF3A
:10921000024B002083F8140210BD00BFC0290020BB
:10922000F8B5224C94F8832A012A03462ED1204F08
:10923000D7F8185215B984F8835A23E0402D23D863
:10924000AEB2402E02D1022284F8832AD4F8881AC2
:10925000184A0A44C3E9542240F201110022A3F83B
:109260004411C3E9566203F5A27118464FF0DBFFC3
:10927000D4F8883A3344C3F30A03AD1BC4F8883AE0
:10928000C7F818520020F8BD4026DFE7022AF9D1BE
:10929000002540F20112C0E95455C0E95655A0F826
:1092A000442100F5A2714FF0BEFFC4E7C8180020AA
:1092B000C029002054230020F8B5284FD7F81C32CD
:1092C0000F2B03F1010203D0C7F81C220020F8BDC8
:1092D000234C0023C7F81C3294F8833A002BF5D1B5
:1092E000D4F8882AD4F8843A9A42EFD0D4F8882A5D
:1092F000D4F8843A9A4295BFD4F8845AD4F8885A5C
:10930000D4F8883AC5F5006598BFED1A402D22D8EB
:10931000AEB2402E0CBF02230123D4F8882A84F871
:10932000833A104B1344C0E9543340F20112002336
:10933000C0E95663A0F8442100F5A2714FF073FF15
:10934000D4F8883A3344C3F30A03AD1BC4F8883A0F
:10935000C7F81852BAE701234026DEE7C0290020EB
:10936000C818002054230020064BD3F880391A79FE
:10937000022A05D19A68920702D558694FF0D2BAED
:10938000704700BFC818002010B50A4CD4F88009F7
:1093900006F0D4FB58B9D4F880090379022B08D120
:1093A00083689B0705D5BDE8104007F0ADBE00BF40
:1093B000ECE710BDC818002073B50A4E441C002508
:1093C000D6F88009012300220DF1070150F062F860
:1093D0009DF80700FF2802D10135A542F0D102B067
:1093E00070BD00BFC818002070B5044608200D46A7
:1093F000FFF7E2FFFF2812D0FE2812D10A4E2B46BB
:10940000D6F880090022214650F044F80022D6F810
:1094100080090223114650F03DF8002070BD012064
:10942000FCE70220FAE700BFC818002037B5124D4C
:109430004FF6FF530024D5F88009ADF8043001AA97
:1094400002232146C5F84C4950F024F80120FFF7CB
:10945000B3FFFF2805D1042385F85039022003B05B
:1094600030BD092385F85039044BD3F89431C5F841
:1094700040392046F3E700BFC8180020C02900206B
:1094800013B540F040038DF800300B0E8DF801301D
:109490000B0C8DF802300B0A8DF80330952304462F
:1094A0008DF804108DF805304CF0DCFB00B964B980
:1094B00007480623D0F880096A4600214FF0EAFFEA
:1094C0000820FFF779FF02B010BDFF20FBE700BFC7
:1094D000C81800202DE9F041194C1E4694F8503967
:1094E000042B0546884617461CD1FFF73DFF94F82C
:1094F0004639FBB969021120FFF7C2FFE0B9052325
:1095000084F850390F4BC4F82C89D3F89431C4F83F
:109510003059C4F83879C4F83C69C4F8403901209E
:10952000BDE8F081082B03D1FFF780FF0228DCD0D3
:109530000020F5E72946DEE7FFF726FFF8E700BF42
:10954000C8180020C029002038B500220D2335217D
:10955000022006F0D7FC224CC4F8800910B984F828
:10956000500938BD002106F077F9012009F072FC9E
:10957000D4F88059686906F029FC95F9103019482B
:10958000194D142202FB03000022D0F8B0000A2378
:1095900011464FF055FFD4F8800906F0CFFA50B9C4
:1095A000124B84F84409D3F89431C4F840390123AC
:1095B00084F85039D5E7013DEDD1D4F88009022176
:1095C00006F04AF9D4F8800906F019F994F84439FC
:1095D000C4F88059013384F8505984F84439C0E7FD
:1095E000C818002000000020A1860100C02900202A
:1095F00038B5134C0023A07BE0B125688D4219D10A
:10960000104C03F581751AB904EB0514A27138BD2D
:1096100004F1180101EB43239A4209D1831E5842F9
:10962000584104EB05144FF0C1FB0123A371EEE791
:109630000020F6E70133082B04F11004DBD1E6E744
:10964000B46000209C500020174838B5002380F8F3
:10965000A03000F1180425688D421ED1A57B032D92
:109660001BD1124C03F581754AB904EB0514042390
:10967000A371D0F89C300133C0F89C3038BD04F1A0
:10968000180000EB4320131A5842584104EB05140C
:109690004FF08CFB0123A371F0E70133082B04F199
:1096A0001004D8D1EAE700BF9C6000209C50002045
:1096B000F8B50446144EFFF7A2FD204602234022CF
:1096C00081214FF0E7FC40220121204602234FF088
:1096D000E1FCD6F8203200251B6886F81452284693
:1096E00086F8F0519847E76838464FF053FE384601
:1096F00001214FF065FE20461F2306F5FA72012175
:109700004FF02AFE2846F8BDC02900202DE9F84F69
:109710000E460121084617461D4606F083FDDFF878
:1097200044800024A54206DC0021012006F07AFDD9
:109730000020BDE8F88F06EB442A07EB0409D8F8AF
:109740002839002BFBD0D3F804B000231A46514629
:109750004846D8470028F2D0FEF7C2FE0028FBD0CA
:109760000134DFE7C81800202DE9F84F0E4601212B
:10977000084615461F4606F055FDDFF848A00024B0
:10978000A74218DD06EB442905EB040801E0FEF7CB
:10979000A7FEDAF8283943B1D3F80CB000231A46F3
:1097A00049464046D8470028F1D1FEF799FE0028E7
:1097B000FBD00134E4E70021012006F033FD002056
:1097C000BDE8F88FC8180020024BD3F8240207F038
:1097D000C3BB00BFC02900200068F022FF2107F0B2
:1097E000C3BCCB4341EA0311CAB20068D22107F0DF
:1097F000BBBC0068B422FF2107F0B6BC0A46006873
:10980000A52107F0B1BC5521F8E700689622FF2199
:1098100007F0AABC0A460068872107F0A5BCCA0168
:10982000006802F08002782107F09EBC38B504463B
:10983000154600680A46E12107F096FC30B1206821
:109840002A46FF21BDE8384008F070BB38BD0A4603
:10985000E121EBE70A46C321E8E738B5021D0D46D2
:10986000F0210446FFF7E2FF08B123792B7038BDE1
:10987000F8B504460E461546071D20683A46FF21F6
:1098800008F054FB30B116B12379DB07F5D40DB1E4
:1098900023792B70F8BD00220121E9E710B50446B9
:1098A000FFF7A7FF18B12046BDE81040F3E710BD51
:1098B00010B50446FFF7A2FF18B12046BDE81040DE
:1098C000E9E710BD70B506460C468D18AC4201D1D3
:1098D000012006E014F8011B3046FFF7E9FF0028DD
:1098E000F4D170BDCC21E3E738B504460D46FFF74F
:1098F0008CFF40B12046FFF7CEFF20B1294620461D
:10990000BDE83840A3E7002038BD70B506460C46D8
:109910008D18AC4201D1012006E021463046FFF708
:10992000E3FF01340028F4D170BD38B50546144674
:10993000FFF770FF2846FFF7AEFF20B11CB12B796F
:10994000C3F34013237038BD10B50446FFF7A6FFDC
:1099500038B12046FFF7C6FF18B12046BDE81040D9
:1099600099E7002010BD73B50546CDE90023FFF748
:1099700095FFA8B12846FFF746FF88B12846FFF7B4
:109980008AFF68B16E46082416F8011B2846FFF7C7
:109990008FFF28B1013C14F0FF04F5D102B070BD77
:1099A0000020FBE7C90138B501F0800104461546E7
:1099B000FFF735FF08B9002038BD002201212046FD
:1099C000FFF756FF0028F6D023795B092B70F3E7E9
:1099D00010B5021D0446FF21006808F0A7FA18B16F
:1099E0002079C04300F0010010BD0F49D1F8883044
:1099F00043F47003C1F888300C4B1A68002042F021
:109A000001021A6098601A6822F0847222F480328F
:109A10001A60074A5A601A6822F480221A60D860D5
:109A2000044B8B60704700BF00ED00E0003802403F
:109A30001030002400000008704782B0002301931A
:109A400000933C4B1A6842F480321A601A6802F4A0
:109A500000320092019A01320192009A1AB9019AD9
:109A6000B2F5A04FF2D11B6813F4003318BF0123E5
:109A70000093009B012B57D12E4B2F491A6C42F0BB
:109A800080521A640A6842F440420A609A689A60F6
:109A90009A689A609A6842F480529A60274A5A609B
:109AA0001A6842F080721A601A689001FCD5244A44
:109AB00040F2027111609A6822F003029A609A687B
:109AC00042F002029A601B4B9A6802F00C02082ACC
:109AD000FAD19A6802F00C02042A27D0082A27D16A
:109AE00059685A685B684902C3F388134CBF15492B
:109AF000154902F03F02B1FBF2F253430D4A52689E
:109B0000C2F3014201325200B3FBF2F3094A9168F9
:109B10000E4AC1F303110A4492F85820D3400C4A6C
:109B2000C2F8003102B0704700BFFDE7054BEDE71A
:109B3000054BEBE70038024000700040193040044C
:109B4000003C024040787D010024F400B00F06087C
:109B5000000000200148FEF78FBA00BF0801002076
:109B60000148FEF789BA00BF54030020024B586F2A
:109B7000C0F30070704700BF003802407047064ACB
:109B8000002352F83310814201D1D8B2704701331B
:109B90000E2BF6D1FE20704718100608704770B5DE
:109BA000002828D04C684CB9426815685679AB89B2
:109BB00002229BB2B24023EA0203AB818A683AB91F
:109BC00043681D68AB8923F001031B041B0CAB81A8
:109BD000816044B1436819685D798C890223AB4088
:109BE00023439BB28B8132B143681A6893899BB23D
:109BF00043F00103938170BD0B4B30B51A4600242E
:109C00001D79854208D1DD68294203D0142303FB66
:109C1000042030BD0029F9D001340A2C03F11403CB
:109C2000EED10020F5E700BF9C0500200028ACBF66
:109C300000F16040064B4FEA0111ACBF00F56140F6
:109C400000F00F00C9B2B4BF195480F80013704778
:109C500014ED00E038B503681B681C68244B07EE60
:109C6000902A93ED407AF8EE677AB8EE477A013998
:109C700087EE270A8DB2DFED1F7A30EE270A51F00A
:109C800099F91D4A23880138944280B29BB212D0C0
:109C900002F5806294420ED0B4F1804F0BD0A2F551
:109CA0008032944207D002F58062944203D002F5DC
:109CB0008062944206D123F070039BB223F4407378
:109CC0009BB206E00D4A944203D002F580629442B2
:109CD000F4D12380084BE5629C42208503D003F534
:109CE00080639C4201D1002323860123A38238BDD7
:109CF000000000200AD7233C000001400010004073
:109D0000F0B543689A795D7912F0040002F0020C14
:109D100011BF0022E6464FF4807284460FBF012433
:109D2000964604201446032D38D8DFE805F00238A3
:109D300072AC1B681D8C25F001052D042D0C1D84B3
:109D40001D8C9F881E8B25F002052D0444EA0E040D
:109D50002D0C26F073062543634C3604360CA342C3
:109D6000BFB246F0600603D004F58064A34209D177
:109D70004FF6F3742C4044EA0C0427F4407744EA8D
:109D8000000517439F801E8359631D841A8B22F0A0
:109D900008021204120C42F008021A83F0BD1D687A
:109DA0002B8C23F010031B041B0C2B842B8CAF88F3
:109DB0002E8B23F020031B0444EA0E041B0C26F414
:109DC000E64643EA0413484C3604360CA542BFB2BB
:109DD00046F4C04603D004F58064A5420CD123F0BC
:109DE000800343EA0C1323F040039BB227F440673F
:109DF00043EA001347EA8207AF802E83A9632B84CE
:109E00002B8B23F400631B041B0C43F400632B8394
:109E1000C4E71D682B8C23F480731B041B0C2B845C
:109E20002B8CAF88AE8B23F400731B0444EA0E0422
:109E30001B0C26F0730643EA04232B4C3604360C25
:109E4000A542BFB246F0600603D004F58064A54287
:109E50000CD123F4006343EA0C2323F480639BB208
:109E600027F4405743EA002347EA0217AF80AE8346
:109E7000E9632B84AB8B23F008031B041B0C43F01A
:109E80000803AB838AE71B68188C20F48050000419
:109E9000000C1884188C9E889D8B20F400500004C0
:109EA00044EA0E04000C25F4E64540EA04300E4C6A
:109EB0002D042D0CA342B6B245F4C04503D004F5E1
:109EC0008064A34203D126F4804646EA82169E802F
:109ED0009D83196418849A8B22F400621204120C78
:109EE00042F400629A8359E70000014043685A79BE
:109EF000032A0FD8DFE802F00205080B1868343097
:109F0000704718683830704718683C3070471868D8
:109F1000403070470020704710B543681A68587980
:109F2000084B0344012093F8D840138CA0409BB207
:109F300023EA00031384138CA140194389B21184CE
:109F400010BD00BFB00F0608F0B5EFF31184102369
:109F500083F31288C5684668AA68136823F0010372
:109F6000136032687779104E938936F817609BB288
:109F700023EA060393812A696D681F2A4FF02003A4
:109F800085BF203A93409340EB6098BFAB60E3B24B
:109F900083F31188C3689B6859601A6842F0010214
:109FA0001A6001230374F0BDB00F06080268137D28
:109FB000012B04BF0223137592F82C100CBF4FF431
:109FC00000730023012904BF022182F82C1092F8AB
:109FD000441008BF43F48063012904BF022182F8C2
:109FE000441092F85C1008BF43F4006301290DD1BE
:109FF000022182F85C1043F4805342681268002109
:10A000005162918989B20B43938101E0002BF4D115
:10A010007047034B0348D3F82812FEF759BD00BF21
:10A02000C02900200000014010B5064C0648D4F8B5
:10A030002812FEF74DFDD4F848120448BDE8104040
:10A04000FEF746BDC029002000000140004001404D
:10A0500010B5064C0648D4F82812FEF739FDD4F89E
:10A060004C120448BDE81040FEF732BDC029002064
:10A07000000001400044014010B5064C0648D4F8E9
:10A080002812FEF725FDD4F850120448BDE8104010
:10A09000FEF71EBDC029002000000140004801401D
:10A0A000034B4FF08040D3F82C12FEF711BD00BFD8
:10A0B000C0290020024B0348D3F83012FEF708BD38
:10A0C000C029002000040040024B0348D3F834129A
:10A0D000FEF7FEBCC029002000080040024B0348E8
:10A0E000D3F83812FEF7F4BCC0290020000C004061
:10A0F0000348D0F8703613B100F264601847704717
:10A10000000000200348D0F8903613B100F28460BC
:10A1100018477047000000200348D0F8B03613B14C
:10A1200000F2A46018477047000000200348D0F8F0
:10A13000D03613B100F2C460184770470000002009
:10A140000348D0F8F03613B100F2E46018477047C6
:10A15000000000200348D0F8103713B100F204705B
:10A1600018477047000000200348D0F8303713B17B
:10A1700000F2247018477047000000200348D0F810
:10A18000503713B100F244701847704700000020A8
:10A190000348D0F8703713B100F264701847704765
:10A1A000000000200348D0F8903713B100F284700B
:10A1B00018477047000000200348D0F8B03713B1AB
:10A1C00000F2A47018477047000000200348D0F840
:10A1D000D03713B100F2C470184770470000002058
:10A1E0000348D0F8F03713B100F2E4701847704715
:10A1F000000000200348D0F8103813B100F6040026
:10A2000018477047000000200348D0F8303813B1D9
:10A2100000F6240018477047000000200348D0F8DB
:10A22000503813B100F64400184770470000002072
:10A23000036823F00103036000230360436083602D
:10A24000C3600361212343612A4B984203D13D221D
:10A2500043F8082C7047284B984204D14FF474629D
:10A2600043F8202C7047254B984204D14FF47412C8
:10A2700043F8382C7047224B984204D14FF0746257
:10A2800043F8502C70471F4B984203D11E4A43F8A5
:10A29000642C70471D4B984203D11D4A43F87C2C17
:10A2A00070471C4B984203D11B4A43F8942C7047CB
:10A2B0001A4B984204D14FF03D5243F8AC2C17E0B2
:10A2C000174B9842C3D0174B9842C7D0164B9842B1
:10A2D000CCD0164B9842D1D0154B9842D6D0154BC6
:10A2E0009842DAD0144B9842DED0144B9842E2D018
:10A2F000704700BF1060024028600240406002408A
:10A3000058600240706002403D00002088600240BA
:10A31000400F0020A060024000003D20B8600240D5
:10A3200010640240286402404064024058640240C5
:10A330007064024088640240A0640240B864024035
:10A340002DE9F0416E4D6F4F182303FB005590B07F
:10A35000064695F869084BF09FFF95F868084BF0A2
:10A360009BFFD5F86C884046FFF762FFD5F864483C
:10A370000023CDE90C33CDE90E330493069304F1A9
:10A380004C030293D5F8703801934FF48C73D5F8D1
:10A39000785803FB0673039314236B434FF48062D6
:10A3A00005934FF40063CDE907234FF400514FF4B8
:10A3B0008073CDE909134FF4003301A90B934BF0DF
:10A3C00079FED8F80030504A43F00103C8F8003055
:10A3D00051684E4B0B4043F4403353606368012D8A
:10A3E00023F04073D4BF0022012223F4807343EA98
:10A3F00002236360A268464B134043F00203A3604C
:10A40000E36A013D23F47003EDB243EA055307F517
:10A4100052720127E3623946537D53B392F90D30EE
:10A42000B34226D1137C957D092B3AD9A3F10A00BA
:10A43000D4F80CC000EB40004FF0070E0EFA00FEFF
:10A440002CEA0E0C05FA00F040EA0C00E060062948
:10A4500035D8481E656B00EB80004FF01F0C0CFADE
:10A4600000FC25EA0C0503FA00F028436063013183
:10A47000C9B20137072F02F10C02CDD1A36843F412
:10A480000073A360A36843F48073A360A36843F0E0
:10A490000103A360A36843F08043A36010B0BDE84C
:10A4A000F081206903EB430E4FF0070C0CFA0EFC11
:10A4B00020EA0C0005FA0EF505432561C7E70C29D3
:10A4C0000ED8CD1F206B05EB85054FF01F0C0CFA45
:10A4D00005FC20EA0C0003FA05F505432563C6E7F1
:10A4E000A1F10D00E56A00EB80004FF01F0C0CFAA3
:10A4F00000FC25EA0C0583402B43E362B7E700BF6D
:10A5000000000020202C002000230140E030FCFF50
:10A51000FDF7FFC02DE9F0410022012603250B685D
:10A5200006FA02F737EA030334D10368540005FA48
:10A5300004FE23EA0E0303600B79D0F800806FEA73
:10A540000E0C03FA04FE013B4EEA080E012BC0F884
:10A5500000E014D883680CEA030383604B79D0F8D9
:10A5600008C0A34043EA0C038360436823EA07035F
:10A5700043608B79476893409BB23B434360C36819
:10A5800005FA04F723EA0703C360CB79C768A34041
:10A590003B43C3600132102AC1D1BDE8F081204B9A
:10A5A0009A6802F00C02042A10B534D0082A34D17B
:10A5B00059685A685B684902C3F388134CBF19494C
:10A5C000194902F03F02B1FBF2F25343144A5268B8
:10A5D000C2F3014201325200B3FBF2F3104C0360AC
:10A5E000A168124AC1F30311114491F8DC10CB4069
:10A5F0004360A168C1F38221114491F8DC1023FA71
:10A6000001F18160A168C1F342310A4492F8DC2073
:10A61000D340C36010BD034BE0E7034BDEE700BF50
:10A620000038024040787D010024F400B00F060895
:10A63000F0B5446B8668A38923F400531B041B0CFC
:10A64000A3818579290201F4806C417901F001032D
:10A650008907218A4FEA053289B221F4405102F478
:10A66000005242EA01022282A289C5F3800722F445
:10A67000B0524FEA83034FEA073722F00C0248BF7B
:10A6800043F008034CEA07011204120C0B43134376
:10A69000A381A38A23F440731B041B0C85B0A382FF
:10A6A0006846FFF77CFF204B9C4203D003F5806394
:10A6B0009C4237D1039BA2891921170401FB03F3A4
:10A6C0004FF064014CBF7600B600B3FBF6F3B3FB6A
:10A6D000F1F001FB10330201A08900044BBFDB0045
:10A6E0001B01323332334BBFB3FBF1F3B3FBF1F356
:10A6F00003F0070303F00F0313439BB22381A38AE4
:10A700002A0755BF23F008039BB21B0443F008033C
:10A7100058BF1B0CA382A3899BB243F40053A381AF
:10A7200005B0F0BD029BC6E7001001402DE9F843DB
:10A730001E46204B9DF820509DF824709842894673
:10A7400090462CD13B462A4631460020FEF72CF994
:10A7500004460020C4E90700C4E90900C4E90B98D5
:10A760006571A660A7712046FFF762FFEA0707D56B
:10A77000636B4FF6DF721A80DA6842F02002DA600B
:10A78000626BAB0742BFD36843F08003D360938909
:10A790009BB243F4005393812046BDE8F883064BF7
:10A7A000984204D13B462A4631460120CEE7002498
:10A7B000F2E700BF0010014000440040816037E72D
:10A7C000417135E72DE9F043654F07EBC00985B0CE
:10A7D00005464FEAC00899F8B00805F06BFB06463D
:10A7E00099F8B10805F066FB044699F8B2084BF0F9
:10A7F00053FD6B1CDBB21EB140F60C12F2803372BB
:10A800001CB140F60C22E280237204223A21304629
:10A8100005F010FB204604223A2105F00BFB07EB64
:10A820000803D3F8AC484F4B9C4263D103F5F23395
:10A830001A6A42F400121A621A6A22F400121A62A8
:10A84000474497F8B338022B6ED0032B6ED0464E98
:10A85000464A012B18BF1646A78827F03F076846CF
:10A860003F04FFF79CFE3F0C029A414BB2FBF3F30F
:10A8700098B20743A780218821F001010904090C3F
:10A8800021803C498E4253D13B4BB2FBF3F2013065
:10A8900091B2042980B238BF04212084A183238887
:10A8A0009BB243F001032380238823F4816323F0C8
:10A8B00002031B041B0C43F4806323804FF480438A
:10A8C0002381238823F080031B041B0C238023880F
:10A8D0009BB243F001032380284B03EB4513012275
:10A8E00083F80126002283F8005683F8022605B07B
:10A8F000BDE8F083224B9C4209D103F5F0331A6A7C
:10A9000042F480021A621A6A22F4800297E71D4B11
:10A910009C4295D103F5EE331A6A42F400021A62A2
:10A920001A6A22F400028AE7124E95E7124E93E764
:10A9300006EB4606B2FBF6F291B2C2F30B020AB97D
:10A9400041F001014FF4967253434FF47A72B3FB16
:10A95000F2F301339BB241F4004123849EE700BF30
:10A96000000000200054004000350C00801A060052
:10A9700040420F00A0860100400D0300C0290020C6
:10A9800000580040005C00402DE9F047B94E4401FA
:10A9900006EB401908F080F999F90026B64B884675
:10A9A000D10003EBC2020746D2F8AC5899F8022650
:10A9B000013A142A00F28380DFE812F0790089005E
:10A9C000A100BA00C700D100DC00F40001010A01B7
:10A9D00017016A018801BA011102240236024102FC
:10A9E0006102840215005F184FF0090A97F8B00859
:10A9F00005F060FA054697F8B10805F05BFAB6F87D
:10AA0000603601339BB207462846A6F8603605F04B
:10AA1000DDF9384605F0DAF91121284605F0E0F9AC
:10AA20001121384605F0DCF94FF0650803E00520F8
:10AA3000002108F06FF9284605F0B7F910B9B8F110
:10AA40000108F4D1284605F0C6F90021052008F0D8
:10AA500061F9284605F0BAF90520002108F05AF9F5
:10AA6000BAF1010AE0D1284605F0B5F90021052028
:10AA700008F050F9384605F0AEF90021052008F03D
:10AA800049F9284605F0A2F90520002108F042F90D
:10AA9000384605F09BF9331993F90006431C01D0A1
:10AAA000FFF790FE3319002283F8022607E02B8877
:10AAB00013F4007340F0D281321982F80236331950
:10AAC00093F80236002B7FF465AFBDE8F0872B8842
:10AAD00023F400631B041B0C2B802B889BB243F4D4
:10AAE00080632B802B889BB243F480732B803319B7
:10AAF000032283F80226614B2344C3E902786049AC
:10AB00002846FDF760FB002800F0A881331993F870
:10AB100012265AB993F81326FF2A04D193F8102667
:10AB20000AB10A22C0E733190422BDE70F22BBE7AE
:10AB3000321992F8113603F0FE032B82052382F8B6
:10AB400002364E4B2344C3E902784E492846FDF7AE
:10AB50003AFB002800F07A8133190622A4E7331962
:10AB600093F813262A82072283F80226434B2344B4
:10AB7000C3E9027844492846FDF725FB002800F088
:10AB800065813219D2F8143653B92B889BB243F43D
:10AB900000732B80394B2344C3E9027801238CE7EF
:10ABA00008238AE72B889BB243F480732B803319E8
:10ABB000092283F80226314B2344C3E90278304945
:10ABC0002846FDF700FB002800F048813319A8E76C
:10ABD000321992F8113643F001032B820B2382F8CD
:10ABE0000236264B2344C3E9027828492846FDF75C
:10ABF000EAFA002800F02A813319D3F81436012B21
:10AC00001CD12B8823F480631B041B0C2B80EFF3D7
:10AC10001182102383F312882B8B2B889BB243F471
:10AC200000732B80D3B283F311880C23321982F87E
:10AC30000236124B2344C3E9027840E7022B15D1B8
:10AC40002B889BB243F400632B80EFF31182102317
:10AC500083F312882B8B2B8823F480631B041B0C3B
:10AC60002B80D3B283F311880D23DFE72B8B0E23C8
:10AC7000DCE700BFC029002000000020C02F00201A
:10AC800001000300820007008400070002000300A7
:10AC900094492846FDF7A1FA934B002800F0DF8085
:10ACA00031192344D1F81826501CC1F81806288AF7
:10ACB0001070D1F81426013AC1F814260122C3E914
:10ACC000027881F81C2681F80226F8E68749284692
:10ACD000FDF783FA844B002800F0C180EFF3118C5C
:10ACE000102282F312882A88301992B2D0F81816EE
:10ACF00042F400722A804A1CC0F818262A8A0A7078
:10AD00005FFA8CF282F31188D0F81826511CC0F833
:10AD10001816298A11706FF00102C0F81426234416
:10AD20000122C3E9027880F81C2680F80226C6E6D4
:10AD30006E492846FDF751FA6B4B002800F08F80D2
:10AD40003219D2F8141603292AD1298821F48061F6
:10AD50000904090C2980EFF3118C102181F312886A
:10AD6000D2F81806411CC2F81816298A01702988E1
:10AD700089B241F4007129805FFA8CF181F3118866
:10AD8000D2F81816481CC2F81806288A0870D2F89B
:10AD900014160239C2F814160C2182F8021649E77B
:10ADA00002290FD8298821F480610904090C29801F
:10ADB000298889B241F400712980298A002182F80A
:10ADC0001C16E8E6D2F81816481CC2F81806288A9D
:10ADD0000870D2F814160139C2F814162AE72B8825
:10ADE00023F4806332191B041B0C2B8092F811365C
:10ADF00003F0FE032B82102382F802363A4B2344E1
:10AE0000C3E902783A492846FDF7DDF9F0B1331974
:10AE100093F81326FF2A04D193F810260AB11322BF
:10AE200042E6331911223FE6331993F813262A829A
:10AE3000122283F802262C4B2344C3E902782D49C1
:10AE40002846FDF7C0F908B13319E8E72A49284632
:10AE5000FDF7C3F910B13319142225E6224B234420
:10AE6000D3E9022342F21071BA1A68EB03038A4253
:10AE700073F10003FFF423AE3319152214E63119E0
:10AE8000194BD1F814268AB1D1F81806234410F8CA
:10AE900001CBA5F810C0013AC3E90278C1F8180641
:10AEA000C1F81426122381F8023608E62A8892B2E5
:10AEB000234442F400722A80C3E90278012381F816
:10AEC0001C36F0E72B889BB243F400732B804FF6BF
:10AED000FF33AB82044B2344C3E9027801223319C8
:10AEE000E2E500BF40000010C02F00200400001069
:10AEF00082000700840007000004001038B5114CE0
:10AF000004EB401494F80156D5B1C4F81436049BF0
:10AF1000C4F81836002384F81C360223490084F84C
:10AF2000132684F8023601229DF8143084F8111695
:10AF300084F8122684F81036FFF726FD94F81C5684
:10AF4000284638BDC029002038B5114C04EB401408
:10AF500094F80156CDB1C4F81436049BC4F81836E1
:10AF60000223490084F8132684F8023600229DF853
:10AF7000143084F8111684F8122684F81C2684F8FC
:10AF80001036FFF701FD94F81C56284638BD00BF67
:10AF9000C029002082B000230193054B0193019B3F
:10AFA00003EB80030193019B196002B0704700BF5F
:10AFB0005028004082B000230193054B0193019B70
:10AFC00003EB80030193019B186802B0704700BF38
:10AFD0005028004010B51C2004F06CFF11210446DD
:10AFE00004F0FEFE204604F0F6FEC82007F032FF13
:10AFF0002046BDE8104004F0E9BE436D064A1A61E0
:10B00000C278012A06D100F2CC5058611A684FF07C
:10B0100080221A60704700BF1800086038B50446E7
:10B0200000296DD190F81131022B28D1D0F83821A8
:10B03000D0F824118A4230D9C378012B02BFD0F84E
:10B0400028315B18C0F82831521AD0F82831C0F8DE
:10B0500038214FF48071002592B2A0F81C11C0E98C
:10B060004A33C0F83451C0F8302100F58E714EF0EB
:10B070005BF82B462A46294620464EF06DF994F897
:10B080001631012B07D1244A2369D2F8A4215A6032
:10B09000002384F81631002038BDD0F83C31B3FBD2
:10B0A000F1F501FB1535A5B9994212D8D0F8402128
:10B0B00093420ED24FF48073C0E94A55C0E94C5513
:10B0C000A0F81C3100F58E714EF02EF8C4F84051F6
:10B0D000CFE7D4F8E435DB682BB194F81221032ACA
:10B0E00001D120469847052384F8113100232046DA
:10B0F0001A4619464EF030F92046FFF77EFFBEE7AC
:10B10000D0F8E4355B69002BC5D090F81221032AF2
:10B11000C1D19847BFE700BFC029002070477047E2
:10B12000704710B50F4C94F86E36B3B14FF0E02273
:10B13000D2F8103D23F00603C2F8103DFEF755FC8F
:10B14000D4F874369B68DB0707D5D4F870271368EA
:10B1500023F0030161F307031360034B4FF48022D4
:10B160005A6110BDC0290020003C01402DE9F04F7C
:10B17000B14CD4F870365A69D0078BB000F1968183
:10B180005A699B6912EA030A00F09081CAF30743E7
:10B190001AF4002F01930FD0D4F87436DFF8A08290
:10B1A0009E69DB691E40360C04F5D76B04F26469B6
:10B1B0000027002E40F07D81019B59070DD5D4F862
:10B1C00074369E4D9F69DB691F40BFB205F11806BA
:10B1D0004FF00008002F40F0AD811AF0020F1FBFA2
:10B1E000954BD3F8703602225A61BAF1000F5FFA1C
:10B1F0008AF51BDA904B93F86E263AB1D3F8702794
:10B20000136823F0030161F307031360D4F8742675
:10B210008A48536823F001035360894BD3F8DC3824
:10B220009847D4F870364FF000425A611AF4006F14
:10B23000CAF307262FD000238DF8173094F87637FD
:10B240008DF817307E4B7D48D3F8D8389847D4F81E
:10B250007026D4F874364FF400619B68516194F8FD
:10B260006E26C2B1DB0716D594F87937012B12D1BF
:10B270009DF81730032B0ED1D4F870371A6842F0BE
:10B2800001021A601A6842F003021A606D4A1369DB
:10B2900043F0060313612F0708D5694B6748D3F8BD
:10B2A000D0389847D4F8703608225A61ED0614D584
:10B2B000D4F87006836923F010038361036AC3F333
:10B2C0004341022903F00F0200F0E981062900F052
:10B2D0000D82836943F010038361F00633D5D4F8FF
:10B2E0007456D4F870866B68002723F001036B60F6
:10B2F000394640464EF064F894F865C65249B9465E
:10B300003B46FF206345C0F0FF814FF0FF33AB6148
:10B310004FF00113EB610B2363F3070763F3070996
:10B320006F61C5F810902B68444823F4FE632B60CE
:10B33000FFF763FE4FF48053C8F81430404B3F488A
:10B34000D3F8D4389847B1066DD5D4F87466D4F8DC
:10B350007C26B3681168C3F34103022B14BF00239A
:10B36000032363F30A011160736843F4807373600D
:10B3700006A8FFF714F9D4F870560799E86820F486
:10B380007050E860B36813F0060FC3F3410200F099
:10B39000C2812E4B2E4A0B44934240F2C0812D4A6B
:10B3A000A1F57403A3F51053934240F2BC812A4BDC
:10B3B0002A4A0B449342C0F0BA81294AA1F18C7306
:10B3C000A3F54343934240F2B681264B264A0B44F1
:10B3D0009342C0F0B481254B254A0B449342C0F000
:10B3E000B281244AA1F1B773A3F558539342C0F038
:10B3F000AD81214B214A0B449342C0F0AB81204BDD
:10B40000204E0B4401224021B34234BF06230523C2
:10B41000094E63F38D204FF40053E86086F86626EA
:10B42000A6F868166B61019BDA0632D5044B034817
:10B43000D3F8E038984727E0C029002024300020C6
:10B440000000002000ED00E038300020401E1BFF0F
:10B450003F420F00DFC810002013FBFE20D6130070
:10B46000FF69180000D3CEFE40771B00C05BB3FE1F
:10B47000C091210040AC2700C01D6AFE40E13300AE
:10B48000803C36FEE09C4100D4F870364FF48012C8
:10B490005A61019B9B0609D5B04BB148D3F8E438FB
:10B4A0009847D4F870364FF400125A610BB0BDE8DB
:10B4B000F08FF10737D5DBF80010D4F874368D68BB
:10B4C0005B691D40EA071ED594F867360125AB423B
:10B4D0008D6007D10969D9F87C33C1F312015B1A79
:10B4E000C9F88C33D8F8C4389D48F9B2984794F815
:10B4F0006736012B07D137B994F87537052B02D180
:10B500009748FFF77AFDAB0742BFDBF80030022512
:10B510009D60280707D5D8F8CC3891489847DBF8C4
:10B52000003008229A60013776080BF1040B09F10C
:10B5300028093EE6FA0772D5D4F8743632681869DD
:10B54000D3F83490916829FA08F94FEAC9195FFADB
:10B5500089F949EA000909EA010919F0010F1FD028
:10B56000596B012000FA08F021EA000159637B4B76
:10B570007B48D3F8C8384FF00109C2F808905FFA49
:10B5800088F1984794F867364B4509D1B8F1000F18
:10B5900006D194F87537042B02D17148FFF72DFDC1
:10B5A00019F0080F1EBF33684FF00809C3F8089060
:10B5B00019F0100F1EBF33684FF01009C3F8089040
:10B5C00019F0400F1EBF33684FF04009C3F80890D0
:10B5D00019F0020F1EBF33684FF00209C3F808903C
:10B5E00019F0800F1BD0D5E94C329B1AD5F82421D5
:10B5F000D6F800B0934228BF13465A4ADBF8180029
:10B6000092F867C6D2F8749603339B080293029BA4
:10B6100080B2984203D9D5E94C03984205D808F185
:10B6200001087F0828350436D4E5C01AD5F824313E
:10B63000984228BF1846C31C9B080293BCF1000F18
:10B640001BD0D5F82811D5F834210144C5F82811AC
:10B65000D5F8301102448A42DBF81800C5F83421CD
:10B66000D5D195F81C11D9F83420012303FA01F142
:10B6700022EA0102C9F83420C9E782B2D6F8B8102C
:10B68000D5F828E10332931003930A466146039BE1
:10B690008B42D6D05EF8213013600131F7E747F6D0
:10B6A000F07119423FF415AE282101FB0241C3F3AA
:10B6B0000A13DD1CD4F834C7D1F8E479AD100021A9
:10B6C0008D420DD1282101FB0242D2F8E419194420
:10B6D000C2F8E419D2F8F0191944C2F8F019F8E5E3
:10B6E000DCF800E047F821E00131E9E7D4F834174D
:10B6F0000D68C4F8305C0968C4F8341C282101FBCB
:10B700000242C3F30A13E5E751F8042F9060CA6BB5
:10B7100001339060F6E54FF40071092378E60122C9
:10B7200040210E2374E6012240210D2370E6012200
:10B7300040210C236CE6012240210B2368E6012204
:10B7400040210A2364E601224021E6E7012240214C
:10B7500008235DE601224021072359E6000000206E
:10B7600024300020C0290020034BD3F87C0908B105
:10B7700004F01BBB01207047C818002008B5FFF774
:10B78000F3FF0A4A18B9002382F8503908BD92F82D
:10B7900044390133DBB2072B82F84439F3D8044B28
:10B7A000D3F89431C2F840390123EDE7C8180020DE
:10B7B000C0290020F0B5C54CD4F8800985B0002818
:10B7C00061D094F85039013B082B44D8DFE813F0DE
:10B7D00009005D00DF004300AA013001860143003B
:10B7E000E601FDF7C1FD00210846FDF749FE0546CB
:10B7F000FDF7CAFD012D29D1002684F84569FDF722
:10B80000B3FD40F2AB110820FDF73AFE05280AD13E
:10B8100084F84559FDF7B8FD94F84539A3B10223E2
:10B8200084F85039CDE70128F4D10423D4F88009F5
:10B83000324669464DF02EFE9DF80330AB2B04BF17
:10B84000022384F84539E5E784F85039D4F88009B3
:10B85000022104F001F894F85039013B022B09D879
:10B860009B4BD4F84029D3F894319B1AC82B01D9AB
:10B87000FFF784FF94F85009042800F0A081A0F19C
:10B8800008035842584105B0F0BDFDF76DFD94F82E
:10B890004559AA1E55425541AD0700213720FDF7F5
:10B8A000EFFD29462920FDF7EBFD0546FDF76CFD70
:10B8B000002DCBD194F84539022B17D1FDF754FD5B
:10B8C00029463A20FDF7DCFD042306462A46D4F833
:10B8D000800969464DF0DEFDFDF756FD16B1FFF714
:10B8E0004DFF6EE7009D2DBAC5F3807584F846596B
:10B8F000FDF73AFD00210920FDF7C2FD10B1FDF76B
:10B9000043FDA3E773481021FDF76EFD06460028AE
:10B91000F5D101217F204AF085F901280546EED1B5
:10B92000022130464AF07EF950B10128E7D11621B4
:10B930003A204AF077F901308002C4F8540918E03F
:10B9400004212C204AF06EF9032107464E204AF0CC
:10B9500069F90C21064636204AF064F90236431C88
:10B96000B340BD40A3FB05355B0A43EAC553C4F8A9
:10B970005439FDF709FDFDF7F7FC00210A20FDF71A
:10B980007FFD08B903234BE7FDF7FEFCA7E7102175
:10B990006846FDF729FD00287FF458AF9DF8003078
:10B9A00084F85A39BDF801305BBAA4F858399DF8CB
:10B9B000033084F85B39019BC4F85C399DF808308A
:10B9C0001A0903F00F0384F86539DDF8093084F8AB
:10B9D00064291BBAC4F860399DF80D309DF80E201B
:10B9E0001B01DBB243EA121303F5FA6302F00F0204
:10B9F000A4F8663984F86829FDF7C6FC94F846393E
:10BA00004BB1D4F88009022103F026FF0023C4F8CB
:10BA10004C39042304E7FDF7A7FC4FF40071102014
:10BA2000FDF72EFD0546FDF7AFFC002DE9D056E7EA
:10BA300094F83419D4F82C29D4F88009802302EB27
:10BA4000C11200214DF026FD94F834390133DBB2E8
:10BA5000042B84F834397FF4FEAE1F4AD4F88009F1
:10BA6000022300214DF016FD0123D4F880090022A5
:10BA700069464DF00FFD9DF8003003F01F03052BC4
:10BA800015D1072384F85039114BD4F83859D3F81D
:10BA90009431C4F84039002D3FF4DDAED4F83C3980
:10BAA000D4F82C29D4F830190120A847D3E6FFF7A1
:10BAB00065FED4F83859002D3FF483AED4F83C39F4
:10BAC000D4F8301900220120A8477AE6C8180020CF
:10BAD000C0290020342200209C1006084AF0C2F839
:10BAE000002862D0002384F84439D4F84C39012B63
:10BAF0000BD9013BC4F84C39D4F848390133C4F8A8
:10BB00004839082384F85039A5E607D1FDF78EFCA3
:10BB100002287FF4A0AEFDF737FC9CE6042384F8EE
:10BB20005039F8E7D4F82C094FF40071FDF75CFCAC
:10BB30000128054619D0022820D000287FF48BAEBA
:10BB4000FDF722FCD4F8386984F84459042384F8BA
:10BB50005039002E3FF47FAED4F83C39D4F82C296C
:10BB6000D4F830192846B04775E6164BD3F894211F
:10BB7000D4F8403964339342BFF46DAEFDF704FC52
:10BB8000FFF7FCFDD4F83859002D3FF41AAE00221F
:10BB9000D4F83C39D4F83019104695E74AF062F8E9
:10BBA00018B1FDF7F1FB0423ACE7064BD3F8942161
:10BBB000D4F84039FA339342FFF491AE4BE60120BA
:10BBC00061E600BFC02900202DE9F341284C05465D
:10BBD0000E4690461F4694F85039042B0DD0082B82
:10BBE00007D1D4F84839AB4219D0FDF71FFC022821
:10BBF000F1D0012002B0BDE8F081FDF7B5FB94F86B
:10BC0000463953B969021820FDF73AFC38B1FDF7FF
:10BC1000BBFBFFF7B3FD0320ECE72946F3E794F8FD
:10BC20005039D4F88009082B14BFFE23FC23FF22CF
:10BC30008DF804208DF8053001AA022300214DF073
:10BC400029FCD4F880098023324600214DF022FCE3
:10BC5000012384F834390623C4F82C69C4F8305918
:10BC6000C4F83889C4F83C7984F850390020C1E719
:10BC7000C818002070B51C4C94F85039042B0546A8
:10BC80000E4610D1FDF770FB00213720FDF7F8FBC1
:10BC900031461720FDF7F4FB90B1FDF775FBFFF778
:10BCA0006DFD032002E0082B01D0012070BDD4F807
:10BCB0004839834214D0FDF7B9FB0228F5D1E1E7FA
:10BCC00094F8463973B969021920FDF7D9FB0028A9
:10BCD000E3D1082384F85039C4F84C69C4F84859B2
:10BCE0000220E3E72946EFE7C8180020044B054A85
:10BCF00003F50F61D3F8F038C2F82819184700BFD0
:10BD000000000020C8180020002108B5084604F0F3
:10BD100089FAFFF7EBFFFCF7E3FB0028FBD00121DA
:10BD2000002004F07FFA002008BD034BD3F8280957
:10BD300008B1436918477047C8180020034BD3F86F
:10BD4000280908B183691847704700BFC818002048
:10BD5000034BD3F8280908B1C3691847704700BFDF
:10BD6000C818002038B50D461446FFF7F1FF0368E8
:10BD70002B604FF400732360002038BD034B1B7809
:10BD8000032B14BF4FF48070802070479C5000201C
:10BD900008B50B4A68B1816811B10723937008BDDB
:10BDA000FFF7ECFFC2E90311C2E90100117504239A
:10BDB000F4E702F58051012381F8B4315370EEE7C6
:10BDC0009C50002010B502784368022A0B4A06D125
:10BDD000D2E9802102EB410202EB532010BD016940
:10BDE000D2F81802D2F8104218400239D2F80C32B8
:10BDF000400A04FB01001844F0E700BF9C600020EB
:10BE0000064B1B78022B0BBF030AC0F3D413C0B23E
:10BE100000F07F000B601060704700BF9C50002056
:10BE200090F91A305A1C0AD003F58172124B03EBB9
:10BE30000213DA7922F00102DA71FF23837690F996
:10BE40001B104B1C16D00C4A01F5817102EB01133B
:10BE500002EB0112DB79D179C3F34503012B86BFD5
:10BE600003F1FF3303F03F03002363F34601FF2395
:10BE7000D171C376704700BF9C50002008B5FFF712
:10BE80007DFF034BD3F810325843400208BD00BF7A
:10BE90009C6000200378022B09D10E4BD3F820229E
:10BEA0004368B3EB422F2CBF01200020704700698C
:10BEB00070B1094B1B78032B0EBF084B80B24FF6B5
:10BEC000F773984294BF0020012000F001007047F2
:10BED0000120FAE79C6000209C500020F7FFFF0F34
:10BEE0004368F7B5C3F308020A44B2F5007F04467D
:10BEF0000D4604D22B446360012003B0F0BDFFF770
:10BF00008FFF0378022B01D16368F3E7154BD3F859
:10BF10001022B5EB422F4FEA422706DCD3F8183245
:10BF200046681E407342AB4201DD0020E5E7AB19D5
:10BF3000BB4210D30169007E01AA4DF017F8012819
:10BF4000F3D123696361019B236163683B449B1BBD
:10BF5000EF1B6360BD192046FFF79CFF0028CBD183
:10BF6000D2E700BF9C60002070B504460E4615461F
:10BF7000FFF7B6FF20B10DB12046A847012070BDE4
:10BF800094F82800022320B9C4E90B5684F828301D
:10BF9000F5E71846F3E738B5174D05F58054014627
:10BFA00094F8E00130BB49B191F828302BB9442214
:10BFB00004F5DC7052F0ACFD012038BD44220F487E
:10BFC00053F0C8FE4FF6FF73A4F8D231032384F870
:10BFD000D0312B780948022B18BF032384F8B831DD
:10BFE000D4F81C32C4F8DC31102384F8D1314AF083
:10BFF00085F9E1E70020E0E79C5000205462002032
:10C00000044A92F8B411012309B982F8B431024A02
:10C01000537070479C6000209C5000202DE9F74F22
:10C0200012F002098A461546019304D018B9FFF7A9
:10C03000E7FF02200CE0684AD2F808625EB1D2E95C
:10C04000831404FB0611884205D3FFF7D9FF0020B3
:10C0500003B0BDE8F08F4FF0FF31604EDFF880B1E4
:10C060008C468E46884600243368B77B984221D19F
:10C07000002F46D0D2F89810594E0131C2F89810CE
:10C0800004F581721201B1502146554C01F58176BB
:10C0900004EB06129279042AC9D801A757F822F0B6
:10C0A00037C100088DC100084FC000088DC10008CD
:10C0B000A1C100080FB3012F10D104F581770BEB5C
:10C0C0000717FF79FB0709D417F07E0F06D1FF0988
:10C0D00015D1B76847453CBFA446B8460134082C83
:10C0E00006F11006C0D100290CDABEF1000F20DAEB
:10C0F000BCF1000FABDB614604E02146EEE7A6464B
:10C10000ECE72146364E41F2180406EB0117385190
:10C11000D2F898400134C2F8984041F21C02BC5059
:10C1200001F58172170106EB0212F45100245460EC
:10C13000ABE77146E6E715F0010213D0294BD3F8BF
:10C140002839002B83D0284F5D68284A002307EB4D
:10C150004121A84700283FF47AAF04EB06140223DC
:10C16000A37174E704EB0610019B90F807C0EF1071
:10C1700067F3C71C032B80F807C02BD94FF6FF725B
:10C18000934228BF134604EB06129380B9F1000FC7
:10C1900006D004EB011000F580501830FCF7C2F90E
:10C1A0006A0741BF04EB0612D37943F00103D37150
:10C1B000EB0608D504EB0614E379C3F3450201321C
:10C1C00062F34603E371084B03EB4123CAF80030E6
:10C1D00001203DE71346D6E79C600020B4600020B4
:10C1E0009C500020C8180020B4500020F195000891
:10C1F0007FB50F4D01AA0C4602A9FFF701FE05F518
:10C200008053029ED3F800020322002303A9304486
:10C21000FFF704FF012808D12978039B019A02291E
:10C220000CBF23F8124043F8224004B070BD00BF99
:10C230009C5000202DE9F04FD1F8009085B01646B3
:10C24000074601AA48460D4602A9FFF7D9FD374A1D
:10C250000299D2F8003201EB0308019B013B9C19C3
:10C26000FFF78CFDA4EB09040444A2F5805AB4FB4B
:10C27000F0F408EB04092B68B342A9EB080103D3DF
:10C28000012005B0BDE8F08FDDF804B00BEB06042B
:10C29000E41AFFF773FD844228BF0446BBF1000F88
:10C2A0001AD1A0428CBF0B220A220B46404603A99A
:10C2B000FFF7B4FE0128E4D19AF800102B68039A26
:10C2C000022903F1010358460CD0A0420CD242F8D7
:10C2D000203001300133F8E70B22E6E722F8103076
:10C2E00001300133A042F9D32B68A3EB0B032344A5
:10C2F000012F2B6014D1B34212D102290BBF04F1DC
:10C30000004404F1804304F1FF3403F1FF330BBF19
:10C310004FF6FF734FF0FF3122F8143042F823102C
:10C32000002308F101080193A5E700BF9C600020ED
:10C330002DE9F04F85B00546FFF720FD0C46174666
:10C34000814601AA206802A9FFF75AFD6B1E012B46
:10C3500066D9019B4BB94E46DFF8C880012D8CBFD2
:10C3600000250125A8F5805A1BE0FFF749FE0220B1
:10C370002BE0D8F87831C3B1D8F89411914214D198
:10C38000D8F81022013B500203EB4223B3FBF0F339
:10C390000B44B3FBF6F206FB12320AB133449B1A8C
:10C3A00023602268BA42E4D32BE0DDF808B0D8F865
:10C3B00000020023092203A95844FFF72FFE012899
:10C3C00006D00228D3D00028EBD105B0BDE8F08F0D
:10C3D0009AF80010019A022907D00329C7D1039BBC
:10C3E00053F8223023F0704302E0039B33F81230FD
:10C3F000D4F800C0B3FA83F35B09AB4204D16745BC
:10C40000E3D827600320E0E732440CEB06039145B4
:10C410002360E0D80BF10103029300230193C0E7EE
:10C42000012699E79C60002037B50446C0690D4697
:10C4300010B9012003B030BD0023032201A9FFF78A
:10C44000EDFD0128F6D1B4F92030002B17DB019A5D
:10C45000012D4FEA431102EB431316D0022D12D0E7
:10C46000E268DA612278032A04D100221A775A7727
:10C470009A77DA77626A5A83110C9982D9E7FFF7C3
:10C48000BFFD0220D6E7E5205054A268E9E738B5A1
:10C49000044694F83430052B2FD8DFE803F0072743
:10C4A000353C444D022084F83400F2E7294DD5F89C
:10C4B000082204F1300102320120FFF739FF012880
:10C4C00005D00238C0B2012817D80520EBE7D5F80F
:10C4D0001012E268236BC5F8143202EB4122E260CD
:10C4E000E26A2361002ADED16362DCE7206B4FF051
:10C4F000FF31FFF77DFE012801D0002038BDE36A3F
:10C50000002BCFD10320CEE7D4E90B01FFF770FE5B
:10C510000128F7D0F1E700212046FFF785FF012829
:10C52000EBD10420BFE794F82830082B04BF002388
:10C5300084F828300120E1E794F82830082B04BF64
:10C54000002384F82830034B012283F8B521022010
:10C55000D4E700BF9C6000202DE9F341044694F825
:10C560003830032B0ED8DFE803F00611767F032066
:10C5700084F83800F3E72046FFF789FF0128F7D059
:10C580000228F4D0002002B0BDE8F081237865686D
:10C59000DFF8E480022B1CBF374BD3F8183220465B
:10C5A00018BF1D40FFF70EFCC5F34F252D1A064698
:10C5B000ADB20023022201A93046FFF72FFDAF19CB
:10C5C0000128BFB2DFD101984FF40072002153F06F
:10C5D000C1FBE3692BB363681BBB019B4FF02032A7
:10C5E0002E211970C3F80120C3F80520A3F80920F3
:10C5F000606A58834FEA104C102083F8201083F8AB
:10C600002110D872C3F82220C3F8262083F82A20EC
:10C61000E26BA3F814C022FA00F199865A8783F8D6
:10C620002B00D8F810124B1E9F4208D24FF4007115
:10C630002046FFF755FC4CF0B9FB0136B9E7C1EBDA
:10C64000C151490201F500712046FFF749FC4CF049
:10C65000ADFB02208CE7002384F82830236C0BB15B
:10C660002046984701208EE7236C002084F828009C
:10C6700003B19847022086E79C60002010B504466D
:10C6800094F83830032B53D8DFE803F00631434DDC
:10C69000022384F83830F3E72649D1F89421226147
:10C6A000FFF7ECFBE3680344E360FFF767FB10442C
:10C6B000C1F89401FFF7E2FBD1F878311B1AC1F8F9
:10C6C0007831FFF7DBFBD1F87C311B1AC1F87C31E4
:10C6D0002263FFF753FBE36A1044606313B962629D
:10C6E0000123D6E7FFF74AFB121A2263F8E7124844
:10C6F0000021FFF799FE0128CAD0431EDBB2012BAF
:10C7000006D894F82830062B04BF002384F828307C
:10C7100010BD626B04F130010120FFF78BFD012891
:10C72000EBD10323B5E700212046FFF77DFEE4E7C8
:10C730000220E2E79C6000200C6200202DE9F74314
:10C7400006460C464FF6F77596F83C30042B73D826
:10C75000DFE803F0290736416300032086F83C0038
:10C76000F2E73A4FDFF8EC8007F580593B78306B01
:10C77000032B4FD140454BD801A949F02FFA01288E
:10C7800057D1306B0021FFF733FD012851D1019BB8
:10C790003363D9F81422013B934294BFC9F8143291
:10C7A000C9F81422E2E7610001F0FE013046FFF70C
:10C7B0003BFE01280CD1736B002B18BF0220CDE784
:10C7C000726B06F130010020FFF734FD0128C4D060
:10C7D00002282ED131E01E48F26AD0F89431C0F818
:10C7E00094219B1AD0F810225343D0F8782102EB01
:10C7F0004322C0F87821D0F87C2102EB4322C0F814
:10C800007C21002100F5B870FFF70EFE0128DFD172
:10C810000420A3E783B2AB42ADE796F82830042B9F
:10C8200004BF002386F82830B36B0BB1304698471D
:10C83000012003B0BDE8F083022096F82830042BD5
:10C8400004BF002386F82830F3E700BF9C50002087
:10C850009C600020F7FFFF0F70B50378027E023B5B
:10C86000012B04461CD8237E990622D42046FFF7CC
:10C87000D7FA237E1A070AD51E4D95F89801C31FD3
:10C88000584258414CF092FA002385F89831002321
:10C89000237084F82830E36A53B1BDE8704018472C
:10C8A00012F0060FDFD00121FFF7BEFD0128DAD01C
:10C8B00070BDE2691049002318010858824211D165
:10C8C0000E4903F5817201EB0213DB79C3F34503D3
:10C8D000012B0BD8002301EB0212D17963F346013F
:10C8E000D171C3E70133082BE6D1BFE7013B03F069
:10C8F0003F03F0E79C600020B46000209C500020C3
:10C9000010B580B1027872B190F828206AB9D0E9E8
:10C91000012494422CBF84608260032280F8282086
:10C92000C162FFF799FF012010BD0020FCE7B1F9BB
:10C9300004300F2B2DE9F34104460D4616460BD16A
:10C940004FF40071FFF7CCFA18B9002002B0BDE82F
:10C95000F0814FF6FF73AB802046FFF733FA94F96E
:10C960001B20531C074624D0244B41F2180103EB33
:10C97000021041588F4212D1183303EB4223019326
:10C98000019A72B1AB8801331BB202EB4312AB8048
:10C9900020463260FFF716FA28600120D6E7FFF73D
:10C9A0002FFB2046FFF776FA0028CED00023336015
:10C9B000F3E72046FFF76EFA80460028F1D1381ED3
:10C9C00018BF01204CF0F2F94346112201A9384664
:10C9D000FFF724FB0128E4D1094A019B9B1A48BFB9
:10C9E00003F2FF13B3F5805F4FEA632203D3FFF72F
:10C9F00007FB4FF0FF32E276C2E700BF9C500020F9
:10CA0000B45000202DE9F0414FF0FF31304A314C55
:10CA10000D460023107804280ED103F5817004EB35
:10CA20000010C079C60707D4681C52F80A0C01D060
:10CA3000884201D201461D460133082B02F1100243
:10CA4000E8D1002D41DB234CDFF8988005F5817794
:10CA500004EB07132E01998841B1D8F828392BB17E
:10CA6000A01941F218029B688058984741F21803B8
:10CA70002644F058D8F828396BB1174ED3F80C80FB
:10CA8000164A002306EB4521C04720B1022810D0EA
:10CA90000020BDE8F081124BD3F89C2004EB071472
:10CAA000013AC3F89C200322A271012283F8A0203E
:10CAB000EEE706F6E87604EB0714D6F89C30013B67
:10CAC000C6F89C300123A371E2E70120E1E700BF33
:10CAD000C26000209C500020B450002049960008FD
:10CAE0009C600020C818002070B5124D124BC5F88C
:10CAF000583C40F20112002385F81432A0F844217A
:10CB0000C0F85C3105F658420D23C0E954220446B2
:10CB100085F8641CC0F8583100F5A2714CF083FB15
:10CB200005F5FA7220461F23BDE8704001214CF044
:10CB300013BC00BFC02900205553425370B50B7879
:10CB400013F06002044638D0202A1ED14A78FE2A0B
:10CB500005D0FF2A1DD04CF065FA022016E04A8865
:10CB6000AAB9CE88012E12D11A0610D5314DD5F8AA
:10CB700020329B699847C0B285F8680C38B13246BC
:10CB800005F6684120464CF023FB002070BD20468E
:10CB9000E1E74A88002AFAD1C9880029F7D11B06A3
:10CBA000F5D4244A82F81412012182F8F0111F23CF
:10CBB00002F5FA724CF0D0FBE7E74B780A2B24D051
:10CBC0000B2B25D0012BE0D191F904600D79C068C1
:10CBD000002E22DA05F07F014CF0F2FB29462046B8
:10CBE0004CF02EFA2946134D0223402220464CF0E9
:10CBF00051FA95F8F031022B12D1812120464CF0E8
:10CC0000DFF9002385F8F031BFE70B490122BAE7CD
:10CC1000084B4A8883F8692CB7E74CF0BBFBDDE78B
:10CC2000002EB2DA012BB0D001212046FFF75CFFC5
:10CC3000ABE700BFC02900202936002010B50B4A01
:10CC400092F81432022B044607D0033B012B02D882
:10CC50000021FFF749FF002010BD92F8011248F0B3
:10CC600005FD0028F7DA01212046F2E7C02900205F
:10CC700070B5314C94F8146205461EB1012E50D0A7
:10CC8000002070BDD4F8F831C4F85C3CD4F8FC3115
:10CC9000C4F8603CB0F8B4331F2B0DD1D4F8F421A4
:10CCA000264B9A4208D194F80112012904D894F82D
:10CCB0000232013B0F2B0AD9202105204BF0F6FF51
:10CCC000022384F8F0312846FCF726FAD8E748F02A
:10CCD000CDFC0028F7DB94F81432013B022BCFD9AE
:10CCE000B4F86A1C21B3D4F8FC3184F8646C99421E
:10CCF00028BF1946D4F8603C5B1AC4F8603C042392
:10CD000084F8143240F20113A5F844310C4BC5E904
:10CD10005616C5E9543305F5A27128464CF083FA3E
:10CD2000AEE794F8011248F0A1FC0028A8DA3146D9
:10CD30002846FFF7D9FEA3E7C029002055534243F8
:10CD40009C400020F0B59C0827010E46154600EBDC
:10CD50000414A04206F1100605F1100508D103F0F5
:10CD6000030339443A4404EB83039C4223D1F0BDCE
:10CD700084469CED006A16ED045AD0ED016A56ED2A
:10CD8000037A90ED027A56ED025A26EE056A66EEB7
:10CD9000A76AD0ED037A05ED046A16ED016A45ED48
:10CDA000036A27EE257A67EE867A103005ED027A5F
:10CDB00045ED017ACDE7F4EC017AB1EC017A67EE4A
:10CDC000877AE2EC017AD0E74A09012350F8222061
:10CDD00001F01F018B40134214BF01200020704757
:10CDE00010B54C09012250F8243001F01F018A408F
:10CDF000134340F8243010BD10B54C09012250F8FF
:10CE0000243001F01F018A4023EA020340F8243055
:10CE100010BD80EA0120082241F2210103B2002B5B
:10CE2000B5BF81EA4303400098B280B2013AF5D120
:10CE3000704738B50C468D18AC4200D138BD14F897
:10CE4000011BFFF7E6FFF7E74840082243B2002B3B
:10CE5000BBBF5B0083F0D5034000D8B2A8BFC0B20F
:10CE6000013AF3D1704738B50C468D18AC4200D169
:10CE700038BD14F8011BFFF7E7FFF7E770B5066848
:10CE800005460C460020B44203D3731C2B6030705F
:10CE900070BD14F8011BFFF7D7FFF4E7DFED0A7A46
:10CEA000C0ED020A20EE270AB7EE007AC7EE007A3C
:10CEB00000230360C0ED017A70EEA77A80EEA77AB6
:10CEC00080ED037A704700BFDB0FC94090ED017A17
:10CED000D0ED007AC0ED020A30EE877AC0EE876AA4
:10CEE00030EE677AE6EE877AB0EE670AC0ED007A38
:10CEF0007047012303700023C364836403650364E4
:10CF000043644365836283657047DFED157A80ED86
:10CF1000010AF4EEE70AF1EE10FAC0ED020A80ED24
:10CF2000031AC0ED051A18DDB4EEE70AF1EE10FAA7
:10CF300008DC9FED0C7A80ED047A80ED0F2AC0EDBD
:10CF40000E2AD6E781EE007AC0EE207AF0EE006A73
:10CF500077EE877A86EEA77AEDE700238360E8E72D
:10CF6000BD37863500000000FDEEC07A17EE903A1E
:10CF70002033402B43D8DFED237A9FED237AB4EEA4
:10CF8000E70AF1EE10FA28DCDFED207A9FED1E7A39
:10CF9000B4EEE70AF1EE10FA22D4DFED1D7AB4EE1A
:10CFA000E70AF1EE10FA1EDD30EE670A37EEC00A2E
:10CFB00060EE007ADFED176A9FED177AA7EEA67A8A
:10CFC000DFED166AE7EE876A9FED157AA7EEA67A7F
:10CFD00020EE276AA6EE070A704730EE470ACEE732
:10CFE00030EE070AD4E79FED0F7AB4EEC70AF1EEF0
:10CFF00010FA44BF30EE270A37EE400AD8E79FED1B
:10D000000A0A7047DB0F4940DB0FC940DB0F49C0FC
:10D01000DB0FC93F9A7C2E36FAAF4FB93587083CF3
:10D02000A4AA2ABEDB0FC9BF00000000DFED027A10
:10D0300030EE270A98E700BFDB0FC93F10B51C464A
:10D04000334BB3FBF2F399429FED325AF0EE404A74
:10D05000F7EE005A53D207EE901A9FED2F7ADFEDCC
:10D060002F6AF8EE677AF8EE002A67EE877A07EE05
:10D07000102AB8EE477A27EE267AC5EE876A87EE41
:10D08000A64AB0EE440AFFF76FFFF0EE403AB0EE6A
:10D09000440AFFF7CBFF74EEA44A012C83EEA43AB6
:10D0A0001CBF35EEC04AF6EE006A33EE257A12BF99
:10D0B00064EE266AF0EE656A20EE224A86EE876A02
:10D0C000C4EE074A60EE227A75EEC35AC7EE876A4D
:10D0D000C5EE877AF0EE465AC0ED005AC0ED014A1F
:10D0E00080ED026AC0ED036AC0ED047A80ED065A55
:10D0F00080ED055A80ED085A80ED075A10BDF0EE1C
:10D10000454AB0EE456AF0EE456AF0EE457AE3E74F
:10D1100020A1070000000000DB0FC940BD378635A5
:10D120009FED010A002389E7F304353F2DE9F04123
:10D13000FCEEC07A13460A4617EE901AD0F8148017
:10D140008769C669056AB0EE600A89B2FFF776FFA3
:10D15000C0F814808761C6610562BDE8F081B0EE59
:10D16000E06AF0EEC07AB4EEE76AF1EE10FAF0EEA3
:10D17000406A4BDCB5EE400AF1EE10FA4BD0B4EE4B
:10D18000E76AF1EE10FAF0EE675A41D5B0EE465A72
:10D1900085EE257ADFED215A9FED215ADFED214AF8
:10D1A000A7EE255ADFED205AE5EE075A9FED1F5AEC
:10D1B000A5EE875ADFED1E5AE5EE075A9FED1D5A80
:10D1C000E7EE054AB7EE005AA4EE875AB1EE657A4B
:10D1D00087EE050AB4EEE76AF1EE10FA48BFDFED1C
:10D1E000167AF5EEC00A48BF37EEC00AF1EE10FA23
:10D1F00048BFDFED127AF5EEC06A48BF37EEC00ACD
:10D20000F1EE10FA48BFB1EE400A7047F0EE465A10
:10D21000B0EE675ABCE79FED0A7ABBE739094E3D8D
:10D22000E3B59EBE69A2163E88FA16BE45FE7FBFD4
:10D23000A7DFA8B499FB243FDB0FC93FDB0F4940B0
:10D240000000000044F25063984203DDA0F50C405A
:10D25000A0387047034B9842BCBF00F50C40A0308B
:10D26000704700BFB0B9FFFF48F69F43984203DD07
:10D27000A0F50C40A03870470028BCBF00F50C405A
:10D28000A030704791ED005A08B5B0EE450AFFF79F
:10D29000CDFEF0EE405AB0EE450AFFF765FE91ED87
:10D2A000015AF0EE404AB0EE450AFFF7BFFEF0EE3D
:10D2B000403AB0EE450AFFF757FE91ED023AB0EE64
:10D2C000405AB0EE430AFFF7B1FEB0EE404AB0EE6E
:10D2D000430AFFF749FE25EE806A63EEC07A24EE2A
:10D2E000847AC0ED017AF0EE467AE5EE077A25EE13
:10D2F000843A64EE806AC0ED037AF0EE437AE5EE9C
:10D30000667AA5EE067AE5EE436A23EE844A64EE79
:10D31000E34A65EEA35A80ED004A80ED025AC0ED63
:10D32000047AC0ED054AC0ED066A80ED077AC0EDCB
:10D33000085A08BD034600F1400100221A615A61F3
:10D340009A61DA6110338B42F8D11022002152F039
:10D3500001BD91ED007AD0ED047AE7EE077AC0EDD9
:10D36000047AD1ED006A91ED017AD0ED057AE6EE0E
:10D37000877AC0ED057AD1ED006A91ED027AD0EDA1
:10D38000067AE6EE877AC0ED067A91ED007AD0ED66
:10D39000077A77EE877AC0ED077AD1ED016A91EDD1
:10D3A000007AD0ED087AE6EE877AC0ED087A91ED42
:10D3B000017AD0ED097AE7EE077AC0ED097AD1ED6E
:10D3C000016A91ED027AD0ED0A7AE6EE877AC0ED35
:10D3D0000A7A91ED017AD0ED0B7A77EE877AC0ED7B
:10D3E0000B7A91ED007AD1ED026AD0ED0C7AE6EE7F
:10D3F000877AC0ED0C7AD1ED026A91ED017AD0ED19
:10D400000D7AE6EE877AC0ED0D7A91ED027AD0EDD5
:10D410000E7AE7EE077AC0ED0E7A91ED027AD0ED42
:10D420000F7A77EE877AC0ED0F7A91ED007AD0ED22
:10D43000107A77EE877AC0ED107A91ED017AD0ED0F
:10D44000117A77EE877AC0ED117A91ED027AD0EDFC
:10D45000127A77EE877AB7EE007AC0ED127AD0EDC5
:10D46000137A77EE877AC0ED137AD1ED017AD1ED98
:10D47000006A91ED027A67EEA77AE6EEA67AE7EE09
:10D48000077A90ED007AA6EEA77A80ED007AD1EDCA
:10D49000016A90ED017AA6EEA77A80ED017AD1EDCE
:10D4A000026A90ED027AA6EEA77A80ED027A90EDFC
:10D4B000037A77EE277AC0ED037A70472DE9F043BF
:10D4C000034685B000F11007054600261C46AC4611
:10D4D00012E0F8EC016A1EED047AD4ED007AE6EE73
:10D4E000C77AC4ED007A98450EF1100EF1D10434DC
:10D4F000BC420CF1040C03D0A7F11008E646F2E799
:10D5000001361C46B646BEF1040F1DD000EB0E1CC2
:10D51000A84604F1100907E0FCEC016A18ED047A52
:10D52000E6EEC77AC4ED047ACC45D4ED047A08F16E
:10D530001008F1D1D3ED006A87EEA67A0EF1010E44
:10D5400084ED047A6446DEE7042E03F1140305F14A
:10D55000040507F11007B9D100230093019302934A
:10D5600003936C4600231427F2EC017A00EB0315B9
:10D5700007FB030C6E466545C4ED007A1FD10133ED
:10D58000042B04F10404EFD104AD103100F140028A
:10D5900075ED017A00EB03170E461446BC4241EDCF
:10D5A000017A13D152ED016A87EEA67A013BA2F10E
:10D5B000140221ED017AEBD105B0BDE8F083F5EC62
:10D5C000016AB6EC017AE6EEC77AD4E7F4EC016AB8
:10D5D000B6EC017AE6EEC77AE0E71FB50C460246E4
:10D5E00069461030FFF76AFFDDED007AB6EE007A8B
:10D5F00067EE877A0120C4ED007ADDED017A67EEEF
:10D60000877AC4ED017ADDED027A67EE877AC4EDA0
:10D61000027A04B010BDB5EEC00AF1EE10FA08B5FA
:10D6200006DB4DF01DFCB4EE400AF1EE10FA01D716
:10D630009FED010A08BD00BF000000002DE9F04188
:10D64000044626461C3004F1640250ED017AB1EC28
:10D65000010A77EE807A40ED017AFBF7A3F81830E3
:10D660009042F2D12C4F6268D7F8943125699B1A09
:10D67000A2680135934225612BD904F13008F36A81
:10D68000012BC3BF03F1FF3307EE903A96ED0A7A00
:10D690009FED220AC4BFF8EEE77A87EE270AFFF76C
:10D6A000BAFF4645D4ED057A15D0F4EEC07AF1EE16
:10D6B00010FA06F11806E2D5237B4BBBD7F894216C
:10D6C000626000222361A261E36222636364A26458
:10D6D000E365BDE8F081F4EEC07AF1EE10FAEBD428
:10D6E00007EE905AD4ED066AF8EE677A022386EECA
:10D6F000A77AD4ED0C6A84ED067A86EEA77AD4ED8B
:10D70000126A84ED0C7A86EEA77A84ED127A00E034
:10D7100003232370DDE700BFC029002000000000C4
:10D7200070B52DED028B0378012B04463CD10569C1
:10D73000254E25B9426812B9D6F89421426094ED7D
:10D74000068A30EE088A013584ED068A256104F1E7
:10D750001C00FBF727F86268D6F894319B1AA26880
:10D76000934221D9E36A012BC3BF03F1FF3307EED4
:10D77000903A94ED0A7A9FED150AC4BFF8EEE77A65
:10D7800087EE270AFFF747FFD4ED057AF4EEC07A5B
:10D79000F1EE10FA0ED5237B4BB9D6F894216260D6
:10D7A00000222361A261E362BDEC028B70BD032302
:10D7B0002370F9E707EE905AF8EE677A022388EEB5
:10D7C000277A84ED067AF3E7C029002000000000E4
:10D7D00008B52DED028BF0EEC08AB0EE408AB7EEB0
:10D7E000000A30EE680AFFF716FF9FED0E7ADFEDB4
:10D7F0000E7AE8EE877A9FED0D7AA7EEA87ADFED34
:10D800000C7AE7EE287AB5EEC08ABDEC028BF1EE19
:10D8100010FA20EE270A44BFDFED067A37EEC00A81
:10D8200008BD00BF306E99BC2716983D843459BEA0
:10D83000A40DC93FDB0F494060EEA00AE0EE000AEC
:10D84000B0EE600AE7E660EEA00AE0EE000AE1EE64
:10D85000010AB0EE600ADEE62DE9F74F90469DF82A
:10D860003020002A0CBF4FF0200A4FF0300A0D9AEA
:10D870001C1E05460F46BABF64424FF0010B4FF025
:10D88000000B12F8011B01B14CB9BBF1000F2DD1F7
:10D89000264636B9A1464FF0FF340D9E0FE0013CFD
:10D8A000EFE7BD4202D251462846C047013EF0E7AD
:10D8B000BD4203D201922846C047019A164632461D
:10D8C00012F8011B0029F3D10D9BA9EB03094E446B
:10D8D000BBF1000F06D0A146B9F1000F09DC002C06
:10D8E000A8BF3619304603B0BDE8F08F4FF00009ED
:10D8F000D3E7BD4202D251462846C04709F1FF395D
:10D90000EAE70FB437B50C4D06ABD5F8701C53F8E9
:10D91000042BD5F86C0C019349F0F6FC0446D5F8BD
:10D92000240203F043FB0028F9D0204603B0BDE8F1
:10D93000304004B0704700BFC02900200EB403B5CA
:10D9400003AB084953F8042BCDE9003001A849F096
:10D95000DBFC019B00221A7002B05DF804EB03B0FF
:10D96000704700BFF98700080CB430B52C4CD4F8D0
:10D97000743CA5B01BB9D4F8783C002B39D094F88E
:10D980007C3C994206D9012303FA00F0D4F8803C8C
:10D9900018422ED0D4F894114FF47A7304A8B1FB36
:10D9A000F3F203FB12131F49FFF7C8FF04AB034454
:10D9B000289A1D490393054629AB03A8029349F011
:10D9C000A3FC039B591C03910A211970039B591C4A
:10D9D0000391002119700246D4F8740C90B10368C9
:10D9E0001B6A03B19847D4F8745C04AC14F8011BAB
:10D9F00021B925B0BDE8304002B07047284603F099
:10DA0000ABFAF3E7D4F8783C002BF2D015440222AD
:10DA1000009204A9AA18FD2027F0B6F9E9E700BF93
:10DA2000C029002033B506089B870008174A38B57F
:10DA3000D2F8845C033005EB9003B3F5007F19D86E
:10DA400002F68844C2F8843C114A02EB810120F0BE
:10DA50000300D1F89023C3F500730244C1F890236A
:10DA60009B000C4A0421002004EB8504FFF77CFF97
:10DA7000204638BD0021084A0846FFF775FF074ACF
:10DA8000136843F0007313600024F1E7C0290020FD
:10DA9000B83A00203FB5060863B50608785601205D
:10DAA0002DE9F84305460068FCF769F80D2804469F
:10DAB00007DD1C4A00210520FFF756FF0020BDE8C6
:10DAC000F883194E06EB80088700D8F82892B9F140
:10DAD000000F18D107216420FFF7A8FF0146C8F8FE
:10DAE000280208B9114AE6E76422494652F032F9A1
:10DAF0000F4AD8F8283224B202EBC402C3E900234B
:10DB0000DB615B63DB643E446879D6F82832182415
:10DB100004FB003200211046C2E903119560117523
:10DB20000430CCE771B50608C029002096B5060878
:10DB30001810060803685A1C026019700368090A65
:10DB40005A1C02601970704703685A1C02601970F1
:10DB500003685A1C02600A0A1A7003685A1C0260A1
:10DB60000A0C1A700368090E5A1C0260197070477B
:10DB700003685A1C02600A0A1A7003685A1C026081
:10DB80001970704738B504460068154652F0E2F83F
:10DB900023682B44236038BD38B504460068154619
:10DBA00050F0B6FF23682B44236038BD03685A1C2D
:10DBB00002601878704703685A1C02601A4612F80F
:10DBC000021B0260587841EA00207047026810B5D5
:10DBD000531C0360134613F8021B0360D31C5478D4
:10DBE000036093781B0443EA04230B43111D016077
:10DBF000D07843EA006010BDD1E900329A4206D0E5
:10DC00005A1C0A6008B11B7803700120704700207D
:10DC10007047D1E900239B1A012B10B50446084632
:10DC200004DDFFF7C8FF2080012010BD0020FCE7C5
:10DC3000A0F16103192B98BF2038704730B50A4412
:10DC40000546914201D1002011E015F8013B11F881
:10DC5000014BA3F141001928A4F1410098BF2033E2
:10DC6000192898BF2034181B01D1002CE9D130BDF0
:10DC70006FF00042E2E710B50388827803F00301F9
:10DC80000C24013A04FB01221149847901EB420280
:10DC9000A3F5FA63B2F8EE2040F2B5519B0801FB00
:10DCA0000323C278013A13440279182101FB0323AC
:10DCB000427900893C2101FB0322064B234401FBEE
:10DCC00002334FF47A720021C3FB020110BD00BF82
:10DCD000B00F060880436D38F8B519460446002396
:10DCE00010464FF47A724CF0C5FA244B3C2503449D
:10DCF00093FBF5F005FB103390FBF5F105FB1100EC
:10DD000060711820A37191FBF0F300FB131140F236
:10DD1000B550217193FBF0F100FB1133B3F5896F1E
:10DD20004FEA810526DA40F2DA218B4224DCB3F592
:10DD3000B77FB4BF00200120114E182101FB0066FF
:10DD40000B2136F811709F4201DD0139F9D105F53B
:10DD5000FA65054425804D1CA5700C2505FB0011B6
:10DD60000848228100EB41010133B1F8EE105B1A43
:10DD7000E370F8BD0320DFE70220DDE780BC92C737
:10DD80009E100608B00F0608F0B5294D07460E464E
:10DD90000FCD8DB06C460FC40FCD0FC495E80F00AA
:10DDA00084E80F0017F003033FD1642197FBF1F2E1
:10DDB00001FB127242B94FF4C87297FBF2F302FBF7
:10DDC0001373003B18BF01237A1EC3F11D03002A01
:10DDD000019340F26D13114607FB03F3B8BFB91C62
:10DDE00003EBA1036FF0630192FBF1F10B444FF4DD
:10DDF000C87192FBF1F213442533072493FBF4F22C
:10DE0000C2EBC2029B1A013E6D46002155F8040F79
:10DE100001310344B14293FBF4F2C2EBC202A3EB23
:10DE20000203F3D1C01A0DB0F0BD0123CCE700BF4F
:10DE300000110608084B53E9021251EA020309D007
:10DE4000064BD3F894315B1842F10002C0E900326E
:10DE50000120704700207047D83E0020C0290020D4
:10DE600037B505466846FFF7E5FF044638B1DDE9FA
:10DE700000232846FFF730FF204603B030BD40F2B4
:10DE8000011328806B80A880A8712881F4E737B53A
:10DE90000546FFF7E5FF044650B1074B0DF10602BA
:10DEA000B3F82034ADF806302946284647F006FE80
:10DEB000204603B030BD00BFB83A00202DE9F04144
:10DEC000044686B094F83030042B13D8DFE813F002
:10DED000150005005D00E9003601DFF8688204F1F5
:10DEE0001C0701AA39464046FEF721FD01280CD047
:10DEF00002282AD006B0BDE8F081924848F0FEF929
:10DF00004FF6FF73238401233CE0019D0DB12B7874
:10DF100063B98C48FDF784FF237EDD0618D548F0F1
:10DF2000EDF94FF6FF73238402232BE0EE7A3007DE
:10DF3000D7D40B2204F13101284650F065FD0028AA
:10DF4000CFD1637E7340D90604D57E48FDF768FFC4
:10DF5000042317E0AA8A6B8B43EA02437A4A63627E
:10DF6000D2F81022EB69A3605202B3FBF2F102FB7C
:10DF7000113109B113445B1A7248E3606676FDF70C
:10DF80004FFF032384F830309CE76F4E96F8E03162
:10DF9000002BAFD104F11C0806F5DC7701AA41463D
:10DFA0003846FEF7C4FC012859D1019D002D38D018
:10DFB0002B78E52B01D0002BF0D1644BEB1A48BF36
:10DFC00003F2FF13B3F5805F4FEA632003D3FEF73C
:10DFD00017F84FF0FF305E4901EB0010FAF7A2FA94
:10DFE00001F5D070FDF71CFF20220021284651F0DA
:10DFF000B1FED4F831302B60D4F835306B60B4F812
:10E0000039302B8194F83B30AB72637EEB7203A8FE
:10E01000FFF73DFF38BB6FF07E032B7447236B7413
:10E020003AE096F8B831022B92D096F8E031002B06
:10E030008ED10922C6E97D3386F8E02186F8F031D9
:10E04000D6F8CC2186F8EC313E48D6F81432C6F822
:10E05000E421C6F8E831FEF77FFA01289ED00228B5
:10E060003FF476AF46E79DF80E209DF80F3043EA67
:10E070004213BDF80C20A2F2BC7243EA42232B8269
:10E080009DF811309DF812205B0143EA52039DF880
:10E09000102043EAC223EB812B8A2B83EB89EB828E
:10E0A0006FE7237E9A0608D5E0690023112202A9B2
:10E0B000FDF7B4FF01287FF41DAF204648F01EF99C
:10E0C0002269237E9AB91B0708D51F4B93F8982124
:10E0D000002A7FF40FAF072283F89821002384F8E9
:10E0E0002830E36A204606B0BDE8F041184703F047
:10E0F000F70213F0040322760AD0E26AA168002333
:10E10000204684F8283006B0BDE8F041FDF72CBF6A
:10E11000122AE3D1E26AA263626A84F83C300421E5
:10E120002046C4E90B22C4E9023384F82810636353
:10E13000636206B0BDE8F04148F0E0B80020E36A51
:10E140002070D0E7546200209C600020B450002072
:10E15000B46000202DE9F34103780446002B76D00B
:10E1600090F82830013B082B71D8DFE803F005094F
:10E17000475B4C6170666B0002B0BDE8F0419DE604
:10E18000344B4568D3F81072D3F818327F021D4023
:10E19000216B2046FDF77EFE05EB0108474506464C
:10E1A00026D880B1D4E901329A422CBFA260A36084
:10E1B000002384F82830E36A002B48D0204602B0C0
:10E1C000BDE8F04118472169207E01AA4AF0CEFE41
:10E1D00001283CD123696361019B236163683B444F
:10E1E0005B1B6360236BDB1B2B4423633546CFE74C
:10E1F0000028D7D163680B446360D3E702B0BDE861
:10E20000F041FEF729BB0121FEF798FA01281ED143
:10E21000216C0023204684F8283002B0BDE8F0418C
:10E22000FEF76EBB002102B0BDE8F041FEF786BAF2
:10E2300002B0BDE8F041FEF721BA02B0BDE8F041FE
:10E24000FEF725B902B0BDE8F041FEF785B902B08E
:10E25000BDE8F0819C600020F0B50124B0FBF4F52E
:10E260008D4203D200261CB91C70F0BD4C43F5E76B
:10E27000B0FBF4F5B4FBF1F704FB15002EB9002D4B
:10E2800003DC8C420CD33C46EDE7092D08DD002A67
:10E290000CBF572437242C4403F8014B0136F2E716
:10E2A0003024F8E703463038C2B2092A0FD9A3F167
:10E2B0006102052A02D8A3F157007047A3F1410279
:10E2C000052A02D8A3F1370070474FF0FF3070479E
:10E2D00070B50446944208461546B4FBF2F602D3E4
:10E2E0003046FFF7F5FF05FB1644024B1B5D00F8B7
:10E2F000013B70BDBBB50608B5EEC00ADFED2D7A57
:10E30000F1EE10FACCBF30EE270A30EE670ADFEDEF
:10E310002A7A20EE270A30B5FDEEC07A87B017EED4
:10E32000904A054684EAE470002303A9A0EBE47058
:10E33000CDE90033029347F0D1FF002CB4BF2D2369
:10E34000202303A88DF800304BF0A2F9012822D138
:10E3500030238DF8013043F23003ADF8023003A9C9
:10E36000684652F0AFFB68464BF092F9C41EE4B227
:10E3700022466946284650F0CBFB00232B550F4917
:10E38000284652F09FFB0DEB0401284652F09AFB01
:10E39000284607B030BD022805D130238DF8013062
:10E3A0008DF80230DBE7032804BF30238DF80130FD
:10E3B000D5E700BF6F12033A00007A44FBEE06086F
:10E3C00030B50278202A034600F10100F9D0092A6D
:10E3D000F7D02D2A4BD10346BFEE000A9FED3C7AC1
:10E3E0001A46F2EE046A134612F8010BA0F130014E
:10E3F000CCB2092C41D92E280BD1F2EE046A114679
:10E40000B0EE666A0B4611F8012B303AD0B20928FB
:10E410003CD91A7802F0DF02452A53D15A782D2AC6
:10E420003FD102330120013B00220A2513F8011FCE
:10E430003039CCB2092C3AD9B2F59A7F1346DFEDC8
:10E44000256A28BF4FF49A731A46F7EE007A072A16
:10E4500030D8DA086FF0070101FB0233F2EE046AEC
:10E4600063BB88B3C7EE276A20EE260A30BD2B2A8D
:10E4700008BF0346B7EE000AB0E707EE901AF8EEC1
:10E48000E77AE7EE267AB0EE677AACE707EE902AF5
:10E49000F8EEE77AC7EEA65A66EE866A37EE257A78
:10E4A000B0E72B2A14BF013302330020BBE705FB82
:10E4B0000212BBE767EEA67A083AC8E767EEA67ACB
:10E4C000013BCDE7F7EE007A67EE276ACCE700BFA5
:10E4D0000000000020BCBE4C70B5034610F8012BB4
:10E4E000202AFAD0092AF8D02D2A0ABF034601258E
:10E4F0004FF0FF35591E00240A2611F8010FFFF7CF
:10E50000D1FE092802D905FB04F070BD06FB040406
:10E51000F3E710B50023802804D893420AD2C854E8
:10E52000581C10BD934205D060F07F04CC54C00944
:10E530000133F0E74FF0FF30F3E7F8B5144D2B78D7
:10E540007E2B23D1012229460020FEF772FC114FB9
:10E550006C1C228862B1A31DBB4217D2A618BE4212
:10E5600014D2052A12D92146FEF763FC3446F0E79F
:10E5700002222146FEF75DFC6388074AC31A043471
:10E58000641B5842A2F8BC455841F8BD0020FCE786
:10E590000040000800800008B83A00202DE9F04F44
:10E5A000724BDFF8DCB18FB0A3EB0B02CDE9012396
:10E5B0004FF00308102200210AA851F0CBFB019B69
:10E5C0000993029B08936A4BCDF81CB01A69002A84
:10E5D000BFBF684A5A6002F188325A600124F322B0
:10E5E000DA604FF000097E23224604A907A88DF8BF
:10E5F0003440CDF830908DF81030FAF7AFF9484537
:10E60000C0F2A180224604A94846FEF712FC5A4CEB
:10E61000ADF81200594B9C423CD30024022205A9BC
:10E6200007A8ADF81440FAF799F9A042C0F28B8020
:10E63000BDF81200022205A9FEF7FBFB0222ADF88D
:10E6400012000DF1120107A8FAF788F9A0427ADB4F
:10E650000B9880B1079B089A0344934273D80AAB86
:10E66000C0F104022146184451F074FB0AA907A81E
:10E67000FAF7D0F80C900C9B002B64DB9DF834204B
:10E6800022B13B490A6942F000420A61B3FA83F3BE
:10E690005B0959E062888DF81990C2F30B06B31D2F
:10E6A000ADF814302388C3F30B011B0B8DF8183021
:10E6B0001304ADF816101ED4062205A907A8FAF710
:10E6C0004DF900283FDBBDF81200062205A9FEF730
:10E6D000B0FB676805463246394607A8FAF73EF9A7
:10E6E000002830DB324639462846FEF7A2FBADF85B
:10E6F000120014348EE700273D460135EDB20622A4
:10E7000005A907A88DF81950FAF728F900281ADB8F
:10E71000BDF81200062205A9FEF78BFB6168824650
:10E720003944324607A80391FAF718F900280ADBA2
:10E73000039932465046FEF77CFB032DADF81200DC
:10E740003744DAD1D5E70023B8F1010808D0002B0F
:10E750003FF430AFFFF7F1FE20B10FB0BDE8F08F0E
:10E76000002BF7D1052004F0CFFE00BF0080000889
:10E77000003C024023016745A0190708C81E07088E
:10E7800000400008034AD2F8C03523EA0003C2F86B
:10E79000C0357047B83A002003460649064888420B
:10E7A00001D3002070470288C2F30B029342F9D0D4
:10E7B0001430F4E7C81E0708A019070870B544888C
:10E7C0000B460546C4F30B0422460021184651F0BF
:10E7D000C1FA2969084A9142034607D3074A914280
:10E7E00005D22246BDE8704050F092B919B1BDE89B
:10E7F00070401846084770BDC81E070883230708E5
:10E8000010B4B0F902404288002C0B4641685DF814
:10E81000044BBEBFC2F30B02DBB203FB0211CDE718
:10E8200030B5094B094CA34200D330BDB3F90220E7
:10E830005988002A06DA5A68DD68C1F30B0100FB2B
:10E8400001222A601433EEE7A0190708C81E070842
:10E8500030B502460144002012F8015B082480EA2A
:10E86000050343F3000323F0730383EA5003D8B294
:10E87000631E13F0FF044FEA5505F0D19142EBD12E
:10E8800030BD2DE9F04F87B0CDE903230025804648
:10E8900001910095039B4046EC0003EBC50AFAF793
:10E8A000FDFF002800F09780002201214046FAF782
:10E8B000DFFF0290002800F08E8098F804309A075D
:10E8C00006D4029A049B10461D7007B0BDE8F08F75
:10E8D000F0214046FAF7ECFF00287CD0039BA4F11E
:10E8E00008024FF0000B0126134434465F4605939F
:10E8F000019BB3B3082C34D804F1FF3943FA09F96A
:10E9000009F0010949464046FAF789FF002862D01C
:10E91000002201214046FAF7ABFF024600285AD0F8
:10E9200098F8041001F0600CBCF1600F4FEAD110B0
:10E9300037D0019B1BB1082C01D88145C1D120B330
:10E940001AF8071031437600013416F0FF060AF872
:10E950000710E4B2CCD10137FFB2082F21D0012635
:10E96000C6E75DB1009BA34208D9059BDA5D16425C
:10E9700014BF4FF001094FF00009C3E7009B1B1BB8
:10E98000D3F1000949EB0309BCE7880940EA5111BA
:10E9900011F0010F1AF8071008BFA34621EA06017B
:10E9A000D1E7402C11D9072150460292FFF750FFC2
:10E9B0009AF80740029A844207D10135EDB2BBF1C3
:10E9C000000F3FF47FAFCDF800B0049B1B78AB4243
:10E9D0003FF660AF76E7002274E700BF90F83C2076
:10E9E000034602F0FF0012B1002283F83C2070477A
:10E9F0004FF48053838170474FF4006383817047E5
:10EA00004FF40063838170474FF400638381704744
:10EA10004FF40063838170474FF400638381704734
:10EA20004FF4006383817047324BF0B51888DC895E
:10EA3000B3F91850B3F91270B3F908E0B3F92060D4
:10EA4000001B9C896043B3F9164005EBE035E402F6
:10EA500094FBF5F404EBE034A4F57A60B3F90650C6
:10EA6000DC6100FB00FC4FEA2C3C45430CFB07F744
:10EA700000FB0EFEED12B3F9100005EBE725B3F92C
:10EA800004700CFB00F0001405EB8705B3F80AC016
:10EA90005B6A00EB6E30B54002300235A3EBA50592
:10EAA00080104CF2503300F5004033416B430CFBB7
:10EAB00000F04FEAD03055BF5B00B3FBF0F3B3FB7F
:10EAC000F0F35B0071B1181240F6DE354043684345
:10EAD000094D00145D4300EB254000F6CF6003EBC9
:10EAE00020130B6022B10A235C4308342411146004
:10EAF0000120F0BDC062002043E3FFFF012070470A
:10EB0000012070472DE9F74F604E9046B38DB26AF1
:10EB1000B6F93CC0B6F93A70B6F938B0C3EB221575
:10EB20005B00C3EBE203B6F92E206D435343B6F905
:10EB300030202D135543AD1305EBE325B36C009343
:10EB4000A5F5FA30B6F936307564894680FB001EAB
:10EB5000DA1703FB0EF401FB0244A3FB0132144459
:10EB6000B6F9342082FB00A21B0A120343EA0463B5
:10EB700042EA1A524FEA0A3A13EB0A0342EB242202
:10EB8000B6F832A002F500420192A3FB0A23019AD3
:10EB90000AFB023A4FEAEA734FEA6A0253EA6A0A48
:10EBA0004FF000045ED087FB00704FEAEC7A0CFB5C
:10EBB0000EFE400401FB0AEE40EAD730ACFB011C1C
:10EBC0007F047F180099F4444CEB0000C1F5801CD1
:10EBD0000CF00041E71941EA5C014FEACC7CBCEB48
:10EBE000070C40F6354400EBCB0061EB0001ACFBB9
:10EBF000040C04FB01C14BF03DFB84460746430B6C
:10EC0000B6F942004A1343EAC14300FB02FEC417AF
:10EC100003FB04EEA0FB03407044624303FB0022AD
:10EC2000A4FB03431A44B6F94030640E44EAC2140C
:10EC30004FEAE37E03FB01F0E4190EFB0C00A3FB9B
:10EC40000C3738444FEAD34343EA403341EB626226
:10EC5000E41842EBE042B6F93E30240A44EA02648A
:10EC600004EB0314B9F1000F02D0240AC9F80040E4
:10EC7000B8F1000F05D005EB850580352D12C8F8D9
:10EC80000050012003B0BDE8F08F00BFC06200203B
:10EC900031B10A4BD3ED197AFDEEE77AC1ED007A76
:10ECA00052B1064B9FED067AD3ED1A7A67EE877A5A
:10ECB000FDEEE77AC2ED007A01207047C0620020C5
:10ECC0000000C8422DE9F74FCDE90012574AB2F8CB
:10ECD0007A30D16EB2F87660B2F87C701B02C91A35
:10ECE000B2F878306EEB0E0EA3FB010403FB0E446A
:10ECF000B2F87430C00940EA44601B04C018A6FB97
:10ED0000013506FB0E55B2F872604FEA132343EA51
:10ED100005634FEAC6364FEAE41444F100049B1938
:10ED2000A7FB012607FB0E664FEAD25242EA4622B3
:10ED30004FEA252545F10005F61512F5FA6C46F166
:10ED4000000BBCF5FA6F7BF1000750DA02FB06F806
:10ED5000A2FB02794FF0050A09EB4809A7FB0A78E4
:10ED60000AFB09884FEA570949EAC879BF08B0EB9E
:10ED7000090947EA887764EB6804DF1B3B462C4FA0
:10ED800065EBA805BC454FF0FF377BEB070748460E
:10ED900022DA40F6AC57D21946F100065643A2FBE0
:10EDA000027202EB46024FEAC208FE00BE1B48EAAE
:10EDB000577862EB0808361844EB08044FF00B084C
:10EDC0003046A7FB087608FB02627F0847EAC27755
:10EDD000DF1B3B4665EB620501FB0EFEA1FB01124A
:10EDE00002EB4E02C90F41EA4201BCEB010C009A52
:10EDF0009AB10E4AD2F88010A1FB033201FB052222
:10EE00005B0D43EAC2231B1A4FEA625262EB040213
:10EE1000DB0B43EA4243009A1360019B0BB1C3F83A
:10EE200000C0012003B0BDE8F08F00BFC062002029
:10EE300024FAFFFF01207047B0F900305943084B16
:10EE4000994208DBB1F5000F07DA0029B8BFFF319E
:10EE5000081200B270470348FBE747F6FF70F8E777
:10EE600001FF7FFF0080FFFF064B0022C3F88420D4
:10EE7000C3F88820C3F88C200022C3F8902001201A
:10EE8000704700BFC0620020104B1A68104BD3F8C7
:10EE90009010521AFA2A16D8D3ED217AFDEEE77AAD
:10EEA00017EE902AD3ED227AC286FDEEE77A17EEAE
:10EEB000902AD3ED237A0287FDEEE77A17EE903A97
:10EEC0004387012070470020704700BF542B00206B
:10EED000C062002090F85F3230B53BB990F85D1207
:10EEE00090F85E320124DAB2914200D830BDB0F819
:10EEF000665204FA03F22A43A0F866220133F2E7CD
:10EF00004379024613F0010006D0D2E90731D268F6
:10EF10005B1A013A03EA020070474379024613F094
:10EF2000020007D0936A516A1269013B5B1A013AE9
:10EF300003EA0200704710B5437913F00103044659
:10EF40000ED0FFF7DDFF034650B1226A6369E16826
:10EF50009B5C0132B2FBF1F001FB1022DBB22262BA
:10EF6000184610BD43799B070AD5436A8269D1547C
:10EF7000436A02690133B3FBF2F102FB11334362CE
:10EF8000704741717047D0E90920131A584258411F
:10EF90007047024BD3F894305B681847C06200207A
:10EFA000024BD3F8943008309B681847C0620020A9
:10EFB00001207047012070470120704701207047F1
:10EFC0000120704731B10C4BD3ED267AF8EEE77A89
:10EFD000C1ED007A7AB1084BDFED086AD3F89C30B6
:10EFE000A3F5D543333B07EE903AF8EEE77A87EE88
:10EFF000A67A82ED007A7047C06200200000C84205
:10F000000120704701207047094A30B505460A249F
:10F0100000201368AB4205D1D3688B421EBF431C4E
:10F02000D160D8B2013C02F11402F2D130BD00BF70
:10F030009C050020044B03EB8003D3F8A0300BB1F8
:10F040009B681960704700BFC062002008B5FFF7D9
:10F05000F1FFBDE808401FF05BBD7047044B40F274
:10F06000FF7203EBC0039142A8BF1146998070471D
:10F07000283F00200C4A13787BB10C4B93F8E0102A
:10F0800059B193F8E11059B150680021FA2883F87A
:10F09000E110A8BF4FF0FF3070476FF001007047DC
:10F0A0006FF00200704700BF60100020C0620020B7
:10F0B0000B4B93F8E2206AB193F8E3206AB1002287
:10F0C00083F8E320074B9868B0F5967FA8BF4FF010
:10F0D000FF3070476FF0010070476FF0020070471B
:10F0E000C062002060100020024BD3F8E4305B685F
:10F0F000184700BFC0620020024BD3F8E4309B6881
:10F10000184700BFC0620020024BD3F8E430DB6830
:10F11000184700BFC0620020014BD868704700BF8D
:10F1200060100020044B93F8E83013B1034B1869CA
:10F1300070476FF001007047C0620020601000202F
:10F140002DE9F041062592F9007086B06B43144614
:10F1500012F80580A0EB080EA0EB070CBEF1000F23
:10F16000B8BFCEF1000EBCF1000FB8BFCCF1000C5F
:10F17000E645B8BF541905F10605B8BF4FFA88F740
:10F18000AB421646E4D11A4433786588BB420BD1B2
:10F1900073884D1BCB1A002DB8BF6D42002BB8BF32
:10F1A0005B429D42C8BF34460636B242ECD1637919
:10F1B000049323790393638802932378054ACDE966
:10F1C0000013034603210120FEF7CEFB204606B0C4
:10F1D000BDE8F08165B606084B1EDBB2062B9CBF6E
:10F1E0001C4AD25C1C4BF0B5A3F1580488BF4FF405
:10F1F0008072002808BF1C46234687B013F9087B9D
:10F200001888C8B9154B93F8E900A3790593A3882A
:10F210000493A378039323880091CDE90123104A36
:10F22000104B0321002818BF13460F4A0120FEF798
:10F230009BFB204607B0F0BD161AD51B002EB8BFA9
:10F240007642002DB8BF6D42AE42BCBF1C4647B2ED
:10F250000833D5E76C110608CC100020C0620020EE
:10F260000FCC0608AAEF06089EB6060808B5006887
:10F2700049F06FFB014BD866012008BDC062002039
:10F2800008B5006849F065FB024BC3F88000012017
:10F2900008BD00BFC062002038B514460D460029E5
:10F2A00043D0344B9FED347AD3ED3B7AB3F9082148
:10F2B000F8EEE77A06EE102AC7EE876AB3F9042162
:10F2C000D3ED3C7AF8EEE77AB8EEC66AC7EE875A15
:10F2D00007EE102AD3ED3E7AB3F90021B8EEC77AD3
:10F2E000B8EEE70AA6EE867AD3ED3F7AF8EEE77A33
:10F2F000E6EE877AA6EEA70A07EE902AB3F9062172
:10F30000B3F9023106EE102A07EE103AB8EEC66ADB
:10F31000B8EEC77AF8EEE77AA6EE867AE6EE877A56
:10F32000A5EEA70A4BF046FE28600CB3114BDFEDAB
:10F33000126A93ED3C7AB3F9F420B3F9F630B8EEE3
:10F34000C77A07EE902A87EE260A07EE103AB8EE43
:10F35000C77AF8EEE77A20EE070AB6EE007AA7EE53
:10F36000870ADFED067A20EE270A4BF023FE2060A5
:10F37000012038BDC06200200000F04A0000C842F1
:10F38000094B10B553F8304007EE901A5CB1F8EE17
:10F39000E77A94ED047A94ED030AA7EE870A4BF01E
:10F3A00009FEA368186010BD283F002010B50C4B63
:10F3B0000C4C1B68D4F80C011B1AFA2B06D904203C
:10F3C00019F08CFD002084F8100110BD11B1D4F8A3
:10F3D00014310B6012B1D4F8183113600120F4E736
:10F3E000542B0020C06200202DE9F0410C4DDFF8C5
:10F3F00034802C686B6901271C400CB9BDE8F08192
:10F40000B4FA84F3C3F11F0307FA03F608EB83038E
:10F4100024EA0604D3F81C01036898476E61ECE700
:10F42000003C0140C0620020F8B583681C68637925
:10F43000DB0724D5A57994F85C3205F001073D4639
:10F44000F3B1E06B43681A68D36AC3F34E035362A7
:10F4500094F86D32012B07D094F8613223B1B4F8DF
:10F4600068320133A4F8683285F0010146F098FD56
:10F470000023A4F866324FF08073C4F85C32F8BD04
:10F4800094F85F62012E04BF94F85D3284F85E3216
:10F490002046FFF71FFD4EB9012384F85F3287EA4B
:10F4A0000301E06BBDE8F84046F07ABD002384F824
:10F4B0005F323946F5E7F0B52DED028B83B00E468D
:10F4C000154642F095FB002869D0364B364C1B6838
:10F4D00094F85C2103F00203002A45D0002B59D098
:10F4E000324F0DF1060022F0B5FFD7F8EC23BDF83E
:10F4F00006309FED2F7A9B1A07EE903AF8EEE77AE6
:10F50000F0EE408A87EE870A07F58067DFED297AFB
:10F5100020EE270AFDF78AFD97ED008AA0EE688AA3
:10F520003CF06AFCD4ED5A0AD0ED057AB0EE480AF8
:10F5300070EEA70AFEF780F97EB1DFED1F7A9FED2E
:10F540001F7A20EE000A20EE270AC0EE077A9FED10
:10F550001C7A77EE877AC6ED007A0DB1194B2B60D5
:10F5600003B0BDEC028BF0BDA3B1B4F98E3101EE56
:10F57000103AB4F98C3100EE903AB4F98A3100EEC9
:10F58000103AB8EEC11AF8EEE00AB8EEC00AFEF77B
:10F590005AF9D1E7D4F8A43193ED340ACCE79FEDC2
:10F5A0000A0AC9E714570120C06200201095002004
:10F5B0000000C84235FA8E3CCDCC9C3F00409C46B2
:10F5C00082E6C547331390430000000070B504463F
:10F5D000012023F0B9FD58B103684BB11A4A2379D1
:10F5E00092F83D1099422DD092F83C209A4229D0B1
:10F5F000164B5E68710612D500212720FAF7FCFA37
:10F60000002105462620FAF7F7FA1DB12A6823687B
:10F610009A4217D018B1026823689A4212D0F203B6
:10F6200008D500212520FAF7E7FA18B12268036807
:10F630009A4207D02079112804D0A0F12103584222
:10F64000584170BD0120FCE75003002014570120F1
:10F6500008B5202151F045FA0346184623B1027837
:10F66000202A03F10103F8D008BD70B50D461446F9
:10F67000FFF7EEFF0646A0B1FEF72EFF40F634037B
:10F680009842A8BF1846B0F5617FB8BF4FF46170CB
:10F69000A0F561731922B3FBF2F32B7023780133C9
:10F6A00023703046FFF7D4FF0646A0B1FEF714FFE3
:10F6B00040F634039842A8BF1846B0F5617FB8BF42
:10F6C0004FF46170A0F561731922B3FBF2F36B7014
:10F6D000237801332370304670BD144901EB80005C
:10F6E00070B5D0F8A801F0B1114A0C2303FB002239
:10F6F00092F90130581C17D0507AA0B119448C25CA
:10F700000C4E91F8B841117A002014226B435D1819
:10F71000013A36F81550214410FA85F0F7D1142338
:10F72000B0FBF3F080B270BD0020FCE7C0620020A7
:10F73000682F0020202C002038B503200D461446E9
:10F74000FFF7CBFF07EE900A8DB19FED0B7AF8EE35
:10F75000677AF0EE006A67EE877AB8EE047AA7EE71
:10F76000A67ADFED067A67EE277AC5ED007A0CB14E
:10F77000034B236038BD00BF6740533A00007A4412
:10F7800033139043064A002352F8041B814204D0ED
:10F790000133042BF8D1002070470120704700BFCF
:10F7A0006864002010B5064A0423002152F8044B77
:10F7B000844208BF42F8041C013BF7D110BD00BFD2
:10F7C0006864002010B5427A044632B101464068B0
:10F7D00051F80A3B98470023637210BD10B4447A75
:10F7E000621C0444D2B24272A172037A934202D8DC
:10F7F0005DF8044BE6E75DF8044B7047EEE710B5A3
:10F8000003681A79022A044602D1987A49F092F8DC
:10F8100000232371236010BDF0B50D4B0D4E04463F
:10F82000B34201D30020F0BD587988420DD11D7933
:10F83000A54200D04CB9D879904206D11868077912
:10F84000AF4202D105689D42EDD00C33E8E700BF1E
:10F85000A00100085003000837B5034600790228CC
:10F8600030D11B4A93F91030009214225343194CA3
:10F87000194AE358934227D0A2F57842934225D003
:10F8800002F5806293421DD101F108020DEB0201E5
:10F890001A8811F8085C22F040021204120C14219C
:10F8A0001A8001FB00441A88E16822F0380231F81E
:10F8B00025101204120C0A431A801A8892B242F0E0
:10F8C00040021A8003B030BD0020DDE70120DBE7F5
:10F8D00000010203B000002000300140C36910B5F0
:10F8E000044623B909211420FEF7A0F8E061E0697D
:10F8F00010BD10B504460068FFF7F0FF8378DBB158
:10F90000B0F90A3007EE903AF8EEE77AC4ED057ADE
:10F91000B0F90C3007EE903AF8EEE77AF1EE677A3C
:10F92000C4ED047AB0F90E3007EE903AF8EEE77ABB
:10F930000120C4ED067A10BD1846FCE710B5044658
:10F940000068FFF7CBFF8378CBB1B0F9043007EE46
:10F95000903AF8EEE77AC4ED047AB0F9063007EE93
:10F96000903AF8EEE77AC4ED057AB0F9083007EE80
:10F97000903AF8EEE77A0120C4ED067A10BD1846F9
:10F98000FCE710B504460068FFF7A8FF8378CBB109
:10F990008388DBBA07EE903AF8EEE77AC4ED047A92
:10F9A000C388DBBA07EE903AF8EEE77AC4ED057A41
:10F9B0000389DBBA07EE903AF8EEE77A0120C4ED4E
:10F9C000067A10BD1846FCE710B500680C46FFF734
:10F9D00085FF0346807840B15B892222DBBA93FB26
:10F9E000F2F303F26D132380012010BD38B50068D7
:10F9F0000D461446FFF772FFD0F8013007EE103ABB
:10FA0000CDB1D0F80530DFED176A9FED176A07EE2C
:10FA1000903AF8EE677A77EEE67A77EEA77AC7EE55
:10FA2000866AF7EE007A76EEE77ADFED106A67EE27
:10FA3000E67AC5ED007A9CB1DFED0D7ADFED0D6A57
:10FA4000B8EEC77A27EE277AC7EE267A9FED0A7AB4
:10FA500077EEC77A9FED097A77EE877AC4ED007A60
:10FA600038BD00BF9AC9CC449AC94C460E76D745DA
:10FA70000000484300E0FF440000484233938843BD
:10FA800037B500680D461446FFF728FFD0F805305B
:10FA90009FED237A07EE903AF8EE677AF2EE046A69
:10FAA00077EEC77A9FED1F7AD0F8013067EE877A3C
:10FAB000B3EE097A67EE877A07EE103AF4EEE67A4B
:10FAC000F1EE10FA06DCFAEE046AF4EEE67AF1EEF4
:10FAD00010FA0CD517EE900A49F046FF124ACDE90C
:10FAE000000104210320FDF73FFF03B030BD2DB11D
:10FAF000DFED0E6A67EEA67AC5ED007A002CF4D031
:10FB0000B8EE477ADFED0A6ADFED0A7AE7EE267A89
:10FB10009FED097A77EE877AC4ED007AE5E700BFBA
:10FB20000000004600008038E8B606080AD778438F
:10FB30000319C83D000048C2339388430379022B60
:10FB40000DD190F9103014225343064AD3581A8924
:10FB5000920746BF1889C0F3C010012070470020EB
:10FB6000704700BFB00000200368DB6B13B504468C
:10FB70002BB923685B6B3BB9FF23E38202E0984714
:10FB80000028F6D102B010BD214601A898470028F0
:10FB9000F2D0BDF80630013B9BB2EEE7036810B52A
:10FBA0009B680446984701236374FF23A37410BD28
:10FBB000036810B504461B689847236820469B6875
:10FBC0009847E37C0133E37410BD036810B5044625
:10FBD0005B689847236820469B689847E37C013B15
:10FBE000E37410BD2DE9F3410446184616460D4650
:10FBF0001F4649F04DFD2368E67328440022A07398
:10FC00000092D3F8148032463B4629462046C0472E
:10FC100002B0BDE8F08130B5046885B0E469089DA4
:10FC200034B10DB90DF10F050095A04705B030BDF9
:10FC30002046FBE703685B6A184703689B6A18471E
:10FC400010B5037B04460BB1437B13B92046FFF785
:10FC5000F4FF23682046DB68BDE8104018470368BE
:10FC60005B6C03B11847704738B504468B68016078
:10FC70000D4698470B4B2361002323752B6B13B163
:10FC8000204698472075084B93F8BB311BB1237D64
:10FC900023F0010323750023E3822046BDE83840AA
:10FCA00062E700BF0001FF00C062002003681B681C
:10FCB00003B11847704703685B6803B11847704782
:10FCC00003681B6A03B11847704703685B6A03B196
:10FCD0001847704730B40468029DA46A1CB10295AD
:10FCE000A44630BC604730BC704730B40468029D05
:10FCF000E46A1CB10295A44630BC604730BC704732
:10FD000003685B6C03B11847704703689B6C03B1D1
:10FD10001847704703689B6F03B118477047036823
:10FD2000D3F8803003B1184770470368D3F88430A4
:10FD300003B1184770470368D3F8883003B11847F8
:10FD4000704721B10B68D3F88C3003B118470020FD
:10FD5000704738B5094C052303FB0044A13C00253E
:10FD6000013514F8010FEDB248F009FC052DF7D16B
:10FD7000BDE83840002048F002BC00BF73110608FF
:10FD800010B5441E14F8010F00B910BDFFF7E1FFD4
:10FD9000F8E7FFF729BBFFF727BBFFF725BBFFF706
:10FDA00023BBFFF721BBFFF71FBB30B1036882887D
:10FDB0001B691A4214BF01200020704728B1036854
:10FDC000828809B11A8370475A83704710B103685B
:10FDD00082881A83704710B1036882885A837047FB
:10FDE00073B50C46054600B30668114B06F13F4259
:10FDF00002F57E0203EB922393F8AA0246F04CFA36
:10FE0000AB88009304F003038DF80430C4F381033E
:10FE10008DF805306946C4F30013304664098DF847
:10FE200006308DF80740FAF775FB02B070BD00BFD1
:10FE30006C110608F7B50C4615460746A8B30668C8
:10FE40001B4B06F13F4202F57E0203EB922393F82F
:10FE5000AA0246F021FAB8880090B0FA80F3C3F104
:10FE60001F0303F00702C3F3CC0306EB83039200E6
:10FE7000196A0F27974021EA07011962196A95400C
:10FE80000D431D6204F003038DF80430C4F38103B5
:10FE90008DF805306946C4F30013304664098DF8C7
:10FEA00006308DF80740FAF735FB03B0F0BD00BF10
:10FEB0006C11060838B50409013C032C00F00F0250
:10FEC00019D80E4D05EB4403B3F8B01241FA02F312
:10FED00013F001000ED001239340013B03EA01001F
:10FEE000254450F0F3FE95F8B832034404480C2240
:10FEF00002FB030038BD0020FCE700BF6C110608C0
:10FF00007C6400202DE9F04F85B0B04D0293B04BDA
:10FF10009D4220D26C798C4240F070812C798442D1
:10FF200002D0002840F06A81EC79944240F066816A
:10FF30002C6884B11C220021201D4FF00BFF25608E
:10FF40002B792371AA79A2600192012B2A7AE260AF
:10FF500006D0022B0DD00024204605B0BDE8F08F5E
:10FF6000E87AFFF7A7FF6B7A2374AB7AA06163741A
:10FF7000F2E7E87AFFF79EFF95F90980A06184F81F
:10FF80001080A87AFFF796FF07466061002800F00E
:10FF9000318114238F4E03FB08F3F218F558002D1E
:10FFA00000F02881937C002B40F0CB8092F80890E1
:10FFB000484646F071F909F01F024FEA591901232A
:10FFC000A9F102099340B9F1030F08D8DFE809F05D
:10FFD0007872026C80490A6922EA03030B611423D8
:10FFE00003FB086308F101095879FFF763FF5FFA23
:10FFF00089F9034620B140F60A32C28080F80890A1
:020000040801F1
:10000000142202FB08620393D079FFF753FF039B8E
:10001000824620B140F60A52C28080F8089014222D
:1000200002FB086203939079FFF744FF039B83462A
:1000300020B140F60A42C28080F80890142202FBE8
:10004000086292F80990019A12F0040201924A465D
:100050003CD04A211846FFF7EDFE4A462A21504679
:10006000FFF7E8FE4A460A215846FFF7E3FE14234D
:1000700003FB086393F804A0BAF1000F06D05046C2
:10008000FFF718FF4A460921FFF7D4FE534B9D4264
:1000900023D103F584335A6A42F480525A625A6A71
:1000A00022F480525A6225E04B494A6922EA03034E
:1000B0004B6194E748490A6A22EA03030B628EE720
:1000C00045494A6A22EA03034B6288E70A21184637
:1000D000FFF7B0FE4A460A21C1E7414B9D423ED19F
:1000E00003F500331A6A42F480421A621A6A22F453
:1000F00080421A62019B002B65D1012202212B88CC
:100100000A4303F44153134343F445732B80AB8BF1
:1001100023F400631B041B0CAB8307232B822B8867
:100120009BB243F040032B80BAF1000F04D050463D
:10013000FFF7C0FEFFF74AFE142303FB0866012306
:10014000B374029BBB710E23FB71002338463B72D4
:100150000921FFF745FE3846FFF738FEFCE6214B44
:100160009D4209D103F5FE331A6A42F400421A6235
:100170001A6A22F40042BCE71B4B9D4209D103F5E9
:1001800082335A6A42F400525A625A6A22F4005286
:1001900088E7164B9D4209D103F568435A6A42F439
:1001A00080125A625A6A22F480127BE7104B9D42F9
:1001B000A0D103F564435A6A42F400125A625A6AA3
:1001C00022F400126EE70022114698E7A001000811
:1001D00050030008B0000020003802400030014009
:1001E00000380040003C0040003401400050014015
:1001F000005401402046FFF702FBACE60C3587E6D1
:10020000074B03EB8003D3F8BC323BB19A881B68E1
:1002100059690A4201D05A8370471A83704700BF58
:100220006C110608034B03EB800081F00101D0F84C
:10023000BC02C3E56C1106080A4B10B5D3F808449C
:1002400024B1094A03212046F9F704FD2046002184
:10025000F9F756FD20460549BDE8104040F62B420F
:1002600045F052BFC0620020009F240028A6002055
:1002700038B5104CD4F8085425B10F4A64212846EB
:10028000F9F7E8FC00212846F9F73AFD6B681A688F
:10029000B2F844306FEA43436FEA53439BB2A2F88B
:1002A000443013889BB243F001031380012384F888
:1002B0000C3438BDC0620020009F2400DFF8B0C1BC
:1002C0002DE9F84F9CF80CE4BEF1000F40F0CC8013
:1002D000DCF8089499F81030002B40F0C5809CF8A9
:1002E00010349CF811249CF81254ACF80EE40CF273
:1002F0001440F0463C268178C778C1F1FF0189B2ED
:10030000002900F0AD80C1F1FF0179430488B4FBFE
:10031000F6FA0912BAF1050F20D8DFE80AF0030D4A
:10032000647283917A1A6243B2FBF6F252FA81F256
:10033000CDB2D2B23B460FE0B4FBF6F306FB13435B
:100340009BB2C3F13C037A1A5343B3FBF6F353FA5F
:1003500081F3CDB2DBB23A464FF0010E1F0247EAFD
:10036000024747EA050B00210127C1F1170A07FAE6
:100370000AFA08EB01041AEA0B0F04F12A0408BF79
:10038000BA46A4B2394F01F1010118BF4FF0020A79
:10039000182947F824A0E7D108F118081FFA88F8AF
:1003A000B8F5406F00F10400A5D18021ACF8141617
:1003B000BEF1000F05D08CF812548CF811248CF883
:1003C00010344FF44063ACF80E349CF81636002B12
:1003D0004AD0484640F62B41F9F7B6FD4846BDE8FD
:1003E000F84FF9F7E3BDB4FBF6F206FB12427D1AB3
:1003F00092B25543B5FBF6F555FA81F5CBB2EDB2A5
:10040000A9E7B4FBF6F206FB124292B2C2F13C023B
:100410007C1A6243B2FBF6F252FA81F2CBB2D2B24C
:100420003D4699E7B4FBF6F506FB15447B1AA4B2EA
:100430006343B3FBF6F353FA81F3CAB2DBB2EFE7DF
:10044000B4FBF6F306FB13439BB27C1AC3F13C03E7
:10045000CAB26343B3FBF6F353FA81F1CDB269E755
:100460003D463A463B4677E7BDE8F88F28A6002090
:10047000C0620020F8B5134BD3F80844054604B316
:1004800093F80C14C9B9E06866688268136823F0B1
:1004900001031360326877790B4E938936F8176041
:1004A0009BB223EA06039381217413889BB243F025
:1004B000010313800177FFF7DBFE2046F9F716FDF5
:1004C0000560F8BDC0620020B00F060838B5104CBA
:1004D000D4F8080450B194F80C343BB194F81736B2
:1004E000032B04D1F9F702FD6423036038BD022B0E
:1004F0004FF0000503D1F9F7F9FC0560F6E784F841
:100500000C54FFF799FE0028F0D184F81606EDE7A9
:10051000C06200200346806B9B7903F0010399427F
:1005200000D053E457E410B5837913F0010F03F0C2
:1005300020020446C36B13D05B68002A1A7A08BFF6
:100540004221606B18BF0221FFF774FC012184F87F
:100550006012A4F85C12E06BBDE81040F9F7DCBC57
:100560005B68002A08BF22211A7AEAE7036C806BD5
:100570001BB15B6801211A7A5CE4012130E42DE9AA
:10058000F04183681C686679B1072FD594F86152F1
:10059000C5B194F962528DB1B4F864124B08A4F855
:1005A0006432204601F00101FFF7B4FFA379013D59
:1005B0006DB2580684F8625218D5BDB9002384F88C
:1005C000613213E0A36A626A94F860129A4225D1FC
:1005D00061B9A3791A0709D5236CA06BD3B15B6805
:1005E0001A7AFFF727FC2046FFF79DFFF10740F13D
:1005F000818094F85C32002B7CD194F85D32013319
:10060000DBB2092B84F85D3235D12046BDE8F041DC
:10061000FEF760BC1946FFF7E3FBE4E75A1CA0694C
:10062000A262C35C2069A7795B0043F40073A4F85D
:1006300064320A23824228BF002284F862320123F6
:10064000A26284F8613299B13B0711D5D4F83C809D
:1006500029464046F9F760FCD8F80430606B1A7AF6
:100660002946FFF7E7FB84F860522046FFF77EFF3C
:100670007D068ED4BAE70A2B3CD194F85F322BB9B1
:10068000B4F8663243F00103A4F86632B4F86602A7
:10069000820501D4C3071AD4B4F86A320133A4F82E
:1006A0006A3294F85F5201239D42A4F85C3221D152
:1006B000A179E06B002384F85F3201F0010145F07D
:1006C0006FFCE06B2946BDE8F041F9F725BCE36A11
:1006D000C0F3470013B1216B9847E2E7E369626911
:1006E000D054E369E2680133B3FBF2F102FB11334A
:1006F000E361D6E7BDE8F081F8B51E4B46681A689D
:1007000004461346B3FBF1F0B0F5803F2ED281B220
:100710002046F9F79FFA23681F687C7974B165B2A7
:1007200003212846F9F782FA002D07DB6109124AF6
:1007300004F01F040123A34042F82130BC7974B1B6
:1007400065B203212846F9F771FA002D07DB61092C
:10075000094A04F01F040123A34042F82130326803
:1007600013889BB243F001031380F8BD012BCBD952
:100770005B08C7E70001002000E100E08160C06B7A
:10078000BAE7002ABCBF80185242002BBCBFC91870
:100790005B420028BCBF121A0020F0B58418002963
:1007A000A4F11D04BCBF5B180021002CC8BF121BA4
:1007B000CC180F3C002CC8BF1B1B0B4E02440B4433
:1007C0003C274FF0200C90420CDC06EB40050C4619
:1007D00004E007FB04FE013425F80EC09C42F8DD5E
:1007E0000130F0E7F0BD00BFD868002008B5114B1C
:1007F0001A6C42F080521A640F4A012111620F4AAA
:10080000FF215162CA215162532151625B6FDB00AB
:1008100009D400210120FAF7BDFBBDE808400849D2
:100820000020FAF7B7BB0020FAF7C4FB044B98424C
:10083000EFD108BD0038024000000E420028004001
:1008400076614E6938B50C4605461946046014B108
:100850002046F9F7FFF9BDF810102046F9F750FAD5
:1008600063681A68B2F844306FEA43436FEA53434F
:100870009BB2A2F8443013889BB243F0010313806B
:100880002046F9F733FB0023A860036038BD2DE94B
:10089000F04F85B007469DF83CB003928A469946D2
:1008A000FDF7FEF8064648B1224B93F8D819072900
:1008B00009D9214A00210420FDF756F800252846D1
:1008C00005B0BDE8F08F4A1C5C205FFA82F883F81F
:1008D000D88903F6DC1500FB013301FB005500212C
:1008E000C3F8DC1983F8E0193879FFF7E3FA044616
:1008F00028B1022380F806A0C37180F80880BBF1FC
:10090000000F0ED03A7A02212046FFF793FABDF885
:1009100038300093039A4B4631462846FFF792FF42
:10092000CDE720461121FFF75BFA2046FFF753FA87
:10093000EDE700BFC06200200AB7060830B51E4BC5
:100940002DED028B1C68B4FBF1F303F57F4383B0FC
:10095000FF331B0CB4FBF3F40023B4FBF1F501925D
:1009600000932246ABB20221F0EE408AB0EE608ADC
:10097000FFF78DFFE0B107EE904AB5EE408AF1EE49
:1009800010FAF8EE677A0ABF07EE105A68EE270AE7
:10099000F8EE470A9FED097AC0EE876A01230371DA
:1009A00027EE667AC0ED046AA8EEA77A80ED037A96
:1009B00003B0BDEC028B30BD0001002000007A4482
:1009C0000023064910B51C46984200DC10BD51F8C2
:1009D00033200AB1926814600133F5E7283F002004
:1009E00013B50F4C8DF80700D4E90423A1685343D5
:1009F0008B4212D06368E0680DF1070118444EF095
:100A000087F8636822691344A268B3FBF2F102FB22
:100A10001133636063690133636102B010BD00BFCD
:100A2000003F00200F4B1B78062B14D8DFE803F0A3
:100A3000041316070A0D10004FF4C87070470A4BD4
:100A4000988870474FF47A6070474FF4FA507047B7
:100A50004FF47A5070474FF47A7070474FF4FA6051
:100A6000704700BFDC3E0020684000202DE9F04FB9
:100A70002DED028BAB4BAC4C1B78AC4FDFF80083F9
:100A800097B0002503932646AB46A246D6F80090C1
:100A9000002257F83210894568D1D2B2424492F808
:100AA000BC2C012A67D0022A6ED03046FEF78EFD9C
:100AB00070B9142202FB0BA2D16801F00C02042AC7
:100AC00006D14846FEF7A0FA0135EDB20544EDB275
:100AD0000BF1010BBBF10A0F06F11406D6D1944EAF
:100AE000A6F1C8073846FEF771FDA8B9F9684B07AB
:100AF00012D501F00C03042B0ED0039B9D424BD268
:100B000021F0080141F004013868F960FEF77CFA31
:100B10000135EDB20544EDB21437B742E2D14FF0E2
:100B200000094D464E464F464FF0080B2046FEF753
:100B30004DFD002837D07F4A3B4601210420FCF7B9
:100B400013FF01370A2F04F11404EFD1754B1E78FF
:100B50000C2E70DD012388F8CA3C774A0C230093E1
:100B6000334600210420FCF7FFFE8AE001320E2A02
:100B70008FD1FF2292E7F268100796D522F0080283
:100B800042F00402F26090E7F26851078DD522F03E
:100B9000040242F00802F5E721F004013868F96028
:100BA000FEF732FAB8E7E16848070AD5039BB3427B
:100BB00007D921F008012068E160FEF725FA013627
:100BC000F6B2E26811071AD5206805A900239D42F4
:100BD0000DDC16AB03EB8902C4F80CB009F1010A75
:100BE000082142F8204CD146FEF70EFAA9E751F849
:100BF00004CFDCF800C0604501D00133E7E75307BC
:100C00009FD520680DAA00234B450DDB0423E3602C
:100C100016AB05F1010A03EB8505042145F8404CAC
:100C2000FEF7F2F955468CE752F8041F096888422E
:100C300087D00133E8E7414B9979414B032919707B
:100C400033D90B1F022B32D8FFF7ECFE3D4A3E4B47
:100C500080B2B3FBF0F31360002353603B4B4FF0C3
:100C6000000A4FF0000BC3E900AB394BC8F8CC3C8D
:100C7000384B13F81130E3B9374A02210420FCF74E
:100C800073FE98F8D03C002B40F0CD80334A02210F
:100C90000420FCF769FE98F8CA0CB0FA80F040090D
:100CA00017B0BDEC028BBDE8F08F2D4BDEE72D4B6E
:100CB000DCE7AE4218DC2C4F9FED2C8A0DF1140BB3
:100CC0000024A642DDDD2A4B5BF8045F5B68C3F3BA
:100CD000007A1B4B1B78062B00F2A180DFE803F0A3
:100CE000961B560B5F5F5F00032388F8CA3C214ABE
:100CF0000095334635E7FFF795FEDFED1F0A014605
:100D00005246B0EE600A2846FFF718FE47F8340056
:100D1000002879D159E0FFF785FEDFED180A01467A
:100D20005246EEE7105701209C05002018100608D7
:100D30006406002045B706085DB706086840002035
:100D4000DC3E0020E83E002040420F00F03E002044
:100D50005DF000083011060889B7060805B80608D6
:100D600081F300085BF00008283F00206F12833AEF
:100D700014570120A7B70608000000006F120339BE
:100D8000C0620020ACC5A737ACC5A736FFF74AFE46
:100D90005FED040A1FED040A01465246B3E7052B36
:100DA0001DD0524A5249062B18BF0A46CDF804A05E
:100DB0004FF0000A2846CDF800A014230221FFF7C7
:100DC00066FD054668B947F83400052388F8CA3C33
:100DD000484A234600210420FCF7C6FD51E7464A55
:100DE000E4E700F11403194600680393122245F06A
:100DF0008BF9039B30B11846482251464EF0AAFFAA
:100E000001232B7147F8345001345AE7FFF70AFEEB
:100E10009FED3A0A01465246F0EE480A73E7002376
:100E200047F83430D1E798F8D15C98F8D23C0135D6
:100E3000ED1A102D0BDD022388F8CA3C304A10232E
:100E4000009300212B460420FCF78EFD23E798F841
:100E5000DC3C012B2ED0022B30D02A4B98F8DC1C26
:100E6000C8F8E03C11F0FD012CD14D452CDC264F9B
:100E7000DFF898A0DFF8AC900DAE0C46AC42BFF6A0
:100E80000AAFD9F80420B8F8D63CBAFBF3F3C2F3A2
:100E900000720192B8F8D42C009203211B4A56F834
:100EA000040F9BB2FFF7F3FC0146A8B147F8040B0F
:100EB0000134E3E746F0E4FF154BCFE746F0E0FFEF
:100EC000144BCBE7144AE2E6042088F8CA0C134A14
:100ED000CDF800902B46B7E7052388F8CA3C104AA6
:100EE00023460420FCF740FDD5E600BF001BB700F9
:100EF000C0C62D00E0B70608808D5B006F12833AF4
:100F00001FB8060835F000086063002040420F005B
:100F100011EB02084DF000084BB8060887B8060828
:100F2000BDB8060814570120034AD2F8E02C12B1CC
:100F30000F2800D810477047C062002040B1013828
:100F40000023FF2803F1010203D840EA032080B206
:100F5000704740081346F4E703681B6818470368A6
:100F60005B68184703689B6818470368DB6970B5BE
:100F700006460C46154683B1BDE87040184730461A
:100F8000FFF7F0FF0028FAD014F8011B3046FFF7F6
:100F9000E3FF2B1B002BF2DC70BD0D44F9E7E4E707
:100FA0000368DB68184703681B69184703685B69B7
:100FB000184703689B6A03B1184770470368DB6AE8
:100FC00003B118477047154B1B6813F0100F01460B
:100FD000134B06D0B3F8E42C12F0040F0CBF0146FB
:100FE000002193F8FE2C72B1D3F8002DA2B19268C3
:100FF00039B1B3F8041D0B4BB3FBF1F35B10136075
:10100000704711607047D3F8080D93F80C3D0BB989
:1010100081F00101FEF7D2BE704700BF7856012073
:10102000C062002040420F00BFF34F8F0549064BBE
:10103000CA6802F4E0621343CB60BFF34F8F00BF76
:10104000FDE700BF00ED00E00400FA0508B572B648
:1010500000224FF0FF31930003F1604303F5614339
:101060000132082AC3F88010C3F88011F3D1FFF7CA
:10107000DBFF012108B50846F9F78CFFFFF7E6FF13
:1010800008B50120F9F796FF012809D10021F9F7E9
:1010900081FF044B1A6882F308885B689847FEE773
:1010A00008BD00BF0000FF1FEFF31183102282F381
:1010B000128809490A6801320A604FF0E0220749A4
:1010C0009069C1F8100D0020C1F8140D1269DBB24F
:1010D00083F31188704700BF542B0020C0620020AA
:1010E000074A084B5168D3F8183D58434FF47A73B8
:1010F000B0FBF3F053685B1A8342FBD9704700BF23
:10110000001000E0C062002010B504464FF4FA70F1
:10111000FFF7E6FF6069BDE81040FEF757BE90F9A3
:1011200010302DE9F0411646142253430D4A52F86F
:101130000380836813F0020504460F4602D140691C
:1011400047F0F0FB3946404648F0CAF93146404680
:1011500048F0C6F915B92046FFF7D6FF0120BDE8D3
:10116000F08100BFB00000207FB50379012B0D4650
:101170000AD0022B19D18368DB0758BF01F07F0129
:1011800004B0BDE87040CAE781688DF80F2001F017
:1011900001010DF10F0200920191417C90F91000C4
:1011A0002A46F9F7ABFE04B070BD0020FBE70068EB
:1011B0002E22F421D8E7044B00681A8C92013432B5
:1011C00002F0FC02F421CFE7C062002008B5312212
:1011D000F4210068FFF7C8FF012008BD0068012264
:1011E0005821C1E7006801224821BDE700680222BA
:1011F0000821B9E7006801220821B5E710B50446C7
:10120000002221210068FFF7AFFF2068FC22202187
:10121000FFF7AAFF206840222421FFF7A5FF2068DE
:101220000C222321FFF7A0FF206800222221FFF7D4
:101230009BFF012010BD10B5012204460B21006860
:10124000FFF792FF20B120681D220921FFF78CFFD4
:1012500000F0010010BD044B0246D3F81C0D08B18C
:10126000802181E7704700BFC062002010B5B02028
:10127000FFF7F1FF4020FFF7EEFF0020FFF7EBFF45
:101280001020FFF7E8FF4FF48064013C0020A4B277
:1012900047F075F9002CF8D110BD10B50446A1F146
:1012A0005000C0B2FFF7D7FF04EB4400400004EB4E
:1012B000440400F00E00FFF7CEFFC4F3C30010306B
:1012C000BDE81040C7E708B55038C0B2FFF7C3FF0C
:1012D0000020FFF7C0FFBDE808401020BBE738B58D
:1012E00000221F2334210120FEF70CFE3C4BC3F8E3
:1012F0001C0D10B90024204638BDAE20FFF7ABFF0F
:1013000004460028F6D0D420FFF7A5FF8020FFF781
:10131000A2FFA820FFF79FFF3F20FFF79CFFD320ED
:10132000FFF799FF0020FFF796FF4020FFF793FF9C
:101330008D20FFF790FF1420FFF78DFFA120FFF70E
:101340008AFFC820FFF787FFDA20FFF784FF12200B
:10135000FFF781FF8120FFF77EFFCF20FFF77BFFA4
:10136000D920FFF778FFF120FFF775FFDB20FFF7AB
:1013700072FF4020FFF76FFFA420FFF76CFFA6204D
:10138000FFF769FFAF20FFF766FFA620FFF763FFB7
:10139000AE20FFF760FF2020FFF75DFF0020FFF782
:1013A0005AFFB020FFF757FF4020FFF754FF0020FF
:1013B000FFF751FF1020FFF74EFF4FF48065013D0E
:1013C0000020ADB247F0DBF8002DF8D18120FFF707
:1013D00042FFC820FFF73FFFAF20FFF73CFF8AE73F
:1013E000C062002008B5FFF7BFFE014B187008BDB2
:1013F000601000202DE9F0411E4690F9103015468E
:10140000142253430E4A52F8038083689A07044615
:101410000F4602D4406947F085FA3946404648F005
:101420005FF833462A460021404648F009F8A36891
:101430009B0702D42046FFF767FE0120BDE8F0813C
:10144000B0000020F7B50779012F16460AD0022F09
:1014500015D18468E40758BF41F0800103B0BDE8AE
:10146000F040C7E7826802F00102CDE900620A4657
:10147000417C90F91000F9F741FD03B0F0BD002068
:10148000FBE707B552BAADF80420022301AAFFF723
:10149000D9FF024B187003B05DF804FB6010002008
:1014A00010B50A4C002384F8203D84F8211D84F8EF
:1014B000222D032304F55262FF21FFF7C3FF00280A
:1014C0000CBF6FF00C00002010BD00BFC0620020F8
:1014D00010B50B4C002384F8203D130A84F8211D1D
:1014E00084F8223D84F8232D042304F55262FF2161
:1014F000FFF7A8FF00280CBF6FF00C00002010BD04
:10150000C0620020024A0068002351219AE700BF10
:10151000E07000202DE9F0411E4690F9103015468C
:10152000142253430E4A52F8038083689A070446F4
:101530000F4602D4406947F0F5F93946404647F076
:10154000CFFF334600222946404647F079FFA36883
:101550009B0702D42046FFF7D7FD0120BDE8F081AC
:10156000B0000020F7B50779012F16460AD0022FE8
:1015700015D18468E40758BF41F0800103B0BDE88D
:10158000F040C7E7826802F00102CDE900620A4636
:10159000417C90F91000F9F7D7FC03B0F0BD0020B2
:1015A000FBE713B5062304466A4600680221FFF7ED
:1015B000D9FFB8B1BDF9003007EE903ABDF902305D
:1015C000F8EEE77AC4ED077A07EE903ABDF90430F9
:1015D000F8EEE77AC4ED087A07EE903AF8EEE77A8B
:1015E000C4ED097A02B010BD13B5022304466A4661
:1015F00000680321FFF7B6FF10B9002002B010BD4C
:101600009DF90130002BF8DA206807236A46122181
:10161000FFF7A8FF0028F0D09DF902209DF80130C7
:1016200043EA022313EB430348BF03339B1007EE47
:10163000903A9DF904209DF8033043EA022313EB0E
:101640004303F8EEE77A48BF03339B109DF9062069
:10165000C4ED047A07EE903A9DF8053043EA022380
:1016600013EB4303F8EEE77A48BF03339B10C4ED56
:10167000057A07EE903AF8EEE77AC4ED067ABDE710
:1016800038B504460068FEF729F90C230546021D0B
:1016900019462068FFF766FFA870B8B1B5F90430A5
:1016A00007EE903AF8EEE77AC4ED077AB5F906301E
:1016B00007EE903AF8EEE77AC4ED087AB5F908300B
:1016C00007EE903AF8EEE77AC4ED097A38BD38B5FE
:1016D00004460068FEF702F90D230546C21C0C21E2
:1016E0002068FFF73FFFA870B8B1B5F90A3007EEE0
:1016F000903AF8EEE77AC4ED077AB5F90C3007EEC8
:10170000903AF8EEE77AC4ED087AB5F90E3007EEB4
:10171000903AF8EEE77AC4ED097A38BD13B50323A1
:101720000C46006801AA2221FFF71CFF30B1BDF969
:10173000053003EB83031B12E633238002B010BD98
:1017400013B5062304466A4600681F21FFF70AFF07
:10175000D0B1BDF80030DBBA07EE903ABDF80230E8
:10176000F8EEE77ADBBAC4ED047A07EE903ABDF8FA
:101770000430F8EEE77ADBBAC4ED057A07EE903A6A
:10178000F8EEE77AC4ED067A02B010BD13B5062371
:1017900004466A4600682521FFF7E4FED0B1BDF893
:1017A0000030DBBA07EE903ABDF80230F8EEE77A87
:1017B000DBBAC4ED077A07EE903ABDF80430F8EED4
:1017C000E77ADBBAC4ED087A07EE903AF8EEE77AEA
:1017D000C4ED097A02B010BD70B506680546304602
:1017E000FEF77CF80E230446021D3B213046FFF72E
:1017F000B9FEA070B8B1A389DBBA07EE903AF8EE53
:10180000E77AC5ED077AE389DBBA07EE903AF8EE9E
:10181000E77AC5ED087A238ADBBA07EE903AF8EE4C
:10182000E77AC5ED097A70BD07B50223006801AA01
:10183000F621FFF797FE20B1BDF80430024A5BBAEB
:10184000138003B05DF804FBC062002007B50323DA
:10185000006801AAF621FFF785FE80B19DF80530EA
:101860009DF8042007491B0243EA02439DF8062025
:101870001343B1F92020C2F10802D3404B6203B0F8
:101880005DF804FBC062002013B5062300686A46B9
:10189000F721FFF767FE134BE8B19DF801109DF8A3
:1018A00000209DF80340090141EA02319DF8022021
:1018B00041EA12119DF804209964120142EA0432AF
:1018C0009DF80540C3F8201E42EA14129A62C3F83C
:1018D000242E02B010BDD3F8202E9A64D3F8242E03
:1018E0009A62F6E7C062002007B50323006801AAE8
:1018F0001946FFF737FEA0B19DF804309DF805109A
:101900009DF904201B0443EA01239DF80610002AD8
:10191000ACBF00224FF07F420B431343024AC2F890
:10192000F03003B05DF804FBC062002007B503236C
:10193000006801AA0021FFF715FEA0B19DF8043050
:101940009DF805109DF904201B0443EA01239DF82E
:101950000610002AACBF00224FF07F420B43134316
:10196000024AC2F8EC3003B05DF804FBC06200200C
:1019700013B5044600680379022B0CBF43210321F1
:1019800006236A46FFF7EEFD18B9E086A06302B0B1
:1019900010BDBDF800305BBAE386BDF802305BBA1B
:1019A0006387BDF804305BBA2387F0E713B50023E3
:1019B000C38683630446062300686A460321FFF753
:1019C000D1FD78B1BDF8003003EB4303E386BDF9E8
:1019D00002305B4203EB43032387BDF8043003EB83
:1019E0004303638702B010BD07B5012301AAFF219D
:1019F0000068FFF7B7FD03B05DF804FBF7B50546D7
:101A00000068FDF76BFF00230370042304460DEB11
:101A100003022868FF21FFF7A5FD10B9002003B0DD
:101A2000F0BD286804236A46FF21FFF79BFD0028CC
:101A3000F4D09DF804309B09023B012BEED9BDF890
:101A40000420BDF80630BDF80050BDF8021052BAAF
:101A500043F6FF77C2F30D02BA42DFD0002ADDD091
:101A60005BBAC3F34A1340F2FF76B342D6D0002BE1
:101A7000D4D06DBAC5F30D05BD42CFD0002DCDD069
:101A800049BAC1F34A11B142C8D00029C6D0561B89
:101A9000002EB8BF7642FF2EC0DC5E1A002EB8BF03
:101AA0007642FF2EBADC01262A440B4432413341F0
:101AB0002670C4F80520C4F80130B0E737B50546F4
:101AC0000068FDF70BFF00230370042304460DEBB1
:101AD00003022868FF21FFF745FD40B19DF804305F
:101AE0009B0907D00B4A04210320FBF73DFF002090
:101AF00003B030BDBDF80420BDF8063052BA5BBA61
:101B000092B2C3F34A1301212170C4F80520C4F82E
:101B10000130EDE7E2B8060807B5022301AAFFF796
:101B200021FD044B1870BDF8040040BA80B203B028
:101B30005DF804FB6010002038B515460C4A0B0A0E
:101B400082F8203D82F8211D022302F55262FF2116
:101B50000446FFF777FC30B101232A46FF212046D7
:101B6000FFF700FD10B96FF00C0038BD0020FCE756
:101B7000C06200202DE9F041104D05F5526816466F
:101B8000002485F8211D02234246FF21074685F8DF
:101B9000204DFFF757FC18B96FF00C00BDE8F0813D
:101BA00002234246FF213846FFF7DCFC0028F3D031
:101BB000B5F8203D5BBA33802046EFE7C0620020D5
:101BC0002DE9F341734D0468DFF8D4810023064604
:101BD00085F8E2302D27B9B218F8012B20460137DD
:101BE000FFF75EFC882FF6D1402287212046FFF7C1
:101BF00057FC00238DF806309DF80630002B6DD081
:101C0000012286212046FFF74BFC00228721204637
:101C1000FFF746FC092208212046FFF741FC00227D
:101C20000B212046FFF73CFC00284FD137680DF10F
:101C300006025E213846FFF79DFFBDF80630B3F57A
:101C4000D77F00F0A38057D8512B00F09D804BD850
:101C50001D2B6ED01E2B00F097803068212146F09E
:101C600061FB34680DF10602DE212046FFF782FF9A
:101C7000BDF806309FED487A2822C3F30903534389
:101C800007EE903AF8EEE77A002267EE877A85F859
:101C9000202DFCEEE77A6C2217EE903A85F8212D84
:101CA0001A0E85F8222D1A0C85F8232D1A0A85F8AC
:101CB000242D85F8253D394AFF2106232046FFF7CC
:101CC000C1FB306840228721FFF7EAFBB0FA80F0C1
:101CD000400985F8E20002B0BDE8F0810DF106018F
:101CE000204646F0B0FB87E7AD2B4FD0D62B01D076
:101CF000602BB2D121241DE040F2E132934247D063
:101D00000CD840F2D922934242D040F2E1229342D1
:101D100002D0B3F5E67FA0D164240BE040F28F42FD
:101D2000934203D040F29152934296D14FF4FA7409
:101D300000E00F24002890D10A224B213846FFF7FB
:101D4000AFFB0F2260213846FFF7AAFB0D2263216B
:101D50003846FFF7A5FBB82269213846FFF7A0FBFC
:101D600040F60D7278213846FFF7B2FB40F60E625E
:101D70007A213846FFF7ACFB00287FF46EAF21468E
:101D8000384646F0CFFA68E71424D3E73224D1E787
:101D9000C824CFE7C06200209A99893FE06F0020F5
:101DA0003414060837B5134D95F8E2300446FBB1FC
:101DB00000680DF1050146F046FB9DF805307BB14A
:101DC0000DF1060220689621FFF7D4FE0A22BDF825
:101DD0000630B3FBF2F3084A9360012385F8E33041
:101DE00020680122862103B0BDE83040FFF758BBD0
:101DF00003B030BDC06200206010002013B5022384
:101E000001AA044651210068FFF7ACFB114AF0B16A
:101E1000BDF804305BBA9BB2D360D368B3F5C87F1A
:101E200002DD4FF0FF33D3600B4B0C4A1968D2F838
:101E3000283E32338B4208D2C2F8281E2068002385
:101E400002F562625121FFF7FDFA02B010BD6FF09A
:101E50000103E8E760100020542B0020C06200203E
:101E600007B50223006801AA0021FFF77BFB0F4B97
:101E700083F8E800B0B1BDF804300D4A5BBA9BB2FC
:101E8000B3F5FA6F3FBF0A21B3FBF1F307EE903AC7
:101E9000F8EEE77A2BBF4FF0FF33FDEEE77A1361E0
:101EA000C2ED047A03B05DF804FB00BFC0620020FD
:101EB0006010002013B502230C46006801AA00211F
:101EC000FFF750FB60B15CB19DF805309DF904202F
:101ED000DB0903EB830302EB820203EB4203238063
:101EE00002B010BDF8B590F91030154614225343D6
:101EF0000D4AD75883689A0704460E4602D44069B3
:101F000046F010FD3146384647F0EAFA0123002238
:101F10002946384647F094FAA3689B0702D4204626
:101F2000FFF7F2F80120F8BDB000002073B5037987
:101F3000012B16460AD0022B15D18368DB0758BF48
:101F400041F0800102B0BDE87040CBE7826802F04A
:101F50000102CDE900620A46417C90F91000F8F7D1
:101F6000F3FF02B070BD0020FBE713B504466A46DC
:101F700000680821FFF7DAFF9DF80030DB0602D485
:101F8000002002B010BD206806236A460021FFF73A
:101F9000E9FA0028F4D09DF801309DF800209DF862
:101FA00004109FED387A1B0203EB02439DF80220D8
:101FB0001C021A449DF8033048BF02F17F42090217
:101FC00001EB034107EE902A9DF80530F8EEE77A21
:101FD0000B44090248BF03F17F43C7EE876A07EE4F
:101FE000903A294BF8EEE77AB3F9582087EE875AF2
:101FF00004EE102A93ED157AB3F95A20D3ED147A32
:10200000B8EEC76A07EE102AB3F95E2004EE902AF4
:10201000B3F9602003EE902AB3F95C2005EE902A14
:10202000F8EEE33AF8EEE55AF8EEE77AE6EEA35A70
:10203000B3F94C20B8EEC44AA5EEA66AB8EEC77A4A
:10204000E6EE267AF8EEE44AE5EE047AA6EEA47A05
:1020500026EE856AF6EE006AE6EE077A07EE102AAB
:10206000B3F94E20C3ED197A07EE902AF8EEE77A1D
:10207000B8EEC77A67EE857AE7EE267AC3ED1A7A6C
:102080007FE700BF00007848C06200202DE9F341DF
:1020900016460DF107021D4607468846FFF746FF24
:1020A0009DF8074006EA0403AB4209D024EA060281
:1020B0002A434146384602B0BDE8F041FFF754B824
:1020C00002B0BDE8F0811FB50446002300688DF81A
:1020D00007300DF107022721FFF728FF60B19DF8B7
:1020E00007301B0708D52068062302AA2821FFF71E
:1020F00039FA20B9E086A063002004B010BDBDF914
:102100000830002BB8BF03339B10E386BDF90A30BB
:10211000002BB8BF03339B102387BDF90C30002B75
:10212000B8BF03339B106387E7E71FB50021044660
:10213000C18681630DF107020068FFF7F7FE10B951
:10214000002004B010BD9DF807301B07F8D52068AB
:10215000062302AA0121FFF705FA0028F0D0BDF8F6
:1021600008305BBAE386BDF80A305BBA2387BDF856
:102170000C305BBA5B426387E3E730B5002585B07E
:102180000446C58685630DF1070200680621FFF746
:10219000CDFE10B9002005B030BD9DF807305B07BB
:1021A000F8D52068062302AA2946FFF7DBF90028A4
:1021B000F0D0BDF80830E386BDF80A302387BDF8BB
:1021C0000C306387E7E707B50DF10702FFF7AEFEB6
:1021D000034B18709DF8070003B05DF804FB00BFC7
:1021E00060100020F8B5144E144F41F00102002198
:1021F0000446FFF7F7F83568C7F82C5E1321204630
:10220000FFF7E1FF10F007000BD001220B21204661
:10221000FFF7E8F8002220461146FFF7E3F8012017
:1022200008E0D7F8302E002AE8D033689BB25B1B59
:102230009A42E3D2F8BD00BF542B0020C0620020B8
:1022400010B50C460121FFF7BEFFC0F30013237049
:10225000C0F3C003A370C0F380036370C0F38013A6
:10226000C0F3C010E370207110BD2DE9F8430F4694
:10227000502114460546FFF7A6FF01304000C0B2CA
:10228000208046212846FFF79EFF2C4E2378013000
:1022900080B273434FF47A78A08003F5FA734FF459
:1022A000FA69B3FBF8F25121B3FBF9F300FB0233F7
:1022B0002846B3FBF8F3E360FFF72EFCC2B2C0F38D
:1022C0000F2023788240013292B27343E28003F5FB
:1022D000FA732846B3FBF8F1B3FBF9F302FB0133C1
:1022E0007021B3FBF8F32382FFF76DFF013040004C
:1022F000C0B2608071212846FFF70EFCC3B2C0F364
:102300000F2083400133FA789BB2238112B1E28817
:102310009B1A2381A3782089734303F5FA734FF442
:102320007A724FF4FA65B3FBF2F1B3FBF5F300FBFD
:102330000133B3FBF2F36382BDE8F883002F3A0068
:102340002DE9F043DB4FDFF874834FF4FA738BB061
:102350000446002689210068C7F8303E87F8E0600F
:10236000FFF731FF40F00102D2B220688921FFF768
:1023700039F8324620688821FFF734F820680122B6
:102380008021FFF72FF820680122FF21FFF72AF8AC
:10239000324631462068FFF725F891212068FFF783
:1023A00012FF314687F8340E01222068FFF71AF831
:1023B00032462068FF21FFF715F832462068802159
:1023C000FFF710F860212068FFF7FDFE40F01202D1
:1023D000D2B220686021FFF705F82068202244214E
:1023E000FFF74FF82068FF220121FEF7FBFF256869
:1023F000012280212846FEF7F5FF0122FF21284611
:10240000FEF7F0FF324631462846FEF7EBFF062284
:10241000FF212846FEF7E6FF83212846FFF7D3FE7B
:1024200040F00402D2B283212846FEF7DBFF0722E8
:10243000FF212846FEF7D6FF012281212846FEF71C
:10244000D1FF012280212846FEF7CCFF6B22942188
:102450002846FEF7C7FF324683212846FEF7C2FF13
:10246000D8F80060C7F82C6E83212846FFF7ABFE32
:10247000002800F04483012228468321FEF7B2FFA2
:1024800092212846FFF79FFE0022C0F3C716804620
:1024900081212846FEF7A6FF06222846FF21FEF7E7
:1024A000A1FF83212846FFF78EFE832100F0FB0267
:1024B0002846FEF797FF28460122FF21FEF792FFEC
:1024C000284601220021FEF78DFF28460022FF2129
:1024D000FEF788FF284600228021FEF783FF0623AF
:1024E00003AAB0212068FFF73DF820680122FF21F0
:1024F000FEF778FF206800224F21FEF773FF206867
:102500002C224E21FEF76EFF20680022FF21FEF7ED
:1025100069FF2068B422B621FEF764FF0025002E73
:1025200018BF0C2608F07F082A460120C5F3C40C0A
:102530000CF128035FFA85FE0DEB030C76451CF8C1
:102540001C3C05F0070102D8904540F0E38200FAF8
:1025500001F123EA01030CF81C3C0135302DE5D1D3
:10256000062303AAB0212068FEF76CFF524B01221C
:102570001870FF212068FEF735FF00221146206801
:10258000FEF730FF20680022FF21FEF72BFF2068B6
:1025900000220921FEF726FF206800221021FEF705
:1025A00021FF206800221121FEF71CFF2068012274
:1025B0002421FEF717FF2068FF222521FEF712FFD6
:1025C000206800227521FEF70DFF20680122FF21FF
:1025D000FEF708FF20682C224E21FEF703FF20683B
:1025E00000224821FEF7FEFE294620682022FEF741
:1025F000F9FE20680022FF21FEF7F4FE294620683C
:102600000922FEF7EFFE206800225421FEF7EAFEC1
:10261000206804223121FEF7E5FE206803223221E2
:10262000FEF7E0FE206883224021FEF7DBFE2068F3
:1026300025224621FEF7D6FE206800226021FEF703
:10264000D1FE206800222721FEF7CCFE206806225A
:102650005021FEF7C7FE206800225121FEF7C2FE7E
:10266000206896225221FEF7BDFE206808225621DE
:10267000FEF7B8FE2A4620685721FEF7B3FE206811
:1026800000226121FEF7AEFE206800226221FEF7E3
:10269000A9FE206800226421FEF7A4FE2068002223
:1026A0006521FEF79FFE2068A0226621FEF79AFEB4
:1026B00006E000BFC062002060100020542B002004
:1026C00020680122FF21FEF78DFE206832222221A0
:1026D000FEF788FE206814224721FEF783FE20685B
:1026E000FF224921FEF77EFE206800224A21FEF7E4
:1026F00079FE20680022FF21FEF774FE20680A227E
:102700007A21FEF76FFE206800227B21FEF76AFE29
:10271000206821227821FEF765FE20680122FF2132
:10272000FEF760FE206834222321FEF75BFE20685E
:1027300000224221FEF756FE2068FF224421FEF7C8
:1027400051FE206826224521FEF74CFE2068052216
:102750004621FEF747FE402211462068FEF742FE62
:10276000206806220E21FEF73DFE20681A22202155
:10277000FEF738FE206840224321FEF733FE206832
:102780000022FF21FEF72EFE206803223421FEF7EF
:1027900029FE206844223521FEF724FE206801220C
:1027A000FF21FEF71FFE206804223121FEF71AFEEA
:1027B000206809224B21FEF715FE206805224C21D6
:1027C000FEF710FE206804224D21FEF70BFE206864
:1027D0000022FF21FEF706FE206800224421FEF7BA
:1027E00001FE206820224521FEF7FCFD206808221A
:1027F0004721FEF7F7FD206828224821FEF7F2FD69
:10280000206800226721FEF7EDFD20680422702178
:10281000FEF7E8FD206801227121FEF7E3FD206844
:10282000FE227221FEF7DEFD206800227621FEF7EF
:10283000D9FD206800227721FEF7D4FD206801220F
:10284000FF21FEF7CFFD206801220D21FEF7CAFD12
:1028500020680022FF21FEF7C5FD206801228021AB
:10286000FEF7C0FD2068F8220121FEF7BBFD2068BD
:102870000122FF21FEF7B6FD206801228E21FEF71E
:10288000B1FD206801220021FEF7ACFD2068002286
:10289000FF21FEF7A7FD206800228021FEF7A2FDA0
:1028A000042220680A21FEF79DFD25688421284620
:1028B000FFF789FC842100F0EF022846FEF792FD25
:1028C000012220680B21FEF78DFD256801A928460D
:1028D000FFF7B6FC05AA01A92846FFF7C6FC9DF83C
:1028E0000430002B00F01C81089D05F684559DF8EE
:1028F0000630002B00F01781089B03F2B22305EB92
:1029000043059DF8073023B1BDF8243003F5257346
:102910001D449DF8083023B1BDF8263003F226236C
:102920001D44E8222068C7F8385E0121FEF75AFDF1
:102930002068294645F0A3FD012220681146FEF7D4
:1029400051FD20684021FFF74DFC002800F0DF809A
:10295000206801210222FEF745FD20680021FFF7D3
:1029600041FC002800F0D3802068DFF8D481E82201
:102970000121FEF737FD206820224421FEF781FD6A
:10298000256801A92846FFF75BFC05AA01A928468E
:10299000FFF76BFC502257212846FEF723FD082243
:1029A00056212846FEF71EFD082250212846FEF734
:1029B00019FDBDF824004FF47A7948F20E6609FB40
:1029C0000060B0FBF8F080B2FEF7B8FA5121024681
:1029D0002846FEF756FD089B09FB0366574B9E42AF
:1029E0009DBFB6FBF8F202F1FF32D2B2FF224621C0
:1029F0002846FEF7F7FCD7F8381E284645F03FFD7D
:102A000001212846FFF7DFFB022206460121284666
:102A1000FEF7E8FC00212846FFF7E4FB32460121DF
:102A20002846FEF7DFFC246801A92046FFF708FCD2
:102A300005AA01A92046FFF718FC482211462046A6
:102A4000FEF7D0FC082247212046FEF7CBFC0322EC
:102A500032212046FEF7C6FC072230212046FEF731
:102A6000C1FC0122FF212046FEF7BCFC20223021C0
:102A70002046FEF7B7FC0022FF212046FEF7B2FCFD
:102A8000062220467021FEF7ADFCBDF826304FF43B
:102A90007A7246F6440002FB03004DF28803B0FB55
:102AA000F3F09DF8073080B21BB1BDF81A3018441E
:102AB00080B2FEF743FA712102462046FEF7E1FCA0
:102AC000D7F8381E204645F0DAFC01212046FFF7F2
:102AD0007AFB0222054601212046FEF783FC0021F5
:102AE0002046FFF77FFB2A4601212046FEF77AFCAD
:102AF0006423C7F8303E012387F8E03007E0D8F8B8
:102B000000309BB29B1BB3F5FA7F7FF6ADAC0BB0E8
:102B1000BDE8F0830B41DB0744BF0132D2B21CE5B4
:102B200040F63635E3E69DF80530002B3FF4E9AE7C
:102B3000089B03F525731D44E3E600BF1B280D0128
:102B40001C0C010070B53B4C94F8E0300546002B9E
:102B500036D094F83C6E012E33D0022E4FD07EBB7F
:102B6000006801228021FEF73DFC28680122FF2138
:102B7000FEF738FC286832463146FEF733FC94F8FD
:102B8000342E28689121FEF72DFC28680122314659
:102B9000FEF728FC28683246FF21FEF723FC286850
:102BA00032468021FEF71EFC286801223146FEF7DE
:102BB00019FC214B1B68C4F82C3E012384F83C3ED1
:102BC00070BD00680021FFF7FEFAC20711D5D4F8E6
:102BD000302E002AF4D0184BD4F82C1E1B689BB260
:102BE0005B1A9A42ECD2154B4FF0FF325A60002329
:102BF000E4E7114B1B68C4F82C3E0223DEE70068B3
:102C00001321FFF7E0FA4307E1D01E212868FEF701
:102C100083FF012206460B212868FEF7E3FB0A2307
:102C2000B6FBF3F6054BB6B25E60012384F8E130E3
:102C3000DDE700BFC0620020542B002060100020A0
:102C400010B5EFF31181102383F312884FF0E023C6
:102C5000C9B29C691A6912F4803F0D4A1EBF012057
:102C6000C2F8140D9C690B4B1868D2F8143D81F31F
:102C70001188D2F8181D4FF47A72034402FB01F058
:102C8000001BB0FBF1F00021E3FB020110BD00BF0F
:102C9000C0620020542B0020124B5B68C3F3080372
:102CA00030B4EBB9EFF31183D3B90F490F4B4FF0A9
:102CB000E0250A68AC6908688242FAD1D3F8100DA1
:102CC0008442F6D8D3F8181D4FF47A7303FB01F051
:102CD000001BB0FBF1F00021E2FB030130BC7047A8
:102CE00030BCADE700ED00E0542B0020C0620020B6
:102CF00010B5074C94F8410E40B1FFF7CDFFD4F862
:102D0000483EC01AC0F5FA5020EAE07010BD00BF7E
:102D1000C0620020F8B506460D46FFF7BDFF044629
:102D20000F46FFF7B9FF021B61EB0703B242AB414D
:102D3000F7D3F8BD38B50D460446FFF7D9FF011E9D
:102D400002DDC917FFF7E6FF064B2068002283F873
:102D5000412E492193F8423E2A46FEF703FC01200A
:102D600038BD00BFC06200202DE9F341384CD4F8D3
:102D7000503EC0F83630B4F8543E438794F8403E95
:102D8000012B064600F1360804F565670CD0022BCE
:102D900026D0A3BB0122022143F029FE012384F89F
:102DA000403E94F8565E10E0FFF7A2FF94F8565E9E
:102DB00058B969463046FFF7BDFF9DF8003008B1AD
:102DC0009B0706D1002384F8403E284602B0BDE8A8
:102DD000F08107220321304643F009FE0223F2E787
:102DE000FFF786FF0028DCD169463046FFF7A2FFD7
:102DF0009DF80630054610B113F0080205D00025F5
:102E000084F8405E84F8565EDFE7B4F9581E6846E1
:102E1000FCF712F84042B4F95A1EF0860DF1020098
:102E2000FCF70AF8B4F95C1E308701A8FCF704F837
:102E3000D6F83630C4F8503E40427087B8F80430B7
:102E4000BB80012384F8402E84F8563EBDE700BFC6
:102E5000C062002010B50446013C00D210BD4FF402
:102E60007A700021FFF756FFF6E738B5056804468B
:102E700000212846FCF7F0FCB62214212846FEF774
:102E800073F96420FFF7E6FF812210212068FEF726
:102E90006BF90120FFF7DEFF152120688022FEF785
:102EA00063F90120FFF7D6FF20680321BDE8384011
:102EB000FCF7D2BC38B50568044600212846FCF76B
:102EC000CBFCB6227E212846FEF74EF96420FFF7A0
:102ED000C1FF00227C212068FEF746F96420FFF73D
:102EE000B9FF04227D212068FEF73EF96420FFF738
:102EF000B1FF8C2240212068FEF736F90120FFF750
:102F0000A9FF022241212068FEF72EF90120FFF7D8
:102F1000A1FF20680221FCF79FFC4FF40063A3810E
:102F200038BD10B504464069FCF755FF0120FFF796
:102F300091FF6069FCF74AFFBDE810400A2089E76D
:102F400073B50468B6227E2105462046FEF70CF9CB
:102F50006420FFF77FFF02212046FCF77DFC20461E
:102F6000FFF7DFFF00227C212046FEF7FDF801205D
:102F7000FFF770FF002259212046FEF7F5F80120E7
:102F8000FFF768FF5E238DF8073094F910301422A4
:102F900053433D4AD658A3689A0702D4606945F066
:102FA000C1FC01230DF107020021304646F048FA2A
:102FB0004FF4A473354A0021304646F041FAA36825
:102FC0009B0702D42046FEF79FF80A20FFF742FF36
:102FD000012259212046FEF7C7F80120FFF73AFFEA
:102FE0008C2240212046FEF7BFF80120FFF732FF78
:102FF000032241212046FEF7B7F80120FFF72AFF00
:10300000234EA96B234A95F83500B6FBF1F109234D
:1030100089B2FCF795F84388B6FBF3F62E64027983
:10302000422142F0C0022046FEF79EF80120FFF741
:1030300011FF082243212046FEF796F80120FFF7F2
:1030400009FF042258212046FEF78EF80120FFF7E1
:1030500001FF0A2253212046FEF786F80120FFF7E0
:10306000F9FE00227C212046FEF77EF80120FFF7C2
:10307000F1FE06227D212046FEF776F8012002B0FF
:10308000BDE87040E6E600BFB00000208F140608DF
:1030900040420F00D8150608F8B5816B0468294A2C
:1030A000294FB7FBF1F10546102389B290F835009E
:1030B000FCF746F800214388B7FBF3F706462F6478
:1030C0002046FCF7C9FB80226B212046FEF74CF816
:1030D0006420FFF7BFFE032268212046FEF744F874
:1030E0006420FFF7B7FE01226B212046FEF73CF873
:1030F0000F20FFF7AFFE18221B212046FEF734F801
:103100000F20FFF7A7FE18221C212046FEF72CF8FF
:103110000F20FFF79FFE32791A212046FEF724F890
:103120000F20FFF797FE727919212046FEF71CF851
:103130006420FFF78FFE20460321BDE8F840FCF72E
:103140008BBB00BF0E16060840420F00F7B50F23D9
:103150000468816B654A664FB7FBF1F1054689B299
:1031600090F83500FBF7ECFF00214388B7FBF3F73D
:1031700006462F642046FCF76FFB0022762120468E
:10318000FDF7F2FF0F224E212046FDF7EDFF0F2045
:10319000FFF760FE72794F2102F00F022046FDF723
:1031A000E3FF0F20FFF756FE7279502102F00F0265
:1031B0002046FDF7D9FF0F20FFF74CFE5221FF22DA
:1031C0002046FDF7D1FF0F20FFF744FE95F835109C
:1031D000072941D0474E96F8E900FBF7FDFF054669
:1031E000012276212046FDF7BFFFAA780C21204658
:1031F000FDF7BAFF2A790D212046FDF7B5FFAA7920
:10320000AB88120142EA1322D2B20E212046FDF70A
:10321000ABFF4FF4807196F8E900FBF7DDFF054640
:10322000022276212046FDF79FFFAA78520002F085
:10323000FE0203212046FDF797FF2A79042120464C
:10324000FDF792FFAA79AB88120142EA1322D2B2AB
:1032500005212046FDF788FF002276212046FDF754
:1032600083FF032214212046FDF77EFF0F20FFF786
:10327000F1FD002263212046FDF776FF6420FFF771
:10328000E9FD082265212046FDF76EFF0DF10702DA
:1032900064212046FEF74AFE9DF8072022F0100226
:1032A00042F06002642120468DF80720FDF75CFFA4
:1032B0000F20FFF7CFFD0DF106024D212046FEF74E
:1032C00035FE9DF8062002F03F0242F040024D21FB
:1032D00020468DF80620FDF747FF0F20FFF7BAFDC7
:1032E00003212046FCF7B8FA03B0F0BD6E160608BD
:1032F00040420F00C0620020F8B5816B04682D4A7F
:103300002D4FB7FBF1F10546102389B290F8350037
:10331000FBF716FF00214388B7FBF3F706462F643F
:103320002046FCF799FA80226B212046FDF71CFF0E
:103330006420FFF78FFD072268212046FDF714FF68
:103340006420FFF787FD00226B212046FDF70CFF6C
:103350006420FFF77FFD01226B212046FDF704FF6B
:103360000F20FFF777FD18221B212046FDF7FCFEFA
:103370000F20FFF76FFD18221C212046FDF7F4FEF9
:103380000F20FFF767FD32791A212046FDF7ECFE8A
:103390000F20FFF75FFD727919212046FDF7E4FE4B
:1033A0006420FFF757FD20460321BDE8F840FCF7F5
:1033B00053BA00BF0E16060840420F009CE710B536
:1033C0007822044600210068FDF7CEFE0520FFF7B5
:1033D00041FD202201212068FDF7C6FE0520FFF7F0
:1033E00039FD002202212068FDF7BEFE6420FFF7B0
:1033F00031FD012010BD10B5072204460A210068E6
:10340000FDF7B2FE0520FFF725FD242241212068AB
:10341000FDF7AAFE0520FFF71DFDC022422120680E
:10342000FDF7A2FE0520FFF715FD012010BD10B528
:103430000122044610210068FDF796FE48B11420D1
:10344000FFF708FD2068A022BDE810401121FDF71C
:103450008BBE10BD13B5044600210068FCF7FCF9D3
:103460000021204643F0AAFA1420FFF7F3FC0F21B5
:10347000204643F0A3FA0A20FFF7ECFC01AA03233D
:103480001021204641F0B8FC0A20FFF7E3FC9DF82C
:103490000420174B8032A3F8582E9DF80520803267
:1034A000A3F85A2E9DF80620002180322046A3F86A
:1034B0005C2E43F083FA0A20FFF7CCFC0DF10302E7
:1034C00001230221204641F097FC01230DF1030264
:1034D0000921204641F090FC2046122143F06EFA6B
:1034E00020680321FCF7B8F9012002B010BD00BF2D
:1034F000C062002008B5006801220921FDF734FEF2
:10350000BDE808406420A5E480B506460A250121EF
:103510000846FCF787FE00210846FCF783FE771C6F
:103520004FF03208052457EA040307D14FF47A70AC
:10353000FFF790FC013DEAD1FDF79BFD0120FCF770
:103540005FFE0020FCF75CFE0120FDF73CFD4046DD
:10355000FFF780FC0120FCF753FE0020FCF750FE33
:10356000FDF731FD4046FFF775FC44B1013CDAD16F
:103570004FF4FA70FFF76EFC4FF0FA08D3E7013F03
:10358000D1E737B50568044600212846FCF764F901
:1035900015227E212846FDF7E7FD6420FFF75AFC3F
:1035A00011227E212068FDF7DFFD0520FFF752FC88
:1035B00020680DF107020321FEF7B8FC9DF80730E3
:1035C00003F03C03142B02D00620FFF79DFF0C22D2
:1035D00040212068244DFDF7C7FD0120FFF73AFC8C
:1035E000A16B224A94F83500B5FBF1F1092389B2A9
:1035F000FBF7A6FD4388B5FBF3F525640279206847
:103600004221FDF7B1FD0120FFF724FC08224121F2
:103610002068FDF7A9FD0120FFF71CFC00224321D3
:103620002068FDF7A1FD0120FFF714FC10225121B5
:103630002068FDF799FD0120FFF70CFC0A225321B9
:103640002068FDF791FD0120FFF704FC8022562140
:103650002068FDF789FD0120FFF7FCFB20680321AE
:10366000FCF7FAF803B030BD40420F00C816060858
:10367000F0B5816B0568514A514FB7FBF1F185B048
:103680000446102389B290F83500FBF759FD00215C
:103690004388B7FBF3F7064627642846FCF7DCF8B7
:1036A00080226B212846FDF75FFD9620FFF7D2FBB5
:1036B000032268212846FDF757FD9620FFF7CAFB35
:1036C00003226B212846FDF74FFD0F200021FFF755
:1036D00021FB10226A212846FDF746FD0F2000211C
:1036E000FFF718FB00226C212846FDF73DFD0F2057
:1036F0000021FFF70FFB727919212846FDF734FDF1
:103700000F200021FFF706FB18221B212846FDF79A
:103710002BFD0F200021FFF7FDFA18221C2128465F
:10372000FDF722FD0F200021FFF7F4FA32791A216C
:103730002846FDF719FD01200021FFF7EBFA0321D0
:103740002846FCF789F82068062302AA4321FDF7E2
:1037500009FFD0B1BDF80830DBBA07EE903ABDF8EA
:103760000A30F8EEE77ADBBAC4ED077A07EE903A52
:10377000BDF80C30F8EEE77ADBBAC4ED087A07EE54
:10378000903AF8EEE77AC4ED097AD4ED087AFDEEC6
:10379000E77ACDED017A9DF9043001330CD1D4EDF7
:1037A000077AFDEEE77ACDED017A9DF90430013319
:1037B00002D10620FFF7A8FE05B0F0BD0E160608E0
:1037C00040420F0018B103685B6803B11847FF203F
:1037D000704718B103689B6803B118470020704711
:1037E00070B450B106798E4207D34579954204D31F
:1037F0000368DB680BB170BC184770BC704710B42D
:1038000040B184798C4205D303681B6913B15DF81C
:10381000044B18475DF8044B704718B103685B69A7
:1038200003B11847704718B10368DB6903B1184743
:103830000020704718B103681B6A03B118470020C5
:10384000704730B50A4658B1041D00F114032068D2
:103850006168154603C508349C422A46F7D1012009
:1038600030BD10B50C4670B92D23002023750A4BCE
:103870002061C4E90000C4E90200C4E90633302332
:1038800084F8203010BD0368DB6A002BECD0984729
:103890000028E9D0F6E700BF3DF0060838B5054D31
:1038A000441E14F8011F01B938BDD5F8600EFBF7AE
:1038B00095FFF6E7C062002070B50C4C0E46054639
:1038C0000B48FFF7EBFF33460A49D4F8600E2A464F
:1038D00043F01AFDD4F8600EFBF774FF94F8643ED1
:1038E00013B1012384F8653E70BD00BFC0620020A3
:1038F00005B90608FDF7000808B50648FFF7CEFF32
:10390000054BB3F8660E18B1BDE80840FFF7A2BA40
:1039100008BD00BFBF140708C062002010B5074CE7
:1039200002460B46D4F8600E054943F0EDFCD4F88E
:10393000600EFBF747FFBDE81040DDE7C0620020E6
:10394000FDF7000808B5FFF7A9FFBDE80840D3E779
:1039500010B504460648FFF7A1FF2046FFF79EFF7B
:10396000044B93F8642E12B1012283F8652E10BD2A
:1039700005B90608C062002010B504460348FFF7E9
:103980008DFF2046BDE81040DCE700BF11B90608F6
:103990000CB4830607B500D551B9049805A9019167
:1039A000FFF7BCFF012003B05DF804EB02B07047E5
:1039B0000020F8E7024B0146D3F8600EFBF70EBF7C
:1039C000C06200200CB407B510F0400009D069B9FE
:1039D0002320FFF7EFFF049805A90191FFF79EFF51
:1039E000012003B05DF804EB02B070470020F8E757
:1039F0000FB413B5094C0A49D4F8600E04AB53F860
:103A0000042B019343F080FCD4F8600EFBF7DAFE40
:103A100002B0BDE8104004B0704700BFC062002093
:103A2000FDF700080FB407B504A951F8040B019184
:103A3000FFF774FF03B05DF804EB04B070470FB4F8
:103A400007B504A951F8040B0191FFF735FFFFF703
:103A500053FF03B05DF804EB04B0704770B5837991
:103A6000164603F007028CB00446062A4FD8DFE85A
:103A700002F0041417191C1E49000D7813F0C0033E
:103A800047D0402B3CD12946204615F007FC0028A2
:103A900059D00CB0BDE87040AAE791F90050EDE7AD
:103AA0000D88EBE7B1F90050E8E70D68E6E791ED26
:103AB000000A6846FAF720FC01462848FFF798FFFD
:103AC000F6B1A3793F2B1BD8204615F041FB00EE41
:103AD000100A6846B8EEC00AFAF70EFC0146204804
:103AE000FFF786FF204615F043FB00EE100A6846FC
:103AF000B8EE400AFAF700FC01461948FFF778FFD4
:103B00000CB070BD15480CB0BDE8704070E70025E2
:103B1000B4E7042A0CBF134813482946FFF768FF8F
:103B2000002EEDD0A3793F2BEAD8204615F010FBEC
:103B30000546204615F01CFB02460C4829460CB0F1
:103B4000BDE8704054E76946204615F00FFA084872
:103B50006A462946FFF773FFD2E700BF16BF060883
:103B600045C1060862B9060894EF0608E115070882
:103B700016B906082DE9F04F8FB001F020034C4C28
:103B8000009381460F464FF000084A4BD3F8600E71
:103B9000FBF718FE94F806B00BF038034B4549D1FB
:103BA000204615F05BFAFAF7F7FD8568204615F018
:103BB0007FFA82462E18204615F0BEFA0BF0070257
:103BC0000146062A6BD8DFE802F0043F44484D5115
:103BD0005D0015F80A200978511A4A424A41009BB3
:103BE00003B13ABB02A92046019215F0BFF97B064A
:103BF00015D5019A9AB9304802A9FFF7F9FE2F4965
:103C000002A845F0E5FC00284BD115F80A30202B1E
:103C100047D12B483146FFF7EBFEFFF76DFE2948F1
:103C200002A9FFF7E5FE002231462046FFF716FF06
:103C3000FFF762FE08F10108B8F5197F04F10B04E3
:103C4000A3D10FB0BDE8F08F15F90A2091F900104B
:103C5000C2E735F80A200988BEE735F90A20B1F92C
:103C60000010B9E755F80A200968B5E796ED007A23
:103C7000D1ED007AB4EE677AF1EE10FA0CBF0122B2
:103C80000022ACE72046019115F072FA0199421C1E
:103C900030464AF0B9FEB0FA80F252099FE700229E
:103CA0009DE7002231462046FFF7D8FEB5E700BF6A
:103CB00032190608C062002033B90608B315070898
:103CC0000EBF060834B9060838B50D46044615F08F
:103CD00033FA2A4601462046BDE83840BEE6F8B52C
:103CE000847914F0C003064602D0402B15D0F8BDED
:103CF00015F03EFA04F00704062C054604D10146EF
:103D0000BDE8F84012488DE6304615F021FA2A4603
:103D10000146BDE8F8400F4884E615F0AFFA0546C5
:103D20000D480E4E0E4FFFF7B9FD00242B79A3422C
:103D300002D8BDE8F840DFE514B13046FFF7AEFD2C
:103D40002B68384653F82410FFF752FE0134EDE794
:103D50003EB906084EB9060865B9060875B90608E1
:103D600045C1060808B50548FFF798FD044BD3F890
:103D7000600EBDE80840FBF725BD00BF11B906087D
:103D8000C062002000485AE677B9060813460A4682
:103D90000146014853E600BF83B9060820B1007808
:103DA000B0FA80F040097047012070472DE9F04FCC
:103DB00087B00346FFF7F2FF064618B107B0BDE82B
:103DC000F04FDFE74649DFF84491DFF844A1DFF820
:103DD00010B105AA18464AF070FE34460546B046B2
:103DE0004FF0FF378DB97EB230461FF031F810B179
:103DF0004568002D5AD1B8F1000F36D139483946FF
:103E0000F9F77FFD07B0BDE8F08F012E0ED0022E2E
:103E100011D01EB92846FAF75FFB074605AA594696
:103E200000204AF04AFE01360546DBE72846FAF74D
:103E300053FB8046F2E7494628464CF0A2FE20B9E3
:103E4000294928464CF09DFE08B144F00104514632
:103E500028464CF096FE28B9244928464CF091FE9D
:103E60000028DBD044F00204D8E7002C08BF03246C
:103E70000023E4B2CDE9008402931A461946304685
:103E80001FF0A4F9054610B919483946B8E7194892
:103E900042463946F9F735FD39461748F9F731FDFD
:103EA000164B2946D3F8680E40F0F4F8144839460A
:103EB000F9F727FD5CB16979A14208D01148224683
:103EC000F9F71FFD2B68E1B29B6928469847EB6A1A
:103ED000002BE1D00C48F9F714FD0023EB62DBE77F
:103EE000DC0D0708A3B9060899F5060898D406085A
:103EF000CBB90608EAB9060855BA0608C062002020
:103F000007BA06081FBA06083FBA0608BBCC06085F
:103F1000A0B906082DE9F04F85B00546FFF73EFF32
:103F2000044630B10021012005B0BDE8F04F40F05B
:103F300009B985492846F9F79BFE20B905B0BDE8C7
:103F4000F04F39F00BBA81492846F9F791FE28B9AC
:103F5000012005B0BDE8F04F39F066BB7C4928462A
:103F6000F9F786FE90BB7B4B93F9272E83F8200E42
:103F7000194693F8D254012D09D0033D052D06D9D9
:103F80000CB181F8272E05B0BDE8F04FFAE693F8A2
:103F9000D354A52D00F1010013D1012A0ED181F8CF
:103FA000202E6D4A81F8210E002382F86C3E81F8A4
:103FB000273E05B0BDE8F04F39F07EBB013A52B262
:103FC0000124782803F11403D3D1D9E72846FAF75E
:103FD00083FA614B93F96C3E009303FA80F6772ED7
:103FE000834600F2A7802846FBF732FB07460028ED
:103FF00000F08C80FAF770FA0124C5B23846FBF75E
:1040000027FB0746002800F08480FAF765FA0134A0
:104010000190E4B23846FBF71BFB804600287AD0BB
:10402000FAF75AFA01340746E4B24046FBF710FBB0
:104030008146002871D0FAF74FFA01340290E4B2B9
:104040004846FBF705FB8246002868D0FAF744FA99
:1040500001340FFA80F9E4B25046FBF7F9FA8246D0
:1040600000285ED0FAF738FA01340FFA80F8E4B28B
:104070005046FBF7EDFA002855D00390FAF72CFADA
:10408000039A0FFA80FA1046FBF7E2FA034600287B
:1040900057D004F0FD04FAF71FFA042C7FF473AF35
:1040A000C3B2012D03D9EA1E052A3FF66CAF23B136
:1040B000A52B02D0482B7FF466AF26480EB980F8B6
:1040C000276E142202FB06020199C2F8C014A52B28
:1040D000029982F8D254C2F8C474C2F8C814A2F883
:1040E000CC94A2F8CE84A2F8D0A482F8D3340AD11A
:1040F000009B194A01335B4482F86C3E90F8273EDE
:10410000013380F8273E05B0BDE8F08F0446054630
:1041100074E701907EE7074687E7029090E78146C3
:104120009AE78046A4E75FFA88F382468046062C29
:10413000B7D028E709487722214605B0BDE8F04FFF
:1041400024E60134E4B2F2E783BA060889BA060825
:10415000A2CA060810950020C06200208EBA060888
:1041600010B50346FFF71AFE30B1FCF7AFF9BDE812
:1041700010400748FFF7E6BB1846FAF7ADF90446CA
:1041800080B2FCF777F921460248BDE8104049E4C7
:1041900097BA0608A3BA060808B50346FFF7FEFD5E
:1041A00040B10C4B0C480022A3F8662EBDE8084035
:1041B000FFF7C8BB1846FAF78FF9014630B1054B37
:1041C000A3F8660EBDE8084004482BE4BDE80840AB
:1041D000D8E500BFC0620020B5BA0608CBBA060811
:1041E0002DE9F04F834689B090460C4616460027CD
:1041F0004FF0190A4FF46179B8F1000F4BD03078C5
:1042000025787178B378F278854242D165788D420D
:104210003FD1A5789D423CD1E578A5EB020CDCF1BD
:10422000000545EB0C05CDE90632059114F016F8B2
:10423000079A069B059901911AFB02921AFB0393B8
:104240000392029343790093144A3B462946584609
:10425000FFF7B8FB207814F001F8E3780F4A1AFB57
:1042600003930393A3781AFB039302936378019358
:104270004379009329463B4658460137FFF788FBB0
:10428000282F04F1040406F10406B5D109B0BDE8F5
:10429000F08F0025C7E74546DCE700BFE2BA060815
:1042A000F7B50746FFF77AFD044630B12E490022E4
:1042B000012003B0BDE8F04092E73846FAF70CF968
:1042C0002728054648DC8600781C8DF80740FBF758
:1042D000BFF9074690B1FAF7FFF8031E0EDB234A39
:1042E0002146DBB202F2945404EBC10CC8009CF8E6
:1042F00005C09C4525D001313929F5D13846FBF759
:10430000A7F9044660B1FAF7E7F80D2808D8184B6A
:10431000334483F86E0E9DF8073001338DF8073073
:10432000114FB11C0DF1070239442046FBF79DF9EE
:104330009DF80730042B02D0002347F8253003B046
:10434000F0BD0B4B0244334492F8982583F86D2E50
:1043500001238DF80730D1E706482722214603B014
:10436000BDE8F04012E500BF2D7100206C11060879
:10437000C0620020F8BB06082DE9F04F3F4FDFF880
:1043800004A189B0814690460C46164602F1300BD6
:1043900094F9045000230C22394802FB03F109561A
:1043A000A94266D00133042BF6D10C36B34504F193
:1043B0000C04EDD109B0BDE8F08F96F90430D6F8C1
:1043C00000E07279B179307A96F807C007939D4280
:1043D0004DD1256875454AD16579954247D1A57972
:1043E0008D4244D1257A854241D1E579A5EB0C0374
:1043F0005D425D4107EB820207EB8C0C07EB80000E
:1044000007EB8101D2F85C27DCF85C37D0F85C0759
:10441000D1F85C170493CDE900E203900291079B69
:10442000524629464846FFF7CDFAE27994F904301E
:1044300007EB82022946D2F85C270492227A07EB26
:1044400082024846D2F85C270392A27907EB8202E7
:10445000D2F85C270292627907EB8202D2F85C27DD
:104460000192226800925246FFF792FA9DE70025DA
:10447000C0E7B8F1000FA0D14546D6E76C11060899
:10448000D0710020F5BA06082DE9FF410346FFF779
:1044900085FC30B144490022012004B0BDE8F04160
:1044A0006AE718465E1CFAF717F8044640B21EF099
:1044B0004BFE054630B93D48214604B0BDE8F04109
:1044C000FFF7BDBA0068696801AB03C3A86818604C
:1044D0003046FBF7BDF80446002852D003782B2B5A
:1044E00005D02D2B42D0F9F7F7FF019009E00134F8
:1044F0002046F9F7F1FF012303FA00F0019B034383
:10450000019302262A4F4FF000082046FBF7A0F83F
:10451000044628B3F9F7E0FF264A002352F8041BAB
:10452000884230D00133112BF8D1002307EB8302EE
:10453000D2F85C27904213D1B8F1020F25D0B8F120
:10454000030F25D0B8F1010F14BF8DF809308DF895
:104550000A3008F101080136B8F1040FF6B2D4D1DF
:10456000012E18D804B0BDE8F0410BE40134204618
:10457000F9F7B2FF012303FA00F0019B23EA0003DD
:10458000BEE70126BEE7DBB2D0E78DF80C30E0E7EE
:104590008DF80B30DDE701AB03CB2860186869604C
:1045A000A86004B0BDE8F0810072002012BB0608CC
:1045B0006C110608C81806082DE9F04F834687B02D
:1045C00090460C46164600274FF0190A4FF46179C1
:1045D000B8F1000F4DD0B078A5783378727896F89E
:1045E00003C096F804E07179854240D125789D4258
:1045F0003DD1657895423AD1E578654537D1257941
:10460000754534D165798D4214BF002501251AFB0B
:1046100002921AFB0393CDE9010303920091CDE9C5
:1046200004CE154A3B4629465846FFF7CBF9237975
:104630000593E378049363780F4A1AFB039303937B
:1046400023781AFB03930293A37801936379009371
:1046500029463B4658460137FFF79AF9142F04F1D3
:10466000060406F10606B3D107B0BDE8F08F0025B9
:10467000CDE74546DBE700BF25BB06082DE9F3473C
:104680008246FFF78BFB064630B13E4900220120EF
:1046900002B0BDE8F0478FE75046F9F71DFF132839
:1046A000054663DC062747430AF101008DF80760E1
:1046B000354CFAF7CDFF04F6747909EB0708064686
:1046C00048B1F9F709FF03289FBFE31983F8790F71
:1046D00001238DF807303046FAF7BAFF064668B175
:1046E000F9F7FAFE0D2809D8062303FB054383F8E2
:1046F000760F9DF8073001338DF807300DF1070272
:1047000041463046FAF7B1FFFAF7A2FF064668B114
:10471000F9F7E2FE3B2809D89DF80730062202FB94
:104720000542013382F8770F8DF807303046FAF7EB
:104730008FFF68B1F9F7D0FE0D2809D89DF8073032
:10474000062202FB0544013384F8780F8DF8073008
:104750009DF80730062B11D0002349F80730A8F840
:10476000043002B0BDE8F047FFF70CBB0748132246
:10477000314602B0BDE8F047FFF708BB02B0BDE824
:10478000F08700BF34720020C0620020F8BB06082A
:104790002DE9F04F2DED088BDFF814A197B00746F7
:1047A00090460C461546002694ED008AB5EE408AE8
:1047B000F1EE10FA73D0D4ED019A94ED029AD4ED93
:1047C000038AB8F1000F40D095ED000A95ED01BACB
:1047D000D5ED02AA95ED03AAB4EE408AF1EE10FAE7
:1047E00062D1F4EE4B9AF1EE10FA5DD1B4EE6A9A12
:1047F000F1EE10FA58D1F4EE4A8AF1EE10FA0CBF3D
:104800004FF001094FF0000912A8F9F775FDB0EE5D
:104810004B0A83460EA8F9F76FFDB0EE6A0A0590C1
:104820000AA8F9F769FDB0EE4A0A049006A8F9F75C
:1048300063FD059B049A0390CDE900B302923346D1
:10484000524649463846FFF7BDF8B0EE480A12A86E
:10485000F9F752FDB0EE690A81460EA8F9F74CFD52
:10486000B0EE490A83460AA8F9F746FDB0EE680A99
:10487000049006A8F9F740FD049B0390CDE901B32D
:10488000CDF8009033465246002138460136FFF7F6
:104890007FF80C2E04F1100405F1100584D117B037
:1048A000BDEC088BBDE8F08F4FF00009ACE700BF0E
:1048B00043BB060870B50546FFF770FA064668B1B7
:1048C000434B444993F886304FF4C87202FB0311FE
:1048D000BDE8704000221031012059E73E49052211
:1048E0002846F9F7ABF970B9394B93F88620394B64
:1048F0004FF4C87101FB02330C220021013A43F846
:10490000101FFBD170BD2846F9F7E6FD0B280446C1
:1049100057D82846FAF79CFE064600283BD0F9F700
:104920004FFD2B4B93F88620192303FB0242294BA2
:1049300003EB021383ED040A01253046FAF788FEE3
:10494000064668B1F9F73CFD214B93F88620192300
:1049500003FB02421F4B03EB021383ED050A0135F3
:104960003046FAF775FE064668B1F9F729FD184B8F
:1049700093F88620192303FB0242164B03EB021324
:1049800083ED060A01353046FAF762FE28B9BDE824
:104990007040FFF7F7B90546CFE70D4B93F88660F7
:1049A000F9F70EFD0B49192303FB064401EB041430
:1049B000032D84ED070AEAD14FF4C87303FB0611F7
:1049C00086E731460548BDE870400B22FFF7DEB9A7
:1049D000B8730020AC72002083BA0608F8BB060842
:1049E0002DE9F347DFF868A081460E4617464FF0E1
:1049F0000208002457B337F8243036F8241037F86B
:104A00000820994220D136F80850A91A4D424D414C
:104A1000CDE900322946234652464846FEF7D2FFEA
:104A200036F80830019336F8243000935246234676
:104A3000294648460134FEF7ABFF042C08F1040870
:104A4000D8D102B0BDE8F0870025E1E73D46E7E7B1
:104A500057BB0608F8B50446FFF7A0F9054628B18C
:104A6000BDE8F840294900220120B9E7284920463D
:104A7000F9F7FEF8A8B9274B4FF47A714FF4FA62B0
:104A8000A3F8AC10A3F8AE20A3F8B010A3F8B2209E
:104A9000A3F8B410A3F8B620A3F8B810A3F8BA206E
:104AA000F8BD2046F9F718FD0328074627D8204609
:104AB000FAF7CEFD044670B1F9F70EFD0125064662
:104AC0002046FAF7C5FD10B1F9F706FD2DB9BDE88E
:104AD000F840FFF757B90546F2E7A6F2EE2240F29A
:104AE000DC539A42F3D8A0F2EE229A42EFD8094B57
:104AF00003EB8703A3F8AC60A3F8AE00D0E7294628
:104B00000548BDE8F8400322FFF740B9647400206F
:104B100083BA0608B873002068BB06082DE9F04F79
:104B200091B0174607900C461546002604F115096A
:104B30000DF1240B0422494658464BF0FFFF002399
:104B40008DF82830D4E90232082B72F100010DF102
:104B50002C0A55D22F491A465046F8F7EFFE002F7F
:104B600056D095F80080237843454ED1D4E902020F
:104B7000D5E902139A4208BF884246D1227D2B7D97
:104B80009A4242D1042205F1150148464BF08AFFB2
:104B900000283AD121692B69CB1AD3F1000949EBDE
:104BA00003091D4B059300230493B5F912300393B9
:104BB000B5F910300293194B194A0798CDE90083D3
:104BC00049463346FEF7FEFECDF814B0237D04932C
:104BD000B4F912300393B4F91030114A0798CDE9B3
:104BE00001A314F8203B0093494633460136FEF7F3
:104BF000CFFE082E05F1200598D111B0BDE8F08F49
:104C000008495046F8F79AFEA9E74FF00009C8E7AF
:104C1000B946D9E794EF06087CD90608C9F9060811
:104C20007BBB060870BB06082DE9F74F0446FFF76B
:104C3000B5F8074630B16E490022012003B0BDE847
:104C4000F04F6BE76B492046F9F712F8014638B987
:104C500067484FF4807203B0BDE8F04F4BF07AB86C
:104C60002046F9F739FC83B2072B054600F2B880DD
:104C70002046FAF7EDFC824600284CD0F9F72CFCD0
:104C800001240FFA80F95046FAF7E2FC68B14FF0C0
:104C90000008411E00F1100C464611F8013F13F0C8
:104CA000DF0F3BD101270134E4B2FAF7D1FC824691
:104CB00000284CD0F9F710FC01340FFA80FBE4B265
:104CC0005046FAF7C5FC0346002842D00190F9F798
:104CD00003FC0134019B0FFA80FAE4B21846FAF79C
:104CE000B7FC0346002836D00190F9F7F5FB0134F4
:104CF000019B42B2E4B218460192FAF7A9FC019A6C
:104D0000034650B30134E4B2032C28D803B0BDE805
:104D1000F04FFFF737B804468146B4E76145C2D08B
:104D2000A3F13002D2B2092A05D9A3F16102052A02
:104D300007D8573BDAB2360146EA187642EA081835
:104D4000ABE7A3F14102052AADD8373BF2E7834632
:104D5000B6E78246C2E70246CDE7274BD4E71FFA03
:104D600089F10229D2D80BF2262189B2B1F5E16F7F
:104D7000CCD80AF2262189B2B1F5E16FC6D8D4B2F7
:104D8000062CC3D81846019344F082FC0428BDD8F1
:104D9000002FBBD0194A019B2DB202EB451102EB4B
:104DA0004512174D81F8C090C1E93286A1F8D0B004
:104DB000A1F8D2A081F8D440D432591E033311F89F
:104DC000010F2C5C04F00304022C08BF203802F809
:104DD000010F087808B18B42F1D103B0BDE8F08F24
:104DE00008480722394603B0BDE8F04FFEF7CEBFB2
:104DF0007874002083BA06087CD90608B8730020AE
:104E0000A11707089CBB06082DE9F04FDFF8AC900E
:104E100087B0834690460C4616460027B8F1000F2F
:104E200049D0707A617AB6F90AC0B6F90CE096F802
:104E300008A08142D6E900323BD12168994238D19D
:104E40006168914235D1B4F90A10614531D1B4F9A4
:104E50000C1071452DD1257AA5EB0A014D424D412B
:104E6000CDE90032CDE9020CCDE904EA3B464A46E1
:104E700029465846FEF7A6FD237A0593B4F90C306F
:104E80000493B4F90A300393637A0293636801933D
:104E900054F8103B00934A463B4629465846013792
:104EA000FEF776FD112F06F11006B7D107B0BDE869
:104EB000F08F0025D4E74546DEE700BFA9BB060812
:104EC0002DE9F74F0446FEF769FF054630B14E491C
:104ED0000022012003B0BDE8F04F95E74B49204682
:104EE000F8F7C6FE30B94FF0FF3003B0BDE8F04F21
:104EF0003AF0BCBE2046F9F7EFFAC3B2102B834656
:104F000007D943481022294603B0BDE8F04FFEF709
:104F10003DBF2046FAF79CFB0646E8B1F9F7DCFAFC
:104F2000012482463046FAF793FB0646B8B1F9F7FA
:104F3000D3FA01348146E4B23046FAF789FB0646DB
:104F400000285AD0F9F7C8FA0128804609D903B0D9
:104F5000BDE8F04FFEF716BF04468246E2E7814601
:104F6000EAE70134E4B23046FAF772FB064600285D
:104F700045D0F9F7B1FA00F5B473B3F5347F0746BD
:104F8000E5D80134E4B23046FAF762FB0346002864
:104F900037D00190F9F7A0FA00F5B472B2F5347F7A
:104FA0000646D4D80134019BE4B21846FAF750FB08
:104FB000034640B10190F9F78FFA0134051E019BB9
:104FC00018BF0125E4B21846FAF742FB08B10134D4
:104FD000E4B2062CBBD10F4B4FFA8BFB03EB0B1348
:104FE000C3E970A983F8C981A3F8CA71A3F8CC6199
:104FF00083F8C85103B0BDE8F08F8046B3E7074699
:10500000C1E70646D1E700BF7875002083BA0608DD
:10501000C9BB0608B87300202DE9FF47DFF8709080
:10502000804617460D4616464FF0000A77B3337890
:1050300029789942D6E9012026D16968914223D185
:10504000AC68211A4C424C41CDE9012000934A46FC
:10505000534621464046FEF7B5FCAB6802936B68A9
:10506000019315F80C3B00934A46534621464046AF
:105070000AF1010AFEF78CFCBAF1080F06F10C06E2
:10508000D4D104B0BDE8F0870024DDE73C46E4E776
:10509000DABB06082DE9F8430446FEF77FFE054615
:1050A00028B1BDE8F8432D4900220120B4E72C497E
:1050B0002046F8F7DDFD014628B9BDE8F84327484A
:1050C00060224AF047BE2046F9F706FAC3B2072B22
:1050D000064606D929462348BDE8F8430722FEF7CD
:1050E00055BE2046FAF7B4FA074628B3F9F7F4F9A3
:1050F000051E18BF012501243846FAF7A9FA07460C
:10510000E0B1F9F7E9F901348046E4B23846FAF73C
:105110009FFA0746A0B1F9F7DFF901348146E4B2FE
:105120003846FAF795FA08B10134E4B2032C09D0F5
:10513000BDE8F843FEF726BE0446DDE78046E5E716
:105140008146EDE7084B76B20C2202FB0636C6E933
:10515000B58986F8D052BDE8F88300BF8876002074
:1051600083BA0608EFBB0608B87300202DE9F04F9C
:10517000DFF8849091B007468846164600240DF16A
:105180002C0A04EB840508EB050358F805001B798D
:105190000290514602A88DF80C303EF029FF4EB324
:1051A000731970591B790490052204A902A88DF87F
:1051B00014304BF077FC0DF1180BB0FA80F559461E
:1051C00004A86D093EF014FFCDF800B023464A460E
:1051D00029463846FEF7F6FB2346CDF800A04A469E
:1051E000294638460134FEF7D3FB802CC9D111B0D3
:1051F000BDE8F08F3546EFE7FEBB06082DE9F04F1E
:1052000089B00546FEF7CAFD044630B16349002265
:10521000012009B0BDE8F04FA8E72846F9F75CF98E
:105220007F28064600F3B2802846FAF711FAB30049
:105230005A4A039306EB8603D118D450584B0C718D
:10524000CDE901430546A346A146A2462746A0460E
:10525000029B05AA13F8010B029394460023AE4665
:1052600015F8011B19B1884201D00A2B0CD120334B
:105270006B444FF00005884203F80C5C08D009B07D
:10528000BDE8F04FFEF77EBD0CF8011B0133E6E7E9
:1052900008F1FF330EF10105032B31D8DFE803F0ED
:1052A000591B026E4FF0010C12F8011B61B33D480F
:1052B000002310F801EB8E455AD00133082BF8D1AA
:1052C0003948002310F801EB714553D10CFA03F370
:1052D00049EA0309E8E7012112F8013BA3B14E2B8B
:1052E0003CD0452B3CD0532B3CD0572B3CD0552B9E
:1052F0003CD0442BF0D1052301FA03F31F43EBE725
:1053000005A8F9F7E9F8834608F101085FFA88F87B
:10531000B8F1050F9CD10399244B019A31445818D8
:1053200003F54C730B4402F00F0204F00F0444EA3F
:10533000071442EA0B123F1180F8302380F831A3A2
:1053400080F83293DC701F7109B0BDE8F04F2CF08B
:1053500037B905A8F9F7C0F80190D5E70023CBE7E6
:105360000123C9E70223C7E70323C5E70423C3E7F3
:105370009A46A5E70133072BA4D195E705A8F9F7CD
:10538000ABF810280446A8BF0024BDE708487F22D8
:10539000214609B0BDE8F04FFEF7F8BCE8760020E2
:1053A0000C1906081119060819190608B873002007
:1053B000F8BB06082DE9FF47DFF86C9080461746DA
:1053C0000D4616464FF0000A67B333882A889A4282
:1053D00026D16C887288A21A54425441F278029203
:1053E000B2782146CDE90032404653464A46FEF7A0
:1053F000E9FAEB780293AB78019335F8043B00931C
:105400004A465346214640460AF1010AFEF7C0FAD1
:10541000BAF1100F06F10406D6D104B0BDE8F0874A
:105420000024DBE73C46E4E708BC06082DE9F04130
:105430000546FEF7B3FC044628B1BDE8F041244917
:1054400000220120B6E72846F9F746F80F2806465D
:1054500036DC2846FAF7FCF81E4FDFF88480054654
:10546000A0362846F9F738F837F8023B98421FDC97
:10547000012C08EB860311D0022C12D0A3F83003C4
:1054800028462C214BF02DFB054668B10135012340
:1054900001346BB1032CE4D1BDE8F08183F8320311
:1054A000EEE783F83303EBE7A21E53425341EFE7E5
:1054B000094B002243F82620BDE8F041FEF762BC0C
:1054C00021460648BDE8F0410F22FEF75FBC00BF51
:1054D0006879002020190608E8760020F8BB060845
:1054E000B87300202DE9F04FDFF8B49085B0064680
:1054F000884614464FF0000B062303FB0BF505F519
:105500003075002718F805A0002C44D0625DAAEB86
:10551000020041424141CDE900725B464A463046B5
:105520000391FEF74FFA0399CDE9007A5B464A46AC
:1055300030460137FEF72CFA062F05F10105E1D1BF
:105540000BF1010BBBF1060FD6D1DFF854904FF4ED
:10555000397518F805B0A5F5397AF4B1635DABEB90
:10556000030257425741CDE900A34A460623394674
:105570003046FEF727FA0623CDE900AB4A46394606
:105580003046FEF705FA013540F2ED239D42E0D1A9
:1055900005B0BDE8F08F2146C6E72746EBE700BF20
:1055A0001ABC06087FB50346FEF7F8FB044630B187
:1055B00019490022012004B0BDE8704092E7174964
:1055C000164E6A46184649F078FA01AD80B1032CB0
:1055D00003D1FEF7D7FB04B070BDF8F77DFF6A4634
:1055E00045F8040B31460020013449F066FAEDE736
:1055F000032CEED1DDE90145039E29463246E0B297
:105600002CF03EF90028E4D0054833462A462146CE
:10561000FEF708FADFE700BFE8760020DC0D070898
:105620001ABC06082DE9FF47DFF898908046174618
:105630000C4616464FF0000A002F41D0B6F9003054
:10564000B4F90010B6F90220B6F9040096F906C0C4
:10565000994233D1B4F9021091422FD1B4F9041018
:1056600081422BD194F90610A1EB0C0569426941E6
:10567000CDE90032CDE9020C53464A4640460D467C
:10568000FEF7A0F994F906300393B4F904300293BD
:10569000B4F90230019334F9083B00934A4653466B
:1056A000294640460AF1010AFEF772F9BAF1100FD5
:1056B00006F10806C0D104B0BDE8F0870021D7E7A5
:1056C0003D46DFE72EBC060830B585B00546FEF73F
:1056D00065FB044610B32E490022012005B0BDE849
:1056E00030409FE72D2B03D0A3F13002092A4AD87E
:1056F000042C04DD05B0BDE83040FEF743BB28466E
:10570000F8F7EAFE04AB621C03EB440424F80C0C2B
:1057100015F8013F303B092BFAD914462B78002BA2
:10572000E0D1052CE6D1BDF80430BDF904500F2BB3
:10573000E0D8BDF90600A0F5FA739BB2B3F5FA6F95
:10574000D8D8BDF90810A1F5FA739BB2B3F5FA6F7A
:10575000D0D8BDF90A209042CCDC9142CADBBDF919
:105760000C4004F17D039BB2FA2BC3D8094B03EB29
:10577000C503A3F81E06A3F82016A3F8222683F873
:10578000244605B030BD202BB4D101352246C4E7F4
:10579000D6790020B87300202DE9F04F80468FB0F5
:1057A00017460C4616464FF0000A23780793B4F9C3
:1057B000029063782068A2880893237994F905B051
:1057C0000A90ADF82C200993B9F1000F3DD0002FBD
:1057D00040D03068BDF828500C9080B2B288ADF847
:1057E0003420854231787378B6F9022096F804E0C7
:1057F0002ED191452CD1BDF82C50BDF83400281A7B
:1058000045424541CDE901320091CDE903EB124A11
:10581000534629464046FEF7D5F8099B0E4ACDF877
:1058200010B0CDE90293089B0193079B0093294692
:10583000534640460AF1010AFEF7AAF8BAF1200FD2
:1058400004F1060406F10606AFD10FB0BDE8F08FF3
:105850000025D7E73D46E0E743BC0608F0B589B030
:10586000044643F015FF10F0FF020DD13E4B3F49B7
:1058700093F886304FF4C87000FB0311D03101203B
:1058800009B0BDE8F04087E7394905222046F8F71E
:10589000D5F9B0B9344B93F88620344B4FF4C87126
:1058A00001FB0233334A15689488D033062606FB81
:1058B00000F29918013020289D508C80F7D109B052
:1058C000F0BD20462C492C4E01AA49F0F6F84FF0C5
:1058D000FF33079302AD002478B1062C02D1FEF706
:1058E00051FAECE7F8F7F8FD01AA45F8040B314648
:1058F0000020013449F0E1F8EEE7042CEFDD029BD3
:105900001F2BECD8039E0F2EE9D8049D262DE6D838
:10591000059C04F57A72B2F5FA6FE0D80698FF2874
:10592000DDD807994A1C402AD9D80F4A92F8862018
:105930004FF4C8777A43062707FB03220F4B134423
:1059400041F2BC029E5441F2BD029D5441F2BE029E
:105950009C5203F58652107041F2C10208489954D6
:10596000FFF77CFFABE700BFB8730020AC720020EC
:1059700083BA060826190608DC0D0708C062002055
:105980007CD906082DE9F04F9BB091460E900F93FD
:105990000C46154600260F9B5A1C01D0B34266D117
:1059A000A446BCE80F0010AF0FC7DCF800303B6026
:1059B00023790993237C0B9394F911300C93A37CE6
:1059C00094F80C8094F813A00A9207460D93B9F14D
:1059D000000F5AD0AE46BEE80F000DF1540CACE8F3
:1059E0000F00DEF80020149BCCF80020534033F069
:1059F0007F43864695F804B0A96895F80CC0E87C0A
:105A00003FD1099A5A453CD177453AD1E04538D142
:105A10000A9A8A4237D1AAEB0003594259410A9B9C
:105A20001B4A0E98CDF81CA0CDE90583099B039372
:105A30000D9B02930C9B01930B9B009304973346A1
:105A40008B46FDF7BFFF0A9B114A0E98CDF81CA0AC
:105A5000CDE90583099B03930D9B02930C9B019356
:105A60000B9B0093049733465946FDF791FF01368F
:105A7000402E04F1140405F114058CD11BB0BDE8CF
:105A8000F08F0021CBE71946C9E7CB46DBE700BF23
:105A90005ABC06082DE9F0418AB004460D4643F091
:105AA000F7FD10F0FF0010D13F4B93F8642E3AB988
:105AB0004FF0FF333D4901200AB0BDE8F04161E7F6
:105AC0006B1C6DD02B460246F4E73949052220466F
:105AD000F8F7B4F838B935484FF47E710AB0BDE82C
:105AE000F04142F049BF20463249324E6A4648F002
:105AF000E4FF01AD002478B1092C02D1FEF742F990
:105B00004EE0F8F7E9FC6A4645F8040B3146002000
:105B1000013448F0D2FFEEE7092CEFD101993F297B
:105B2000ECD8DDF808E0BEF1010FE7D8DDF80CC0D5
:105B30000CF10103402BE1D8049F342FDED8059EE1
:105B4000072EDBD8069D1C4A05F5742303F5107358
:105B50009342D3D8079C072CD0D8089800F574231B
:105B600003F510739342C9D8099AFF2AC6D8134B7C
:105B70004FF0140808FB013309B2C3F8A806104817
:105B800083F8B0E683F8B1C683F8B27683F8A466EA
:105B9000C3F8A05683F8AC4683F8B326FFF77AFF24
:105BA0000AB0BDE8F08100BFC0620020587A002032
:105BB00083BA0608DC0D070880841E00B873002035
:105BC0007CD906084FF0FF3164E72DE9F04F074616
:105BD00087B016460C4615464FF0000BD4E9009AE4
:105BE000D4F8088066B3A8688045D5E9002125D19E
:105BF000914523D1AAEB010359425941CDE9019ABC
:105C0000104ACDF800805B4638460591FDF7DAFE74
:105C100005990C4ACDF800805B46CDE9019A3846DB
:105C20000BF1010BFDF7B4FEBBF1080F04F10C04FE
:105C300005F10C05D2D107B0BDE8F08F0021DDE7FA
:105C40003146E6E77BBC060870B586B0044643F0F3
:105C50001FFD10F0FF0205D12149012006B0BDE86B
:105C60007040B2E71F4905222046F7F7E7FF38B931
:105C70001B4840F2FF3106B0BDE8704042F07CBEE8
:105C800020461949184E01AA48F017FF02AD00241A
:105C900078B1042C02D1FEF775F81FE0F8F71CFC70
:105CA00001AA45F8040B31460020013448F005FFF5
:105CB000EEE7042CEFD1029A072AECD80B4B0C48E4
:105CC0000C2101FB0233039AC3F8A82B049AC3F8F2
:105CD000A02B059AC3F8A42BFFF7B6FF06B070BD42
:105CE000587F002083BA0608DC0D0708B87300202F
:105CF0007CD906082DE9F04FA1B0174610900C464C
:105D000015460026A646BEE80F000DF1480CACE88B
:105D10000F0023680B939EE80700238A0C93638A85
:105D20000D93A38A0E93E38A94F80480D4F808B004
:105D300094F80CA094F818900F938CE80700002FAB
:105D40005CD0AE46BEE80F000DF1640CACE80F006D
:105D50009EE807008CE8070095F818C029682879A4
:105D6000AB682A7BCC4547D1804545D10B9888420A
:105D700042D1924540D19B453ED1169A1D9B9A42F5
:105D80003AD117991E9BCB1A594259410F9B089340
:105D90000E9B07930D9B06930C9B194A1098CDF808
:105DA0000CA0CDE904B30B9BCDF80090CDE90183A5
:105DB00033461191FDF706FE11990F9B08930E9B38
:105DC00007930D9B06930C9B0D4A1098CDF80CA0E1
:105DD000CDE904B30B9BCDF80090CDE901833346A8
:105DE0000136FDF7D5FD042E04F11C0405F11C0558
:105DF00088D121B0BDE8F08F0021C7E73946DCE744
:105E00008CBC0608034B9A780021101A997018BFB1
:105E1000012070473C74002010B5114B014603F17E
:105E2000180253F8044B41F8044B9342F9D11B88F4
:105E30000B800B4900F11A0351F8044B43F8044B53
:105E40009142F9D111881980054B343053F8041B65
:105E500040F8041B9342F9D11B88038010BD00BF9A
:105E600084330608104A117A537A0B43D17C0B43D2
:105E700051780B4391780B43D1780B4311790B4345
:105E8000917B0B43917E0B4392F823100B4392F8C6
:105E90002F100B4305D192F83D00013818BF0120A7
:105EA00070470120704700BFD8D6002070B5234C42
:105EB00094F84C3005460E4643B1D4E91423904281
:105EC00071EB030324BF002384F84C30E36E1C48BD
:105ED000984710F0010320D080F00203C3F3400381
:105EE00084F84C30D4E918325B1946EB0206C4E959
:105EF0001436012384F88030430744BF012384F81B
:105F00008130D4F88830ED1A002D0FDD012384F89C
:105F10008030012000F0010070BD8207ECD594F8BC
:105F20004C20002AE8D084F84C30E5E794F8803023
:105F3000002BEED194F88100ECE700BFD8D600200A
:105F400030D700202DE9F0438DB0044643F0A0FB8C
:105F500010F0FF0206D13F4901200DB0BDE8F0432B
:105F6000FFF7C8BE3C4905222046F7F767FE38B95F
:105F700038484FF47E710DB0BDE8F04342F0FCBCF0
:105F800020463649354E01AA48F097FD02AD00245F
:105F900078B10A2C02D1FDF7F5FE57E0F8F79CFA2C
:105FA00001AA45F8040B31460020013448F085FD74
:105FB000EEE70A2CEFD1DDF80880B8F1030FEAD83C
:105FC000DDF80CE0BEF1010FE5D8DDF810C0BCF142
:105FD000070FE0D8059F224A07F5742303F51073D5
:105FE0009342D8D8069E072ED5D8079D05F5742371
:105FF00003F510739342CED8089CB4F5004FCAD273
:106000000998B0F5004FC6D20A99B1F5004FC2D237
:106010000B9AB2F5004FBED2124B4FF01C0909FB90
:106020000833A3F8A200104883F8A8E083F894C0CE
:10603000C3F8907083F89C60C3F89850A3F8A04010
:10604000A3F8A410A3F8A620FFF77CFF0DB0BDE8CD
:10605000F08300BF68D7002083BA0608DC0D07086C
:1060600080841E00D8D600207CD9060870B505466D
:1060700008460E4643F00CFB3146044602462846CD
:10608000F7F7DCFD60B92B5DA3F13002092A06D9D0
:1060900023F02003413B192B01D90134281970BD8D
:1060A0000020FCE72DE9F04FDFF864A0DFF864B0D2
:1060B00085B00646894615461F460024002F01DBA1
:1060C000A7421CD119F80480FDB12B5DA8EB030297
:1060D0000AEB83035142DB690093514123465A4640
:1060E00030460391FDF76EFC03990AEB88085A4687
:1060F000D8F81C30009330462346FDF749FC0134A4
:106100000E2CDBD105B0BDE8F08F2946EDE700BFCE
:1061100084330608C7BE06082DE9F04FA1B0CDE9CB
:106120000C011546002414AE0D9A02EB44126301D3
:106130000DF1400C02F1200E10685168674603C74C
:1061400008327245BC46F7D1002D00F081802B4407
:1061500018AF03F1200C186859683A4603C2083397
:1061600063451746F7D19DF840300B939DF86010BA
:106170000B98BDF842709DF84480BDF846909DF89C
:1061800048A0BDF84AB09DF84C30BDF84E20814281
:106190005CD1BDF86210B94258D19DF864104145F8
:1061A00054D1BDF86610494550D19DF8681051454D
:1061B0004CD1BDF86A10594548D19DF86C109942F0
:1061C00044D1BDF86E10914240D11CA914A8CDE96C
:1061D0000E3243F0FDF9DDE90E32B0FA80F14909E3
:1061E000CDE905B30B9B0093CDE90726CDE9039AD2
:1061F000CDE90178174A0C980B912346FDF7E2FB95
:106200000B99BDF84E3007939DF84C300693BDF8BE
:106210004A3005939DF848300493BDF84630039307
:106220009DF844300293BDF8423001939DF8403010
:106230000093084A0C98089623460134FDF7A8FB02
:10624000032C7FF471AF21B0BDE8F08F0021C7E7C8
:106250002946D6E7DFBE06082DE9F04190B0044696
:1062600043F016FA10F0FF0205D14549012010B0A5
:10627000BDE8F04150E74349434F01AA204648F0AA
:106280001CFC41496A4648F018FC06AE002435461D
:1062900000286ED0092C61D13A4901AA002048F0AB
:1062A0000CFC0646002869D043F0F2F9044638B1E8
:1062B0000F2828BF0F242246314602A848F028FCA8
:1062C00004F14003DDF818800DEB0304B8F1020F70
:1062D0004FF0000304F8383C4DD8DDF81CE0BEF167
:1062E000070F48D8DDF820C0BCF1FF0F43D8099F45
:1062F000072F40D80A9EFF2E3DD80B9C072C3AD87A
:106300000C98FF2837D80D99022934D80E9AFF2A05
:1063100031D81E4B03EB481303F5887303F8084C80
:1063200003F810EC23F80ECC03F80C7C23F80A6C6D
:1063300023F8060C03F8041C23F8022C02AC2246B6
:1063400003CAAA4218605960144603F10803F6D143
:106350000F48FFF781FF10B0BDE8F081F8F7BCF8F7
:106360006A4646F8040B39460020013448F0A5FB84
:106370008EE7092C90D0FDF705FDECE704469FE77A
:10638000D8D7002079DA0608DC0D0708D8D6002017
:106390007CD90608F8B50C4C0C4E0D4F33252068FF
:1063A000FDF77CFA616811B13046FDF721FBA16869
:1063B00011B13846FDF71CFBFDF79EFA013D04F1D3
:1063C0001004ECD1F8BD00BFB033060806DB0608A8
:1063D00013BF060830B5274885B0FDF75FFAF5F71B
:1063E000C3F928B9244805B0BDE83040FDF7AABA82
:1063F000F5F7A4FC08B92148F5E7F5F7A9FC026810
:10640000037D81790446407C0290207C0190608A63
:10641000009052081A48FDF7EBFAE51D0C3415F808
:10642000010BFDF7C7FAA542F9D1164C1648FDF746
:1064300035FA6378022B06D007D9032B10D1134805
:10644000FDF72CFA0CE01248FAE704F580541148E5
:10645000FDF724FA94F8B431022B06D0032B06D0B2
:1064600005B0BDE83040FDF747BA0B48E8E70B48F8
:10647000E6E700BF19BF060823BF060831BF0608BC
:1064800040BF06089C5000206EBF06087EBF06086D
:1064900084BF060891BF060897BF0608B0BF06086C
:1064A0002DE9F3473549DFF8D49001AA48F005FB00
:1064B0004FF0000A4FF0FF35564654465746A8465F
:1064C00078B9BAF1040F3DD0BAF1050F44D0BAF152
:1064D000030F13D02A492B46424601203DF0BEFE51
:1064E0000EE0BAF1040F09D8DFE80AF0030D121725
:1064F0001C00F7F7F1FF804603281BD9FDF742FC8B
:1065000002B0BDE8F087F7F7E7FF05469528F4E706
:10651000F7F7E2FF07463F28EFE7F7F7DDFF04460E
:106520003F28EAE70378482B03D0562BE6D1012613
:1065300000E0002601AA494600200AF1010A48F0BD
:10654000BCFABDE70F4B962202FB085203EB420355
:10655000B3F86061C6F34036962303FB0855A401E7
:10656000084B04F47C6407F03F0703EB45033C430E
:1065700044EA4634A3F86041C2E700BFDC0D0708D7
:1065800038D80020D8D600202DE9F3412249DFF881
:10659000888001AA48F091FA002504462F464FF062
:1065A000FF366CB9022F0BBF1C491C498D55334671
:1065B00012BF2246334622460120FFF773FD04E056
:1065C00037B1012F12D0FDF7DDFB02B0BDE8F0813D
:1065D0002046F7F781FF0D280646F4D801AA414668
:1065E000002048F06AFA01370446DAE70C482146F1
:1065F000F7F73EFB05460028F0D00A482146F7F79A
:1066000037FB38B108482146F7F732FB0028DAD1CA
:106610000225E3E73D46E1E7DC0D07087C6F00203B
:10662000C2BF0608EDD806086B0207082DE9F04F37
:106630002DED028B4D484E4D9FED4E8A8BB0FDF7F0
:10664000F1F90027B946BA464B4B4C4A196800236A
:106650008B4227DB01371A2F05F14805F4D1484951
:10666000484BD1E90021520942EAC1624649186803
:1066700009684FF47A73B0FBF3F34448FDF7D2F99D
:106680000A2299FBF2F302FB139000909AFBF2F1BD
:106690003F4802FB11A2FDF7C5F90BB0BDEC028B20
:1066A000BDE8F08F52F8040BA84201D00133CFE7C8
:1066B000AC6A4CB107EE904AB8EEE77AC8EE077ABA
:1066C000FDEEE77A17EE904AAB6B0893D5E90C63C1
:1066D0007609E96B46EAC3665B090993089B4FEAB2
:1066E000E47B6143A4FB030C03FB0B1141F28833F1
:1066F000C01841EB0C014FF47A72002343F00AFEFC
:10670000099A804604FB02F1A4FB060C41F288338F
:10671000C01806FB0B1141EB0C014FF47A720023F9
:1067200043F0F8FD2B6C0196042F4FF47A72B3FB03
:10673000F2F306934FF00A0318BF814490FBF3F283
:1067400003FB1200CDE9042098FBF3F203FB128354
:10675000CDE90223089B00932A680E482346394658
:1067600018BFC244FDF75EF974E700BFC7BF060853
:106770001009002000247449205701208056012070
:10678000EC560120F4560120FC56012043C00608B7
:1067900065C006080EC006081FB5094B0293094BD9
:1067A0000193094B0093094A094B0A490A48FDF72E
:1067B00039F90A490A4805B05DF804EBFDF732B92A
:1067C000B1C00608BAC00608C3C00608A0B40608CF
:1067D00093C00608AFB4060899C00608CFC00608E3
:1067E000DFC00608F8B50C480C4E0D4F0D4DFDF7F7
:1067F00019F90D4B1A68C2F500729200002422B1FB
:1068000056F824103846FDF70DF90134222C02D039
:1068100055F82420F3E7F8BDE8C00608E03606087E
:10682000FEC00608483E0020443600202DE9F84FFF
:10683000054642F02DFFDFF8EC800446D8F80090C2
:10684000C0B93048304D314FFDF728F8012655F8D2
:10685000041B59B10B783BB106FA04F313EA090F94
:1068600002D03846FDF7C4F80134F0E7BDE8F84F30
:10687000FDF742B8024626492846F7F7DFF978B90E
:106880002448214C214DFDF709F854F8041B002938
:10689000ECD00B78002BF8D02846FDF7A9F8F4E7E8
:1068A0002B78DFF864B02D2B03BF013504F1FF34E2
:1068B0004FF0010A4FF0000A00265BF8047B1FB975
:1068C000BDE8F84F3DF028BC224639462846F7F788
:1068D000B5F9A8B90120B040BAF1000F0AD0F7F716
:1068E00051FF0D48FCF7DAFF39460C48BDE8F84F78
:1068F000FDF798B840EA0900C8F800000848F1E739
:106900000136DAE70CC1060868370608B91107082E
:1069100011D0060816C1060822C1060845C106089E
:106920002BC10608784000202DE9F84F054642F0BB
:10693000AFFEDFF8F4800446D8F81866C8B93148CD
:10694000314DDFF8D480FCF7A9FF0127E3B205EB56
:106950008302D2F8681441B107FA03F3334202D03C
:106960004046FDF745F80134F0E7BDE8F84FFCF785
:10697000C3BF024625492846F7F760F960B92448A5
:10698000244C254DFCF78AFF54F8041B0029ECD059
:106990002846FDF72DF8F7E72B78DFF878B02D2B98
:1069A00003BF013504F1FF344FF0010A4FF0000A34
:1069B0004FF000095BF8047B1FB9BDE8F84F3DF0CC
:1069C000ABBB224639462846F7F738F9B8B9012358
:1069D00003FA09F3BAF1000F0CD026EA03030F48BB
:1069E000C8F81836FCF75AFF39460D48BDE8F84F8D
:1069F000FDF718B833430B48C8F81836F2E709F129
:106A00000109D7E70CC106088433060811D006082F
:106A100016C10608EC370608B911070822C1060896
:106A200045C106082BC10608D8D600202DE9F0473D
:106A3000814642F02DFE494E0446376800BB484867
:106A4000484D494EFCF7D4FF4FF00C0808FB04F307
:106A50005A5D0123013A93403B4206D020461CF088
:106A600039F801463046FCF7C3FF0134182CEDD14C
:106A700017B93E48FCF712FFBDE8F047FCF73CBFF2
:106A800002463B494846F7F7D9F8054678B93948F0
:106A9000FCF704FF2C46344D20461CF01BF8013453
:106AA00001462846FCF7A4FF1A2CF5D1E4E799F833
:106AB00000302D2B03BF09F1010904F1FF344FF021
:106AC000010A4FF0000A002528461CF003F8224670
:106AD000804601464846F7F7B1F8002836D1BAF1AA
:106AE000000F1CD0182D17D0192D0AD17368224819
:106AF0003360FCF7D3FE41462048BDE8F047FCF781
:106B000091BF1F4B0C2202FB053393F8A0240123F5
:106B1000013A93403B43EAE76FF07F43E7E7182DE4
:106B200003D1C6F800A01748E3E7192D01D177601B
:106B3000F9E7134B0C2202FB053393F8A024012341
:106B4000013A934027EA03033360ECE701351A2D3D
:106B5000BAD1BDE8F0473DF0DFBA00BFB46F002006
:106B600033C106082438060844C106083DC106089A
:106B700011D0060849C1060822C1060845C1060809
:106B8000843306082BC106082DE9F341044642F080
:106B90007FFD04283DD1661E2546E71C16F8010F2F
:106BA000F7F746F8BE423070F8D1DFF87880271D3D
:106BB00015F8016B4046314649F093FF20B131464C
:106BC000284649F08EFF20B102B0BDE8F041FDF744
:106BD000D9B8BD42ECD1204621F026F80F48FCF789
:106BE0005DFE0F490F48002311F8012F10F8014BEB
:106BF00008326A440133042B02F8084CF4D1002314
:106C000009488DF804306946FCF70CFF02B0BDE876
:106C1000F0810028E2D0FDF7B5F8DFE754C106089F
:106C2000F4DC00205C39060816BF060808B50446E7
:106C30000648FCF733FE064B1868F8F7C3FD054B12
:106C400018681CF00FFC204606F030FF5AC10608F9
:106C50002071002028710020034808B5FCF71EFEB3
:106C60000120FFF7E3FF00BF66C106087FB5154BA3
:106C700093F81C26012A21D193F821360A2B05D03E
:106C8000114807B05DF804EBFCF708BE0E220021A6
:106C90000DF1070049F05EF80C4B00930C4B1B788C
:106CA0008DF80430B2238DF8053068460323152192
:106CB0008DF8063021F0F2F90648E2E707B05DF8FA
:106CC00004FB00BFD8D600207FC10608A64115EB03
:106CD0002C1100208EC1060808B50A48FCF732FEC8
:106CE000094B1868F8F76EFD084B002483F83E4600
:106CF000C3F8804683F8844613F0FAFC2046FFF779
:106D000095FF00BFA8C1060820710020D8D600203A
:106D100008B5214B214C1D68D4F890061CF0A2FB4D
:106D200028461CF09FFBD4F8900641798B0704D4C9
:106D3000036841F002019B69984700210846F9F772
:106D400071FA00210120F9F76DFAD4F89006FAF7EC
:106D500006F978B101210020F9F764FAD4F8900619
:106D6000FAF71EF901462846FAF7F6F80021084618
:106D7000F9F758FA2846FAF7F2F80028E5D0012189
:106D80000846F9F74FFA2846FAF70AF90146D4F807
:106D90009006FAF7E1F8D4E728710020D8D6002051
:106DA000F7B50546FCF7FAFF044620B103B0BDE88D
:106DB000F040FCF7E7BF28461E491E4F01AA47F0E6
:106DC0007CFE2646254640B90B2D18D901461A48A7
:106DD0000B22FCF7DBFF03B0F0BD44B1012C0AD05D
:106DE00001AA39460020013447F067FEEBE7F7F7C8
:106DF00073FB0546F4E7F7F76FFB0646F0E7022C56
:106E00000ED1A6F57A73B3F57A7F05D90B484FF406
:106E1000FA624FF47A71DCE7094B03EB45039E807D
:106E2000074B084803EB45032946B3F90420FCF758
:106E3000F9FDD0E7DC0D0708F8BB0608FFDB060804
:106E400020570120D2C1060870B50446FCF7A6FF02
:106E5000C0B11F4B5E68013630461BF03BFE344626
:106E60000546E8B901341A2CA8BF002420461BF0BF
:106E700031FE0546A0B9B442F4D1BDE870401548D2
:106E8000FCF760BD2046F7F727FB04461BF022FE07
:106E9000054628B921461048BDE87040FCF7C2BD40
:106EA0000B4B5C601CF08EFD2A460C482146FCF71B
:106EB000B9FD192C9DBF0A4B0C2202FB04330020A4
:106EC000BDE8704098BF93F8A0041CF093BD00BFCC
:106ED0002C110020DFC10608F3C1060809C206080C
:106EE0008433060838B517490522044649F006FEE2
:106EF00058B9154A13781BB901211170134A137040
:106F0000BDE838401248FCF71DBD12490322204657
:106F100049F0F4FD80B90C4D0C4C2B7843B123782B
:106F200033B10D48FCF78BFD00232B70237038BD67
:106F30000A48FCF707FDF7E7BDE838400848FCF7CA
:106F40007EBD00BF7CC8060824710020257100208A
:106F50001EC20608C3CA060834C206086BC2060869
:106F60007FC2060838B50E4D2B7863B10D4C2378DF
:106F70004BB10D48FCF763FD0C48FCF760FD0023A6
:106F80002B70237038BD0A48FCF788FC20F030FED7
:106F9000F7F704FB20F036FE0020FFF747FE00BFA6
:106FA000247100202571002034C206088EC2060814
:106FB000ACC206082DE9F0478CB0074610F8013B3B
:106FC000202BFAD000251F4CDFF88080DFF880905E
:106FD000DFF880A02E466946204611F0C7FF3946EB
:106FE000684649F0CEFDE0B169464046FCF700FD39
:106FF0004946684642F0ECFAF8B9204612F09CF88F
:10700000114B01460078202814BF50461846FCF763
:10701000EFFCFCF771FC2046FCF761FEFCF76CFC12
:1070200001360135B5F5197F04F10B04D3D10EB942
:107030003DF072F80CB0BDE8F08700212046FCF767
:1070400043FEE6E7321906080EBF060838B90608FF
:10705000B315070816BF06082DE9F04F2DED028B7A
:107060008DB00578202D064600F10100F9D030469C
:1070700042F00EFB044618B1012820D12A2D1ED162
:107080009248934D934FFCF75DFC002628466946D5
:1070900011F06CFF69463846FCF7AAFC0136284619
:1070A0002146FCF711FEFCF727FCB6F5197F05F128
:1070B0000B05EBD10DB0BDEC028BBDE8F08F3D218F
:1070C000304649F00EFD002800F0F980034699464D
:1070D00013F8012D202AFAD0A9EB060901308046C9
:1070E000074610F8013B202BF9D0794D4FF0000AEC
:1070F0005FFA89F96946284611F038FF684642F080
:10710000C7FA6946024683463046F6F797FD704B4C
:10711000044658B9CB4509D10B2202FB0A339B79AF
:1071200003F00706062E39D13E4612E00AF1010AA5
:10713000BAF5197F05F10B05DCD13CF0EDFFB9E79D
:1071400016F8013BA3F16102192A02D8203B06F888
:10715000013C404642F09CFAF31B83420446EFD3C5
:107160005D49684642F034FA20B15C49684642F015
:107170002FFA80B998F80030222B0CD108EB0403C9
:1071800013F8013C222B06D1A21E08F1010128466A
:1071900012F090F88EE722464146F8E713F0C0035C
:1071A0000AD0402B5BD04E48FCF7D2FB2846FCF7B8
:1071B00096FDFCF7A1FB7DE798F80030002BF2D09C
:1071C0004849404649F0CDFC0446404642F060FA4A
:1071D0008442E8D14046F7F7F3F82846B0EE408AFB
:1071E00011F0B6FF07EE900AF8EEE77AF4EEC87AEF
:1071F000F1EE10FAD7D8284611F0BAFF07EE900A40
:10720000F8EE677AF4EEC87AF1EE10FACBDB052ED1
:107210000BD118EE104A284611F08EFF052E3FD8EC
:10722000DFE806F03D3D4747494B042E12D13A4670
:1072300017F8013B202BFAD0092BF8D0013A002493
:107240000A2112F8013F303BDBB2092BE3D801FBE6
:107250000434F6E74046F7F73FF90446DBE72846F3
:1072600012F00CF890F804B0814627462346A24657
:10727000BB4500D91BB1BAF1000F94D0CBE7D9F8C8
:107280000030414653F82700F6F7F2FC002805BF0E
:107290003C46012300234FF0010A0137E8E7047060
:1072A00069461148FCF7A4FB00212846FCF70CFDB9
:1072B00000E70480F4E70460F2E70460F0E730469A
:1072C0000DB0BDEC028BBDE8F04F73E6B3C206080B
:1072D0003219060838B90608B3150708C5C20608EA
:1072E000E9C20608D0C20608DEC206082DE9F04F42
:1072F000A3B0BF4B0293BF4B0193BF4BBF4AC049E2
:10730000C0480093C04BC14CC14DC24FFCF78AFB33
:10731000C149C248FCF786FBC14BC24819684FF40B
:107320007A73B1FBF3F1FCF77DFB06A8F6F798FD45
:1073300006A916A841F02CFB16A9BB48FCF772FB66
:1073400021F016FB6423B0FBF3F103FB110094F86A
:10735000BD3605EB830382B2D3F8E035009394F891
:10736000BC36B24889B2FCF75DFBB14BB148196835
:10737000B14BB1FBF3F1FCF73BFBD7F81C800026C7
:1073800005F5BE6904F2BE6A05F20C6B0123B34039
:1073900013EA080F0BD059F8263043B11AF806202B
:1073A0005BF8261053F82220A448FCF721FB013695
:1073B000072EEBD1FCF7A0FAA1489F4EFCF7C2FACA
:1073C00009A8F3F7ECF809999E48B1FBF6F1FCF730
:1073D00029FB0A999C48B1FBF6F1FCF723FB0B99BA
:1073E0009A48B1FBF6F1FCF71DFB0C999848B1FBEC
:1073F000F6F1FCF717FB21F0C7FC05EB8000D0F895
:107400003416059121F0CAFC05EB8000D0F83486D3
:1074100021F0D4FC05EB8000D0F8349621F0F2FC8A
:1074200005EB8000D0F834A621F010FD05EB8000BC
:10743000D0F834B621F058FD05EB8000D0F8346662
:1074400021F038FD05EB8000CDE900ABD0F83436F3
:1074500005998048CDE9026342464B46FCF7E2FAC3
:107460007D4B1B68DB031CD57C4B93F80080B8F187
:10747000000F16D07A48DFF84892DFF848A241465C
:10748000FCF7D0FA0026B9F9022031465046013601
:10749000FCF7AEFAF3B2984509F11009F3D8FCF7FE
:1074A0002BFA0020FEF796FF6E4B6F4A1E886F4B3B
:1074B0006F491B686F48DFF810A2DFF81092DFF801
:1074C0001082DFF810B2C3F500739B00FCF7AAFA34
:1074D000694A6A4B6A48D31A6A4AB6B23146128878
:1074E000FCF7A0FA6848FCF72DFA04265AF8041BAA
:1074F0006648FCF77DFA6648FCF7D0F919F8011BDD
:10750000002940F095816348FCF7C8F96248FCF710
:10751000C5F958F8041B002940F08E815D48FCF73E
:1075200011FA013EE2D1398C5C48FCF761FA5C4902
:107530000A6F5AB107EE902ADFED5A6AF8EEE77A41
:1075400086EEA77AFDEEC77A17EE902AD1F80031C1
:107550005BB107EE903ADFED536AF8EEE77A86EE1C
:10756000A77AFDEEC77A17EE903A896A59B107EE0D
:10757000901ADFED4C6AF8EEE77A86EEA77AFDEE18
:10758000C77A17EE901A0091B4F8CC164648474FC8
:10759000DFF84491FCF746FA4548FCF77FF93E686E
:1075A00026F0004626F07F064FF00108002E40F03E
:1075B0004781FCF7A1F93B685F0113D50DA811F0D5
:1075C000EFFD78B90D9BB3F5197F3DBF39480B220C
:1075D00002FB0300304616A911F0C8FC364816A974
:1075E000FCF72DFA3548FCF759F9D4F8D01675E0B8
:1075F000B1C00608BAC00608C3C00608A0B4060891
:10760000AFB406089BC0060893C00608D8D6002071
:107610008433060820570120CFC00608E1C00608C1
:10762000542B00202CC3060846C3060857C306087F
:10763000000100207CC3060840420F008CC30608EE
:1076400094C30608A9C30608BBC30608CDC3060831
:10765000DFC30608F1C306081457012010570120A4
:1076600044C40608203000200000022044360020D8
:107670000018000078C406080080000800400008D8
:10768000B0C4060874400020EAC40608FDC4060819
:1076900005C506083FC106081BC5060825C506081E
:1076A000100900200024744935C5060878560120C9
:1076B00072C506083219060889C506089DC5060860
:1076C0009C3F002069C40608C83906089DDD0020DB
:1076D0006864002014C5060845C10608002900F0AA
:1076E000C2800B7B4A7B6D488968FCF781F9FCF707
:1076F00003F96B48FCF7D2F8D4F8D406FCF769F824
:10770000002800F0B4800DA9D4F8D406FCF7A9F83D
:107710009DF848109DF85430149A6248FCF768F9B7
:10772000119911B16048FCF763F90F9911B15F48E5
:10773000FCF75EF9FCF7E0F85D4B1B6818066AD5AC
:1077400094F8D836012B66D85A48FCF7A7F8D4F835
:107750009436B3F5487F00F0988000F28C80B3F542
:10776000167F00F09480B3F52F7F00F0928052498D
:10777000524AB3F5FA7F08BF114694F89B0694F875
:10778000993694F89826072896BF05EB80000020CC
:10779000D0F8B40600904A48FCF72AF9FCF7ACF898
:1077A0004848FCF73FF94848FCF7CCF84748FCF755
:1077B000C9F894F8E43619070AD594F8EC2694F839
:1077C000ED164348C2F3C002C1F3C001FCF72AF929
:1077D00094F8E4365A070AD594F8EC2694F8ED1696
:1077E0003C48C2F38002C1F38001FCF71BF994F816
:1077F000E4369B070AD594F8EC2694F8ED16364843
:10780000C2F34002C1F34001FCF70CF994F8E8160A
:107810003248FCF707F9324B1B7833B105EB83058F
:107820003048D5F8D416FCF7FDF823B0BDE8F08F4A
:107830005846FCF7DDF869E65846FCF7F3F870E6C1
:1078400096FAA6F3B3FA83F308FA03F2062B26EAB4
:1078500002067FF7ABAE05EB83034846D3F8381634
:10786000FCF7C6F8A2E62048FCF718F83FE71F48E7
:10787000FCF714F85EE7B3F5617F0CD00E491C4AA3
:10788000B3F57A7F08BF114677E71A4975E71A49B9
:1078900073E71A4971E71A496FE700BFA3C50608E5
:1078A000BCC50608C2C50608E0C50608E9C5060845
:1078B0007840002005C6060824C30608F9C2060859
:1078C0000BC6060832C6060847C6060868C606087C
:1078D00074C6060886C6060897C60608A9C606081E
:1078E0008A6F0020C0C60608B0C50608F8C506089D
:1078F0001CC306080EC3060800C3060807C3060813
:1079000015C306082DE9F3411A481B4C1B4E1C4FAA
:10791000DFF87080FCF786F80025E2792168A3790A
:1079200094F808C006EB820201F13F41D2F8EC0660
:10793000A28806EB830301F57E01890AB2FA82F27E
:10794000D3F85C334131C2F11F02BCF1000F0CD0FF
:10795000CDE900C04046FCF765F80135312D04F152
:107960000C04DAD102B0BDE8F08100903846FCF793
:1079700059F8F2E7DAC606087C640020843306086A
:1079800006C70608F6C6060810B5F4F7CEF9124C7D
:10799000D0B11248FBF7F0FF1148FBF77FFF2068DA
:1079A000F7F710FF4FF47A70FBF754FA0D4B186895
:1079B0001BF058FD0C4B1878F9F702F80221012052
:1079C000F3F7E8FAF9F742FB0848FBF767FF20688E
:1079D000BDE81040F7F7F6BE2071002014C7060876
:1079E0005AC10608287100201057012034C7060824
:1079F0002DE9F0410446254E254DDFF8B0800020EA
:107A0000FEF700FA2348FBF7B7FFB17822480131AF
:107A1000FCF708F821462020FCF7ACF81F48FBF7DC
:107A2000ABFFB3781E4A4FF4C87707FB0353D3ED7F
:107A3000047AF5EE407AF1EE10FA0CBF0121002134
:107A40002046FBF7A5FFB1787943103108EB01021E
:107A500020462944FCF79CFE1248FBF78DFFB378C3
:107A6000114A07FB03532046B3F9D210B1FA81F152
:107A70004909FBF78DFFB1787943D03108EB01025A
:107A800020462944BDE8F041FDF786BE3C74002045
:107A9000088B002063C7060871C7060884C706085C
:107AA00097C70608A6C70608B9C70608AC72002023
:107AB000A0F2DC50164BB0F5FA7FA8BF4FF4FA7075
:107AC000984210B5B8BF18460C4611463CF02FFC42
:107AD00000B207EE900A9FED0F7AF8EEE77AE4B273
:107AE00087EE870AFBEE096AE0EE006A07EE904A2D
:107AF0009FED097AF8EE677AA7EEA67AF3EE097A97
:107B000020EE070A80EE270A43F054FA00B210BDB7
:107B10000CFEFFFF0000C84200401C452DE9F84F55
:107B2000844D95F8F5062DED028BB0EE408A78B3C2
:107B3000814E824F00244FF0060805F5DE6995F866
:107B40001C3708FB0373234493F86A3753B1012BA6
:107B50000DD00134042C06F10206F0D1BDEC028BED
:107B6000BDE8F88F09EB44031B8E3380F1E7032C4B
:107B700001D00023F9E7724B1B68DB0405D412F037
:107B80003BFD00B26F4B5885E3E740F2DC50F9E76C
:107B90006C4C20F069F8D4F82CA0D5F8287795F82B
:107BA0002C871AF4807B14BF7E7B3E7A4246314696
:107BB000FFF77EFFA0848146012020F055F8424661
:107BC0003146FFF775FF8046E084022020F04CF834
:107BD000BBF1000F77D0B97B95F82D27FFF768FF31
:107BE000464236B22685BBF1000F6ED0FB7B642285
:107BF00013FB09F393FBF2F3A3843B7C13FB08F321
:107C000093FBF2F3E3847B7C13FB06F393FBF2F329
:107C1000238510F00BFF95F8F436608543B9B4F96D
:107C20002830626AC5F82027A5F82437A5F826076A
:107C30001AF0400F92D0B4F9343007EE903AF8EED3
:107C4000E77AB2EE047A87EE878AB5F95C3707EEF9
:107C5000903AF8EEE77A38EE678ADFED3B7ABDEED0
:107C6000C88A18EE103A1BB208EE103AB8EEC88A6D
:107C700028EE278AB0EE480AF5F7D8F9F0EE408AE8
:107C8000B0EE480AF5F770F9B4F9263006EE903AEE
:107C9000B4F9243007EE103AF8EEE66AB8EEC77A87
:107CA00067EE007A20EE660AE6EEA87AA7EE280ACA
:107CB000FDEEE77ABDEEC00A10EE103AA38417EE8F
:107CC000903AE3844AE7797A86E795F83877B0EE18
:107CD000480A122F4FF00001484608BFC5F83C97EC
:107CE00012F0E0FB122F00B208BFC5F84007A084D5
:107CF000B0EE480A4FF00101404608BFC5F844877E
:107D000012F0D0FB122F00B208BFC5F84807E0847C
:107D1000B0EE480A4FF00201304608BFC5F84C6784
:107D200012F0C0FB122F00B2208508BFC5F8500723
:107D30006FE700BFD8D600204457012084330608DF
:107D4000185701202057012035FA8E3C2DE9F043C9
:107D5000DFF8F891774CD9F80030D3F82880764BCB
:107D60001B6813F0100F87B040F0A68094F83830ED
:107D7000002B00F0A180714E06F5EC65D6F868374F
:107D800028469847002800F0978096F8C537002BC2
:107D900043D1022384F85830B6F9C63707EE903A3B
:107DA000B6F9C837F8EEE77AC5ED0A7A07EE903AE9
:107DB000B6F9CA37F8EEE77AC5ED0B7A07EE903AD6
:107DC000F8EEE77AC5ED0C7A5D4903AAA1F10C0043
:107DD0003DF010FC03A996F8A427084620F07AFF8E
:107DE00003A820F039FF95ED060A5649554D03A822
:107DF0003DF00DFC05F178070026B5EC010AD4F83A
:107E0000243185ED020A384698470136032E05EDE8
:107E1000010A07F12407F0D14EE094F85830012B05
:107E2000D2D1EB6903932B6A049303A96B6A059380
:107E300004F15800F5F702FC94F85830012B4FF08C
:107E4000000772D0022B67D0039704970597DDEDEA
:107E5000037A9DED047ADDED056AC5ED0A7A85EDBC
:107E60000B7AC5ED0C6AFDEEE77ABDEEC77AFDEE42
:107E7000E66A17EE903A17EE102A16EE901A1BB229
:107E800012B209B2A6F8C637A6F8C827A6F8CA17CC
:107E90000120CDE9002104212B4AF5F765FDD9F831
:107EA000003000200021C3E90C01C3E91001C3E93F
:107EB0000E0127646764A764E3695B0629D51F4D3B
:107EC00095F8F8372BB34FEAE8763146404642F052
:107ED0008BF905F5FA6307EE900AD4ED106A93ED7D
:107EE0000F7AD5F81828D5F81C18A7EEA67A12EB49
:107EF000080246EB0106D4ED116A83ED0F7A93ED8B
:107F0000107AC5F81828A7EEA67AC5F81C6883ED84
:107F1000107A07B0BDE8F083236F0393D4F888305C
:107F20000493D4F8A030059391E7AF62EF622F631A
:107F3000BFE700BF2057012078560120D8D6002087
:107F400060DE002060570120C6C706080C570120DC
:107F5000034B012283F82828022283F8292870473E
:107F6000D8D6002070B50D4E35782D1A18BF0125D2
:107F70000328044634BF044600242046F6F750FC8C
:107F8000074A347002F62A031A2104FB0133C2F8AF
:107F900028371AF043FC284670BD00BF3C7400200F
:107FA000D8D60020022810B50C4618D8FFF7DAFF03
:107FB0000B48FBF7E1FC0B4B0B4819780131FBF741
:107FC00031FD21460820FBF7D5FD21461020FBF7A7
:107FD000D1FD21462820BDE81040FBF7CBBD10BDE8
:107FE00086CF06083C74002077C7060838B5154CC4
:107FF000154DAC4213D30020F6F712FC13481FF0C6
:1080000013FE134A136843F48003136000BF114B3F
:108010001878FFF7A7FFBDE8384029F0D1BAB4F9C6
:108020000230002B4FF00001204607DAF6F7E8FB9C
:1080300001212046F6F7E4FB02212046F6F7E0FB9B
:108040001434D6E7A0190708C81E0708EDC70608AC
:10805000784000203C74002010B504460A48FBF725
:108060001DFCFFF7C3FF1FF0C3FDF6F797FA1FF0E3
:10807000C9FD064B0649002220461A70FDF7F6FF9F
:1080800008B9FEF7D3FD10BDF6C70608257100201C
:10809000B4C8060810B5064B5C78241A18BF012432
:1080A000032828BF0020587020F024FC204610BD73
:1080B0003C740020022810B50C4610D8FFF7EAFFE8
:1080C0000748FBF759FC074B074859780131FBF784
:1080D000A9FC21461820BDE81040FBF74BBD10BDA0
:1080E0000CC806083C7400201CC806082DE9F04F97
:1080F0000D468DB0B6490746FDF7B8FF0646002885
:1081000040F0B780B3493846FDF7B0FF0646002877
:1081100040F0B180B0493846FDF7A8FF0646002878
:1081200040F0AB80AD493846FDF7A0FF0646002879
:1081300040F0A580AA493846FDF798FF002806467A
:108140000ABF012410243E466D4205F020052C4351
:10815000A44DA54F95F800A095F8019095F80280E0
:10816000DFF8F8B25F45C0F08C80FFF73FFF504664
:10817000FFF7F8FE4846FFF78DFF4046FDF742FE49
:108180009A493046FDF772FF08B144F0400414F0FC
:108190001103019300F05D829548FBF7EDFB002091
:1081A000FEF7FAFA9348FBF7E7FB9348FBF7CAFBA5
:1081B00004F03003302B02D19048FBF7DDFB9048F0
:1081C000904FFBF7D9FB9048FBF7D6FB4FF0FF33FE
:1081D0008E4A8F492046FDF765FF8E48FBF7CCFBA2
:1081E0008D4A8E492046FDF71DFA8D48FBF7C4FBEA
:1081F0008C4A8D492046FCF70FFF8C48FBF7BCFBEF
:108200008B4A8C492046FCF7FFFD8B48FBF7B4FBFB
:108210008A4B1E688A4BD3F800908A4B00939B468A
:1082200069EA06034FF0000A02935BF8043B002B57
:1082300034D01A78D2B1029A03934FF0010808FAA9
:108240000AF812EA080F14BF012100213A4620461D
:10825000FBF7B8FB66EA090212EA080F039B3A46ED
:1082600014BF012100212046FBF792FB0AF1010A0D
:10827000DBE7012468E7022466E7042464E70824B6
:1082800062E77B88C3F30B021B04D7E9011048BFE8
:1082900002EB420246F03CFC143763E71F46DFF86E
:1082A000C0A169EA06030293009B53F804BB009344
:1082B000BBF1000F25D09BF8002002B34FF001085E
:1082C00008FA07F819EA080F0BD066EA090212EA61
:1082D000080F5B46524614BF012100212046FBF7E0
:1082E00071FB16EA080F0AD0029B13EA080F5246E8
:1082F0005B4614BF012100212046FBF749FB0137F3
:10830000D2E75148DFF85CA1FBF736FB4F4AD2F8C1
:1083100000804F4A126888EA02025E46D343DFF8C3
:1083200048B10093009B0127B7403B4214BF4FF078
:1083300001094FF0000918EA07070CBF52465A46D8
:10834000304603921AF0C6FB039A02900346494650
:108350002046FBF737FB0136002F0CBF5A4652462A
:10836000029B49462046FBF713FB182EDAD1394809
:10837000DFF8F8A0DFF8F880DFF8F890FBF7FCFAF8
:10838000354BD3F880780026F3B20AEB8302D2F89B
:1083900068B4BBF1000F6FD00121994039405B46B2
:1083A0000CD04A4600212046FBF7F2FA5B464A46CB
:1083B00000212046FBF706FB0136E5E74246204652
:1083C0000091FBF7E5FA00995B464246F1E700BFF2
:1083D00046C8060886CF06080CC8060863C7060804
:1083E0004DC806083C740020A019070851C80608AB
:1083F000AFD306085EC8060876C8060882C8060815
:10840000E1CF0608FAC80608BDC806087C6F002040
:10841000188E0020CDC80608D679002018850020C7
:10842000DDC806088876002088880020E6C806088F
:1084300078750020E888002000CE06087C400020E7
:1084400078400020683706089CCC06080C8E002077
:10845000B46F002011C90608D8D60020C81E07082E
:1084600006C906083BC8060831C806088433060852
:1084700026C906081AC906089848FBF77DFA984AE3
:10848000DFF824C3CDF820B0CDF810B0A2F51A70F3
:108490000426012712F8013F1CF801EB03F130011B
:1084A000694401F820EC10F8011F01F13008E8449C
:1084B00008F810EC002F00F0EF80A3EB010EDEF1C6
:1084C000000141EB0E01013E0F46E3D1854A8DF8D4
:1084D000146008AB2046FBF775FA04AB3946814AB5
:1084E0002046FBF755FA8048FBF746FA7F4A804959
:1084F0002046FBF741FF7F48FBF73EFA7E4A7F4963
:108500002046FCF733FE7E48FBF736FA7D4A7E496B
:108510002046FCF74FFF7D48FBF72EFA764A774955
:108520002046FCF7DFFF7A48FBF726FA794A7A49BA
:108530002046FBF755FE7948FBF71EFA784A794941
:108540002046FCF739F87848FBF716FA774A78495D
:108550002046FCF745FA7748FBF70EFA764A77494A
:108560002046FCF7DBFA7648FBF706FA7549204609
:108570003BF0E8FD7448FBF7FFF94FF0FF331A4674
:10858000724920463BF06AFE7148FBF7F5F94FF05F
:10859000FF33704A70492046FDF7F4F96F48FBF746
:1085A000EBF96F4A6F492046FDF70FFB6E48FBF76A
:1085B000E3F96E4A6E492046FDF79CFB6D48FBF7D8
:1085C000DBF96D4A6D492046FDF7A6FD6C48FBF7C7
:1085D000D3F921463046FBF7CDFAE7065ED52046B3
:1085E00095F800806F7895F80290FFF701FA214620
:1085F0003046FFF7D7FC21460120FFF7D3FC214688
:108600000220FFF7CFFC21463046FFF753FD2146FD
:108610000120FFF74FFD21460220FFF74BFD4046AA
:10862000FFF7A0FC3846FFF735FD4846FDF7EAFBAB
:108630005448FBF7A1F9544809F10101FBF7F2F99D
:10864000524808F10101FBF7EDF95148791CFBF79D
:10865000E9F90026200704D5AB7813B92046FFF7C7
:10866000C7F9A10703D528782146FFF79BFC6207CD
:1086700003D568782146FFF71DFD019B13B14548DE
:10868000FBF77AF92EB14448FBF776F94348FBF73C
:1086900059F9434C434D1CE0394614E7AB7813B904
:1086A0002046FFF7A5F928782146FFF77BFC68787C
:1086B0002146FFF7FFFC0126CCE76388C3F30B02DA
:1086C0001B04D4E9010148BF02EB420246F020FA44
:1086D0001434AC42F1D30DB0BDE8F08F33C90608B5
:1086E0005CDF002049C9060850C906080072002056
:1086F000388D002056C90608E876002098850020AD
:108700005BC90608687900201888002065C906083A
:1087100074C906082D7100206C8D002080C90608E0
:1087200034720020C08C002097C9060864740020B1
:10873000F88A0020A8C9060878740020F88900206B
:10874000B4C9060880DF0020D3C90608E0E800208D
:10875000E4C90608587A002018800020F7C90608E6
:10876000587F0020B87F002015CA060868D700206F
:1087700090ED002032CA0608D8D7002000EE002075
:1087800046C8060847CA06086ACA060870CA060824
:108790007BCA06088ECA0608A7CA0608BDCA06080C
:1087A000A0190708C81E07085C39060800219DE4C7
:1087B00001219BE42DE9F74FBA4CDFF824A3BA4B13
:1087C0009C42C0F05D81B94C2078FFF7CBFB60780C
:1087D000FFF760FCA078B64CFDF714FB94F8A036C8
:1087E00094F8A126B3489A4224BF002384F8A03607
:1087F000F5F7C8FFB04B1A68B04B934312D1002174
:108800002520F1F7F9F9054660B100212720F1F79D
:10881000F3F938B102682B689A4203D14FF48030E3
:10882000F5F7B0FF0026A64F35464FF0FF0848F297
:10883000B83957F826004308810801F0333103F0B6
:1088400077330B44C10801F01131C31A5B1A03EBF3
:10885000131310F0010203F00F33B3FBF8F1C1EB77
:10886000012118BF0135A3EB010318BFEDB2012BA5
:1088700040F27E81022B00F0728191480D2140F080
:108880007BF8B4F8D036B4F8CE26643B9342A8BF48
:108890001346A4F8CE3600BF94F83C3713B908232A
:1088A00084F83C37002010F07BFC864F3B680028A2
:1088B00000F0678123F080633B60834BDFF8248204
:1088C000D3F8286711F098FE804B31781D8883B269
:1088D0002D1A6422009305FB01F393FBF2F313FAC4
:1088E00080F0A4F8520796F80190C1F16E0301EBF5
:1088F000810CA2EB090B9BB24A42C1F1640E4FEA14
:108900004C0C92B201935FFA8EFE4FF00A0A16B237
:10891000002E40F33981704606FB06F310FB00F091
:1089200009FB03F393FBF0F35B44734393FBFAF30C
:1089300063441BB24FF47A706B4393FBF0F30098DF
:10894000034428F8023B0A32019B92B29342DED1E3
:108950001FF0EAFF19F01EFD302200215C4847F0AD
:10896000F9F910F046FA584B93F8F4264ABB93F8FD
:108970003A00C3F800276421C82511FB0050C3F852
:10898000F80693F83B00C3F8042711FB0051C3F825
:10899000FC16C3F8082793F83D10C3F80C27C3F85A
:1089A0001027C3F8142783F81D2783F81E2783F8A0
:1089B000F526C3F820274FF07A7283F81C17C3F806
:1089C00024273B6843499B060A6800F1E180B4F81C
:1089D0009606B4F894360343B4F8980603431BB2E2
:1089E000002B40F0D580B4F99A36B3F5805F40F0A3
:1089F000CF80B4F99C36B3F5805F40F0C980B4F9FC
:108A00009E36B3F5805F40F0C38022F400720A60A6
:108A10001FF0A8FEB4F88427DFED2F7A2F4B07EE66
:108A2000102AB8EEC77AB4F88627C7EE276A07EE91
:108A3000102AB8EEC77AC3ED506AC7EE276AB4F8B9
:108A4000882707EE102AB8EEC77AC3ED516AC7EE41
:108A5000276AB4F88A2707EE102AB8EEC77AC3ED62
:108A6000526AC7EE276A94F88C2783F85021C3ED29
:108A7000536A18F043FE03B0BDE8F04F35F09CBADE
:108A8000B4F90230DFF86080002BA7BF002637461C
:108A90000326012700257919C9B28E4226D2143443
:108AA0008DE600BFA0190708C81E07083C74002007
:108AB000D0E7002020631406784000204000010029
:108AC0000072002078560120D8D60020684000208F
:108AD00024EF00201457012000401C46205701209D
:108AE000014000084858012000800008534603F167
:108AF000060BC3454FD21A88002A4CD003EB020C58
:108B0000C44548D2052A46D92088B3F802E0C0F30C
:108B10000B00864521D1587900F0030088421CD112
:108B20002946204693F804900092F5F769FE2188C3
:108B3000009AB9EB113F0ED161886068C1F30B0355
:108B4000063A9A42A8BF1A46090448BF03FB05002B
:108B5000594645F0DDFF01359DE76346C7E712B191
:108B600010EA090F04D13EF051F900283FF485AE18
:108B700003360C2E7FF45DAE013D022D7FF681AEF3
:108B80007BE643F0806397E60CBF01200846C3E60E
:108B900042F400723BE729462046F5F731FEDAE75A
:108BA00010B5154C94F82938022B18D11FF020F875
:108BB000F5F7F4FCFFF7FEFD1FF024F801201AF092
:108BC00057FF0E4B0E491B6803F59C5300220833D8
:108BD00084F82828C1F8943784F8292810BD012B7F
:108BE000FCD11FF005F8F5F7D9FC1FF00BF80023B6
:108BF00084F82938F2E700BFD8D60020542B002093
:108C0000D0E7002010B50446FFF7ACF938B11EF0EC
:108C1000EFFFF5F7C3FCFFF7CDFD1EF0F3FF601C7F
:108C2000C0B2BDE810401AF023BF38B50C4D044661
:108C30002046FBF7B3F838B10A4B0B481978BDE86A
:108C400038400131FAF7EEBE2046F5F745FC013811
:108C5000022804D8C0B2FFF7D5FF2C46E8E738BD9C
:108C60007CD906083C74002070CA060810B504467A
:108C7000FFF710FA38B11EF0BBFFF5F78FFCFFF7D6
:108C800099FD1EF0BFFF601CC0B2BDE810401AF095
:108C9000EFBE38B50C4D04462046FBF77FF838B1DF
:108CA0000A4B0B485978BDE838400131FAF7BABE93
:108CB0002046F5F711FC0138022804D8C0B2FFF7AE
:108CC000D5FF2C46E8E738BD7CD906083C74002067
:108CD0007BCA060810B50446FDF794F838B11EF0BB
:108CE00087FFF5F75BFCFFF765FD1EF08BFF601C4F
:108CF000C0B2BDE810401AF0BBBE70B50C4E0446C1
:108D00002046FBF74BF8054638B10A4B0A489978DC
:108D1000BDE870400131FAF785BE2046F5F7DCFB6F
:108D2000012804D12846FFF7D5FF3446E8E770BD97
:108D30007CD906083C7400206ACA060838B5144D70
:108D4000EC69630702D538F0B3FEF8B1200703D50C
:108D5000104B1B68D90519D5A20602D538F048FF7B
:108D6000A0B138F061FE10B9FDF77CF868B995F84C
:108D70005431012B04D1A30702D5FDF773F820B9B4
:108D800020F030F980F00100C0B238BD0120FCE7CE
:108D900020570120145701202DE9F8438F4D2C68EE
:108DA00014F0040705D0BDE8F84301210020F7F7CF
:108DB00039BAFFF7C3FF8A4E002800F0B08044F4B0
:108DC00000742C6086F89877864F2C6897F81E37C9
:108DD000012B96F89A3714BF44F4802424F480249D
:108DE0002C603BB90FF0F2FD002800F0A68024F4BF
:108DF00000242C6036F002FD50B197F82F072C6844
:108E00000FF0CCFD002800F09B8044F400042C609F
:108E1000754BDFF8F491D3F800802C68B9F8203056
:108E200018F0080F0CBF44F4807424F48074632B92
:108E30008CBF44F4806424F4806400202C6035F0FE
:108E400011F800287FD044F40064D9F81C301A07C8
:108E50007CD518F4807F79D144F480549B072C6032
:108E600077D518F4007F74D1FCF7FCFF002870D090
:108E700044F400542C6020F04FF800286CD144F4E6
:108E8000004412202C600FF03BFE002867D044F411
:108E9000803417202C600FF033FE002862D044F499
:108EA00000341B202C600FF02BFE00285DD044F016
:108EB00080742C60F9F7F0FED6F8A0374B4AC01A40
:108EC00052684B4B61EB02015A7A022A50D8494B47
:108ED000494C002A18BF23462C68984271F10001C2
:108EE00097F82A3034BF44F0005424F000542C602A
:108EF00093B12A200FF004FE002840D096F8A8373E
:108F0000002B43D0B6F89E2732B13C4BD6F8AC17B5
:108F10001B685B1A934239D224F0805438E096F8EB
:108F2000983724F400742C60002B7FF44DAF01209F
:108F300086F898071AF05EFD46E744F4002458E7E7
:108F400024F4000463E724F400647EE724F48054EE
:108F500084E724F400548DE724F4004491E724F4DA
:108F6000803496E724F400349BE724F08074A0E773
:108F7000234B204C033A012A88BF2346ACE7012348
:108F800086F8A8371D4B1B68C6F8AC3744F08054F0
:108F900000202C600FF0B4FD1A4B1C4216D0B8B163
:108FA00044F480442C602A681A4214BF0123002331
:108FB0005B0086F8B037F9F76FFED6F8B437C01A01
:108FC000002808DBBDE8F8431AF0E0BC0028EAD12D
:108FD00024F48044E6E7BDE8F88300BF785601201A
:108FE000D0E70020D8D600201457012070EF0020D1
:108FF000B46F002000171100407E0500542B0020A4
:1090000060CC050080FFFF7F2057012070B5454DE3
:109010002B685C0775D5444C84F8B807F9F73CFE1B
:1090200004F5F863C3E900012B68404A23F0040308
:109030002B6013683E4D23F0006313602B68190307
:1090400007D594F8C8370A2B5CD8082B64D8012BB5
:109050005AD8384EF36A1A0406D51420F7F7C0FC24
:10906000F36A23F40043F36294F8E037ABB3324B76
:10907000D4F8E4271B689B1A42F20F7293422CD952
:109080004FF47A72B3FBF2F3D4F8D4271344C4F844
:10909000D43733F0FFFBD4F8E837C01A6423B0FBB1
:1090A000F3F0D4F8D83718442B68C4F8D8079B07D6
:1090B00011D51FF0A9FC70B1D4F8F027D4F8EC3723
:1090C0009B1AD4F8DC271A44C4F8DC27D4F8F42718
:1090D0001A44C4F8F427FEF73BFF1BF071FE174853
:1090E000F3F707FF1648F3F704FF1648F3F701FFFD
:1090F0001548F3F7FEFE05201AF07CFC002384F8E7
:10910000A83770BD0B2BA4D00B4B1B68C4F8D0370D
:109110000B2384F8C8379CE70021FF2021F0F6FFDD
:10912000F2E700BF78560120D0E700201457012055
:109130001857012020570120542B0020D45801201B
:109140003459012094590120F4590120184B2DE97C
:10915000F04F1B68174FD3F828803B68164D174C0B
:10916000174E07EE908A2DED0C8BF8EEE77A9FED07
:10917000159AC5F8CC8667EE897A99B0CDE90201D7
:1091800013F00401C4EDCD7A20D10022002346E97A
:10919000022356E91023821A039860EB03030A485E
:1091A000904271EB03036AD2FFF7FAFC5AE000BF6A
:1091B0000C57012078560120D8D6002020570120D6
:1091C000D0EF0020BD37863520A10700C54B1B68B6
:1091D000D80606D536F012FB18B194F84033032BAD
:1091E00040D9C1497268D1F8003813EB080342EB4B
:1091F000E872C1F80038726056E90232BB4913EBDD
:10920000080342EBE87246E90232A1F1240300228E
:10921000F1EC017A93ED127AF4EEC77A93ED137ABA
:10922000F1EE10FAF4EEC77A48BFC3ED127A0132BC
:10923000F1EE10FAC8BFC3ED137A032A03F1080355
:10924000E6D194EDDD1AD4EDDC0A94EDDB0AF4F7F7
:10925000FAFAD4EDEA7AB4EEE70AF1EE10FA01DD9B
:1092600084EDEA0A56E90232A14999424FF000031F
:1092700093413FBF9B4A136823F00063136094F847
:1092800038300BB11FF0DAFEE369990707D53E6865
:1092900016F0100600F01A86012384F8AC33954BC3
:1092A000029A53E9026843F8082C039A43F8042C05
:1092B000E3699B0740F1D08694F8AC33002B00F0B3
:1092C000CB869FED8D7AD4ED107A8C489FED8C0A79
:1092D00067EE877A00F10C01C0ED007AD4ED117AC7
:1092E00067EE877AE838C0ED3B7AD4ED127A67EE04
:1092F000877AC0ED3C7A3CF08AF994EDDE0AF4F707
:109300008AF9F0EE408A94EDDF0AF4F784F9B0EEC2
:10931000408A94EDE00AF4F77EF995F83837062B89
:109320001DD1DFED787AD4F88833C5F8483768EE78
:10933000A78A28EE278AFDEEE88ABDEEC88A18EED5
:10934000902A20EE270AC5F83C27BDEEC00A18EE89
:10935000102AC5F8402710EE102AC5F84427029BB2
:10936000981B039B63EB080140F03EFF00EE100AE0
:1093700020EE090A10F0ACF994EDCD0A5A4EFEF732
:10938000CDFBFFF709FD95F834362BB1DDE902235B
:1093900096F810080FF060F996F81038002B00F0DE
:1093A000298132F0E1FF584B3A681B68D6F814184F
:1093B000C6F81438500713D55B1A07EE903A534A93
:1093C0009FED537AD2ED006AF8EEE77A02F540633A
:1093D00067EE877A93ED447AA6EEA77A83ED447A16
:1093E00034F034FD40B196F818382BB90E201AF03D
:1093F00001FB012386F81838464FFB7B2BB1162062
:109400000FF07EFB08B901233B7416200FF078FBA8
:10941000F87336F007FA32F06DFCDFF8FC803B7829
:10942000DFF8C0B0302202FB0383D3F890370093FB
:10943000E36A019313F4007F00F04286DBF800300A
:10944000590306D5009AD20444BF23F46053CBF8E5
:1094500000300023BB812F4C2F4AA3732378224F67
:10946000302101FB0322019BD2F8942723F48323AC
:1094700023F0B80343EA0208284B2E20C3F82C80BF
:109480000FF03EFB8146002801F07E8018F4006F4B
:1094900041F07A8034F02EFF002841F07580E28898
:1094A00040F202239A4208BF0E4BD7F8302808BF7B
:1094B00018684FF001036375134B1B68A3EB02039D
:1094C00008BFC0F34000B3F57A7F29D297F8B136D0
:1094D00033B3002384F8263EA4F8203E84F8253ECA
:1094E0001EE000BF14570120D0E700208C5A012055
:1094F00040420F00E0EF002035FA8E3C745B012003
:109500008F2A75440000C842542B00201099002077
:109510006F12833A109500208433060820570120EB
:1095200094F925AE002801F02480BAF1030F01F070
:109530002780DFF8608498F80A3043B913200FF0D1
:10954000DFFA80F00100C0B288F80A0010B1484686
:109550004FF0010A84F825AE002845D013200FF003
:10956000CFFA002840D094F9263E0BB933F0F6FE2E
:1095700032F042FC01460BA83DF0E0F994F9263E9A
:109580000B99142000FB03424FF0000CC2F8C014EA
:109590000C99C2F8C4140D99C2F8C814B2F8D014CA
:1095A000C2F8CCC441F00101A2F8D0144AF2015132
:1095B000A2F8D214012284F8202E23B15A1E00FBF7
:1095C000024282F8D3C401335BB2782B84F8263E82
:1095D00084F8233E84F8213E14BF0223032384F839
:1095E000253E002388F80A30002032F0E1FF63783E
:1095F000A7F83438DFF87093DFF89083002389F8F8
:10960000103899F8363809F6380A09F50864002B3D
:1096100041D1DAED0E7A9FEDD27A0023002277EE67
:10962000877AC4E92A23C4E90223C4E90C23C4E9E4
:10963000162398F8C537C4ED487A0027C4ED497A57
:10964000C4F83071C4F83471C4F83871C4F83C718E
:10965000C4F8CC700BB138F00BFAC24BE36363660D
:109660000123C4F8BC70C4F80871C4F81471C4F8BC
:10967000C070C4F80C71C4F81871C4F8C470C4F890
:109680001071C4F81C71A763276467642766A76616
:10969000E76686F83638F9F7FFFA0091D4E92AB17F
:1096A000009B01910746C4F8A870C4F8AC300FF0D5
:1096B000D1FF0199002840F075870023C4F8B0302D
:1096C000C4F8B430C4F8B83098F8C5370BB138F0E6
:1096D000CFF9D4E94001009B381A63EB010140F057
:1096E00083FD08EE100A28EE098A009B8DED0B8A97
:1096F000C4F80071C4F804310FF0ACFFDAED0EAA23
:109700000190002841F05A80DFED959A7AEEA99AEF
:109710008346F0EE698A944C0098D4F8E029D4F896
:10972000E439DFF87482DFF87492C4F880B8BA1AAA
:1097300060EB030344F62060824204F5086A73F18B
:109740000000CAED488ACAED499AC0F08C81C4F87D
:10975000EC39009BC4F8E079C4F8E829C4F8E4398E
:1097600026F0CCFCB8F93470002801F00086B4F97A
:10977000C06938F069F907EB870B06EB86034FEAFF
:109780004B0B7A4E5B00D8B1B27AC2B996F8482436
:10979000900714D0510712D4D6F8EC03D6F8581419
:1097A000ABEB00000844CDE90023F3F75DFD009A20
:1097B000019BC6F8580442F0040286F848240220AF
:1097C00007EE90BA9FED6A7AB072F8EEE77AC6E9D2
:1097D000FBB387EE878ADFED677A28EE278AB0EE43
:1097E000480AF3F7C1FB86EDFD0AB0EE480AF3F72D
:1097F0001DFC614B9AED427A93ED0EAADAED437AA5
:1098000086EDFE0AB4EEE8AAF1EE10FABDEEC7BA94
:10981000FDEEE7AA41F3AE85DAED458A9AED468A78
:10982000C6EDF07AF0EE480AB0EE680AC6EDF67AB8
:1098300086EDEF7AC6EDF28A86EDF38A86EDF57A4B
:10984000C6EDF88A86EDF98AF3F7F6FF4B4B4C49E3
:1098500083ED000A0223F37133720123B370494B85
:10986000FDEEE87A1B68C6F8203417EE903A47F60A
:10987000FF708342A8BF03468B42FDEEC87AB8BF93
:109880000B461AB217EE903A8342A8BF03468B42AA
:10989000B8BF0B461BB21BEE101AB4EEE9AAC4F80F
:1098A000F0191AEE901AF1EE10FA9AED440A9AEDB8
